:100000000C9414290C9404FC0C94D9FB0C94AEFBB6
:100010000C9483FB0C9458FB0C942DFB0C9402FB6A
:100020000C94D7FA0C9445290C9445290C94452935
:100030000C9445290C9405520C9445290C9445299F
:100040000C9445290C948E540C9445290C94452904
:100050000C9445290C9445290C94A3520C942FFC24
:100060000C9445290C943F5B0C9445290C9445292C
:100070000C9445290C9445290C9445290C94452948
:100080000C9445290C9445290C9445290C94452938
:100090000C9445290C9445290C9445290C94452928
:1000A0000C9445290C9445290C9445290C94452918
:1000B0000C9445290C9445290C9445290C94452908
:1000C0000C9445290C9445290C9445290C944529F8
:1000D0000C9445290C9445290C9445290C944529E8
:1000E0000C9445298E439143804384438A43C843FB
:1000F000954399439F43A343A743AD43B143B543BE
:10010000C843BB43BF43C343415345536E5372532C
:1001100054535F532E53735B795B8A5B955B9D5B96
:10012000B25BA15BB25BA55BA95BB25BAF5B2A8FE5
:100130002F8F348F3E8F488FC18F528F5A8F628F8F
:100140006C8F768F808F8F8F998FC18FA38FAD8F9C
:10015000B78FBFB4BFB4C6B4C6B4C6B4CDB4CDB403
:10016000CDB4DAB4D4B4D4B4D4B4084AD73B3BCE7B
:10017000016E84BCBFFDC12F3D6C74319ABD5683A6
:100180003DDA3D00C77F11BED9E4BB4C3E916BAA5E
:10019000AABE000000803F05A84CCDB2D44EB938AD
:1001A00036A9020C50B9918688083CA6AAAA2ABE94
:1001B000000000803F0020746F6F206C6F6E67201E
:1001C000657874727573696F6E2070726576656E8E
:1001D0007465640A0020636F6C64206578747275BE
:1001E00073696F6E2070726576656E7465640A005F
:1001F000536C6565702E2E2E004C756C7A426F74B0
:100200002054415A20352072656164792E00526570
:1002100073756D696E67207072696E7400436C69E6
:10022000636B20746F20726573756D652E2E2E00C2
:100230004E6F206D6F76652E00456E642066696C8A
:1002400065206C6973740A00426567696E2066698F
:100250006C65206C6973740A004D3132350053446B
:10026000207072696E74696E67206279746520000F
:100270004E6F74205344207072696E74696E670A01
:100280000046696C652064656C657465643A004479
:10029000656C6574696F6E206661696C65642C209D
:1002A00046696C653A20006F70656E206661696C06
:1002B00065642C2046696C653A2000256973002529
:1002C000696D20256973002569682025696D2025E1
:1002D000697300256964202569682025696D2025DA
:1002E00069730025697920256964202569682025BE
:1002F000696D20256973005072696E742074696D90
:10030000653A2000000125301D0CFF24311C0BFF35
:10031000232F1B0AFFFF040306080202222B1A41A7
:1003200042212A193F40033809FF3607FF372829A1
:100330004527444350726F74656374656420506947
:100340006E0A0045787472756465722025692025EF
:1003500073004C756C7A426F742054415A203520DA
:1003600072656164792E006F6B00436F6F6C696E0C
:100370006720646F6E652E0048656174696E672042
:10038000646F6E652E0020573A004578747275646C
:100390006572202569202573004C756C7A426F7454
:1003A0002054415A20352072656164792E004265DF
:1003B0006420646F6E652E0020573A004265642009
:1003C00068656174696E672E0042656420636F6FB3
:1003D0006C696E672E004C756C7A426F74205441C4
:1003E0005A2035204F66662E004361703A454D45D0
:1003F0005247454E43595F5041525345523A310A94
:10040000004361703A434153455F4C494748545F4C
:100410004252494748544E4553533A300A004361CB
:10042000703A544F47474C455F4C49474854533AFC
:10043000300A004361703A534F4654574152455F6A
:10044000504F5745523A300A004361703A4C455676
:10045000454C494E475F444154413A300A0043619C
:10046000703A5A5F50524F42453A300A0043617029
:100470003A4155544F4C4556454C3A300A00436179
:10048000703A5052494E545F4A4F423A310A004343
:1004900061703A50524F47524553533A300A004325
:1004A00061703A4155544F5245504F52545F544534
:1004B0004D503A310A004361703A454550524F4D14
:1004C0003A310A004649524D574152455F4E414D1F
:1004D000453A4D61726C696E20204649524D574134
:1004E00052455F56455253494F4E3A312E312E35C3
:1004F0002E36342045585452554445525F54595075
:10050000453A466C6578794475616C6C7920763231
:1005100020534F555243455F434F44455F55524C1E
:100520003A68747470733A2F2F636F64652E616C30
:100530006570686F626A656374732E636F6D2F6494
:100540006966667573696F6E2F4D41524C494E2036
:1005500050524F544F434F4C5F56455253494F4EA4
:100560003A312E30204D414348494E455F54595051
:10057000453A4C756C7A426F742054415A203520AC
:1005800045585452554445525F434F554E543A32A4
:1005900020555549443A63333235356339362D3465
:1005A0003039372D343838342D386564302D646552
:1005B000643266663962616536310A002F2F200089
:1005C0007A5F6D696E3A2000795F6D696E3A20003E
:1005D000785F6D696E3A20005265706F7274696E53
:1005E0006720656E6473746F7020737461747573C3
:1005F0000A0053657474696E672054726176656C85
:1006000020416363656C65726174696F6E3A2000A6
:1006100053657474696E67205265747261637420E7
:10062000416363656C65726174696F6E3A20005353
:10063000657474696E67205072696E7420416363DB
:10064000656C65726174696F6E3A200053657474ED
:10065000696E67205072696E7420616E64205472F6
:100660006176656C20416363656C65726174696F66
:100670006E3A2000205A00205900580020204D6179
:10068000783A2000205A00205900580020204D6957
:100690006E3A20004F6E20004F666600536F6674FE
:1006A00020656E6473746F70733A2000000000C0A0
:1006B00000000000000000004F6666736574732040
:1006C0006170706C696564004572723A20546F6F96
:1006D000206661722100546F6F206661722066721D
:1006E0006F6D207265666572656E636520706F69F7
:1006F0006E740A004E6F2063617365206C696768D1
:10070000740A004163746976652045787472756473
:1007100065723A2000556E6B6E6F776E20636F6D59
:100720006D616E643A202200434F4D4D554E494352
:100730004154494F4E0044525952554E0045525271
:100740004F525300494E464F004543484F0010005A
:10075000C90210012C014001220170011801B001F1
:100760000E01F00104015002FA00B002F000300363
:10077000E600D003DC009004D2007005C800A0069B
:10078000BE000008B400B009AA00D00BA000600EA3
:10079000960060118C000015820020197800C01DA1
:1007A0006E00A0226400B0275A00902C5000003147
:1007B0004600E0343C0010383200903A2800603C9B
:1007C0001E00A03D1400803E0A00203F00000000F3
:1007D00020002300260029002C002F0032000001F9
:1007E0000000030106010901000000C00000000034
:1007F0000000000000008F4300008A4300007A439D
:100800004D31343520533C696E6465783E206F75F8
:1008100074206F662072616E67652028302D312943
:100820000A00490744073D07360728076F66660038
:1008300044454255473A001000AD0330016A01506B
:10084000022B0170030A019004F500B005E500D009
:1008500006D800F007CE001009C500300ABE0050CF
:100860000BB700700CB100900DAB00B00EA600D01D
:100870000FA200F0109D0010129900301395005047
:1008800014920070158E0090168B00B0178700D060
:10089000188400F0198100101B7E00301C7B005072
:1008A0001D7900701E7600901F7300B0207000D07C
:1008B000216E00F0226B0010246900302566005084
:1008C0002663007027610090285E00B0295C00D08C
:1008D0002A5900F02B5600102D5400302E51005094
:1008E0002F4E0070304B0090314800B0324500D0A0
:1008F000334200F0343E0010363B003037370050B2
:1009000038330070392E00903A2900B03B2300D0D4
:100910003C1B00F03D1100103F0100F03F00004B78
:10092000494C4C45442E200024F4D43050C38E2032
:10093000C2A24017828B7011127A910D816CD90A74
:10094000A861E108C7586607615143061E4B5D0563
:10095000C145A7041A411104093D980371393103B7
:100960004036DB0265339102D4305402802E1D02E2
:10097000632CEE01752AC501B028A0011027810162
:100980008F2564012B244B01E0223401AC211F018F
:100990008D200D01801FFC00841EED00971DDF00DF
:1009A000B81CD200E61BC600201BBC00641AB200B3
:1009B000B219A8000A19A0006A189900D11791006D
:1009C00040178B00B516840031167E00B3157900F0
:1009D0003A157300C7146F0058146A00EE136600CE
:1009E0008813630025135E00C7125B006C1257006A
:1009F00015125400C111510070114F0021114B000C
:100A0000D61049008D1047004610440002104200E5
:100A1000C00F4000800F3E00420F3C00060F3B001D
:100A2000CB0E3800930E37005C0E3500270E3400D5
:100A3000F30D3200C10D3100900D3000600D2E001D
:100A4000320D2D00050D2C00D90C2B00AE0C290009
:100A5000850C29005C0C2700350C27000E0C2600A5
:100A6000E80B2400C40B2400A00B23007D0B230003
:100A70005A0B2100390B2100180B2000F80A1F0027
:100A8000D90A1E00BB0A1E009D0A1D00800A1D0017
:100A9000630A1C00470A1B002C0A1B00110A1A00DB
:100AA000F7091A00DD091900C4091900AB0919007A
:100AB000920917007B091800630917004C091600FA
:100AC00036091600200916000A091500F508150058
:100AD000E0081400CC081400B8081400A40814009E
:100AE000900813007D0812006B08130058081200CC
:100AF00046081200340811002308110012081100E2
:100B000001081100F0071000E0071000D0071000E6
:100B1000C0071000B0070F00A107100091070E00DA
:100B200083070F0074070F0065070E0057070E00BC
:100B300049070E003B070D002E070E0020070D0091
:100B400013070D0006070D00F9060C00ED060D0059
:100B5000E0060C00D4060C00C8060C00BC060C0015
:100B6000B0060C00A4060B0099060C008D060B00C5
:100B700082060B0077060B006C060B0061060A006C
:100B800057060B004C060A0042060A0038060A0007
:100B90002E060A0024060A001A060A00100609009A
:100BA00007060A00FD050900F4050900EB05090028
:100BB000E2050900D9050900D0050900C7050900AB
:100BC000BE050900B5050800AD050800A50509002A
:100BD0009C050800940508008C05080084050800A1
:100BE0007C050800740508006C0507006505080011
:100BF0005D050700560508004E050700470507007C
:100C00004005080038050700310507002A050700E0
:100C1000230507001C050600160507000F05070041
:100C20000805060002050700FB040600F50407009E
:100C3000EE040600E8040600E2040700DB040600F8
:100C4000D5040600CF040600C9040600C30406004C
:100C5000BD040600B7040600B1040500AC0406009C
:100C6000A6040600A00405009B04060095040500E8
:100C7000900406008A04050085040500800406002F
:100C80007A04050075040500700405006B04050076
:100C900066040500610405005C04050057040500B6
:100CA000520405004D0405004804050043040500F6
:100CB0003E0404003A040500350405003004040035
:100CC0002C04050027040400230405001E0404006E
:100CD0001A04040016040500110404000D040400A5
:100CE000090405000404040000040400FC030400DB
:100CF000F8030400F4030400F0030400EC03040010
:100D0000E8030400E4030400E0030400DC0304003F
:100D1000D8030400D4030400D0030400CC0304006F
:100D2000C8030300C503030024F404D9201BC40C2A
:100D30005C0E9804C4095F0265077101F405F900AF
:100D4000FB04B30048048700C10369005803550041
:100D500003034500BE023A008402310053022A0018
:100D60002902250004022000E4011C00C80119002A
:100D7000AF011700980114008401130071011000E5
:100D80006101100051010E0043010D0036010B00FE
:100D90002B010B0020010B00150109000C010900BB
:100DA00003010800FB000800F3000800EB00070047
:100DB000E4000600DE000600D8000600D2000600AF
:100DC000CC000500C7000500C2000500BD000400FE
:100DD000B9000400B5000400B1000400AD00040037
:100DE000A9000400A5000300A20003009F00040066
:100DF0009B0003009800030095000200930003008D
:100E0000900003008D0002008B00030088000200A8
:100E10008600020084000300810002007F000200BF
:100E20007D0002007B0002007900020077000100D3
:100E300076000200740002007200010071000200DE
:100E40006F0002006D0001006C0002006A000100EA
:100E500069000200670001006600010065000100F2
:100E600064000200620001006100010060000100F6
:100E70005F0002005D0001005C0001005B000100FA
:100E80005A000100590001005800010057000100FC
:100E900056000100550001005400010053000000FD
:100EA00053000100520001005100010050000100F8
:100EB0004F0001004E0000004E0001004D000100F7
:100EC0004C0001004B0000004B0001004A000100F3
:100ED00049000100480000004800010047000100EF
:100EE00046000000460001004500000045000100EA
:100EF00044000100430000004300010042000000E4
:100F000042000100410000004100010040000100DA
:100F10003F0000003F0001003E0000003E000100D5
:100F20003D0000003D0001003C0000003C000000CE
:100F30003C0001003B0000003B0001003A000000C3
:100F40003A000100390000003900010038000000BB
:100F500038000000380001003700000037000100B1
:100F600036000000360000003600010035000000A9
:100F7000350000003500010034000000340000009E
:100F80003400010033000000330000003300010092
:100F90003200000032000000320001003100000089
:100FA000310000003100010030000000300000007E
:100FB000300001002F0000002F0000002F00000073
:100FC0002F0001002E0000002E0000002E00010066
:100FD0002D0000002D0000002D0000002D0001005C
:100FE0002C0000002C0000002C0000002C00010050
:100FF0002B0000002B0000002B0000002B00010044
:101000002A0000002A0000002A0000002A00010037
:10101000290000002900000029000000290000002C
:10102000290001002800000028000000280000001E
:101030002800000028000100270000002700000011
:101040002700000027000000270001002600000004
:1010500026000000260000002600000026000100F7
:1010600025000000250000002500000025000000EC
:1010700025000000250001002400000024000000DD
:1010800024000000240000002400010023000000D0
:1010900023000000230000002300000023000000C4
:1010A00023000000230001002200000022000000B5
:1010B00022000000220000002200000022000100A7
:1010C000210000002100000021000000210000009C
:1010D000210000002100000021000100200000008C
:1010E0002000000020000000200000002000000080
:1010F0002000000020000000200001001F00000070
:101100001F0000001F0000001F0000001F00000063
:101110001F0000001F0001001E0000001E00000054
:101120001E0000001E0000004D38342058205920B9
:101130005A2045004572723A204D494E54454D5053
:1011400020424544004D494E54454D50207472692B
:10115000676765726564004572723A204D494E5466
:10116000454D50204531004572723A204D494E544C
:10117000454D50204530004572723A204D4158543B
:10118000454D5020424544004D415854454D502056
:10119000747269676765726564004572723A204DC2
:1011A000415854454D50204531004572723A204D0A
:1011B000415854454D50204530000201050800FFBC
:1011C000060121023520FFFF07FF06FF090050221C
:1011D0001656808080800080153353A0A0A002574F
:1011E000575050F850F850500257572070A07028B0
:1011F000702013355580A040A02002475740A0A082
:1012000040A0A05025135380808012265640808035
:1012100080804012265680404040408002455590D4
:1012200060F060900255552020F820201133536063
:101230004080044151F011335340E04002465610C3
:10124000102040808012365640A0A0A0A040123648
:101250005640C0404040E00246566090106080F02A
:10126000024656F020601090600246562060A0F0C2
:101270002020024656F080E01090600246566080C2
:10128000E0909060024656F0102020404002465602
:10129000609060909060024656609090701060126E
:1012A0002555C0C000C0C011365660600060408047
:1012B000123656204080804020034353F000F01245
:1012C000365680402020408012365640A0204000F4
:1012D00040015858304898A8A890403002465660BF
:1012E0009090F09090024656E090E09090E0024698
:1012F00056609080809060024656E090909090E01A
:10130000024656F080E08080F0024656F080E08091
:101310008080024656609080B09060024656909061
:10132000F0909090123656E040404040E002465621
:1013300070202020A04002465690A0C0A0A090029D
:1013400046568080808080F002465690F0F0909063
:101350009002465690D0F0B0B09002465660909001
:10136000909060024656E09090E080800147576080
:101370009090D0B06010024656E09090E0909002BD
:101380004656609040209060123656E04040404003
:1013900040024656909090909060024656909090F1
:1013A000906060024656909090F0F0900246569001
:1013B0009060609090025656888850202020024607
:1013C00056F010204080F0123656E080808080E099
:1013D000024656808040201010123656E020202011
:1013E00020E016325240A0014151F01622528040B6
:1013F000024454709090700246568080E09090E0D5
:1014000012345460808060024656101070909070C4
:1014100002445460B0C060024656205040E0404054
:1014200001455560907010600246568080E09090B3
:10143000901236564000C04040E01137572000203F
:101440002020A040024656808090E09090123656B0
:10145000C040404040E0025454D0A8A8A8024454E0
:10146000E090909002445460909060014555E09067
:10147000E080800145557090701010024454A0D057
:10148000808012345460C020C00246564040E04084
:10149000502002445490909070123454A0A0A04068
:1014A00002545488A8A850024454906060900145AA
:1014B000559090709060024454F02040F0024757DD
:1014C000304020C0204030221656808080808080AE
:1014D000024757C02040304020C006425250A0FF73
:1014E000FFFFFFFFFFFFFFFFFFFFFFFFFFFFFFFF0C
:1014F000FFFFFFFFFFFFFFFFFFFFFFFFFFFFFFFFFC
:1015000009005022165680008080808001465620B7
:1015100070A0A070200246562050E04050A0025516
:101520005588705070880256568850F820F820224E
:101530001757808080008080800247577080E0903D
:101540007010E0173151A002565670A8C8C8A87094
:1015500014355560A06000E003435350A05012338F
:1015600053E02020143151E002565670E8D8E8D8F4
:1015700070173151E015335340A04012355540E00B
:101580004000E014355540A02040E0143555C020FF
:10159000C020C01622524080014555909090E080B6
:1015A00002565678E8E86828282411518011225202
:1015B000408014355540C04040E014355540A040AF
:1015C00000E0034353A050A0024757808080A060F2
:1015D000F0200247578080A0D0102070024757802B
:1015E000408060A0F02012365640004080A04002AB
:1015F000475740206090F0909002475720406090FD
:10160000F0909002475760906090F090900247579A
:1016100050A06090F0909002475790006090F0903A
:101620009002475760906090F0909002465670A0EC
:10163000A0F0A0B0014757609080809060400247C2
:10164000574020F080E080F00247572040F080E0D3
:1016500080F00247576090F080E080F0024757909A
:1016600000F080E080F01237578040E0404040E0DA
:101670001237572040E0404040E012375740A0E08A
:10168000404040E0123757A000E0404040E00256A2
:10169000567048E848487002475750A090D0B09024
:1016A000900247574020609090906002475720403A
:1016B00060909090600247576090609090906002B8
:1016C000475750A0609090906002475790006090FC
:1016D000909060123353A040A002465670B0B0D034
:1016E000D0E00247574020909090906002475720EA
:1016F00040909090906002475760909090909060DA
:1017000002475790009090909060025757102088A1
:101710005020202002465680E09090E080024656FD
:101720006090A0A090A00247574020007090907059
:101730000247572040007090907002475720500099
:101740007090907002475750A000709090700246C1
:101750005650007090907002475760906070909063
:1017600070025454F068B078113555608080604044
:1017700002475740200060B0C06002475720400039
:1017800060B0C06002475760900060B0C060024621
:1017900056500060B0C060123757804000C04040D3
:1017A000E0123757204000C04040E012375740A0B9
:1017B00000C04040E0123656A000C04040E0024762
:1017C00057A040A01070906002475750A000E090D2
:1017D0009090024757402000609090600247572049
:1017E0004000609090600247576090006090906069
:1017F00002475750A00060909060024656900060EB
:101800009090601235554000E0004002445470B0A2
:10181000D0E0024757402000909090700247572038
:1018200040009090907002475760900090909070A8
:1018300002465690009090907001485820400090C9
:10184000907090600147578080E090E08080014771
:10185000579000909070906001050700FE0500FB16
:1018600001F220FFFE05FE05FE0200400215258064
:1018700080800080053242A0A002556550F850F8E3
:10188000500146562070C030E0200255659010206F
:101890004048025565608068906805122280800289
:1018A00025354080808040022535804040408004BE
:1018B0003343A040A003334340E040012232408044
:1018C000043141E00211218002556508102040805A
:1018D0000245556090909060022535C040404040E0
:1018E000024555E0106080F0024555E0106010E0C0
:1018F0000245552060A0F020024555F080E010E040
:101900000245556080E09060024555F0102040404F
:10191000024555609060906002455560907010607F
:101920000313238000800214248000808002354548
:101930002040804020033343E000E00235458040F2
:10194000204080024555E0106000400255657088D7
:10195000B8A870024555609090F090024555E0900F
:10196000E090E00235456080808060024555E0905F
:101970009090E0023545E080E080E0023545E0806F
:10198000E080800245557080B0907002455590907F
:10199000F09090023545E0404040E002455530105F
:1019A00010906002455590A0C0A0900235458080FF
:1019B0008080E002556588D8A8888802455590D077
:1019C000B090900245556090909060024555E0902F
:1019D00090E080014656609090906010024555E07E
:1019E0009090E09002455570806010E0023545E02F
:1019F000404040400245559090909060024555907F
:101A000090A0A04002556588A8A8A850024555900E
:101A1000906090900245559090701060023545E0BE
:101A2000204080E0022535C0808080C0025565805E
:101A300040201008022535C0404040C005324240D9
:101A4000A0024151F005223280400244547090902F
:101A50007002455580E09090E002344460808060E0
:101A6000024555107090907002445460B0C06002FE
:101A700035452040E0404000465670909070106020
:101A800002455580E090909002152580008080806E
:101A9000002737400040404040800245558090A0DC
:101AA000E0900215258080808080025464F0A8A810
:101AB000A8024454E09090900244546090906000DA
:101AC0004656E09090E080800046567090907010EE
:101AD00010023444A0C0808002445470C030E00240
:101AE000354540E0404020024454909090700244BC
:101AF000549090A040025464A8A85050023444A0CE
:101B00004040A0004656909090701060024454F0FF
:101B10002040F002354560408040600215258080FD
:101B2000808080023545C0402040C005425250A010
:101B3000FFFFFFFFFFFFFFFFFFFFFFFFFFFFFFFFB5
:101B4000FFFFFFFFFFFFFFFFFFFFFFFFFFFFFFFFA5
:101B5000FF020040FFFFFFFFFFFFFFFFFFFFFFFF50
:101B6000FFFFFFFFFFFFFFFFFFFFFFFFFFFFFFFF85
:101B7000FFFFFFFFFFFFFFFFFFFFFFFFFFFFFFFF75
:101B8000FFFFFFFFFFFFFFFFFFFFFFFFFFFFFFFF65
:101B9000FFFFFFFFFFFFFFFFFFFFFFFFFFFFFFFF55
:101BA000FFFFFFFFFFFFFFFFFFFFFFFFFFFFFFFF45
:101BB000FFFFFF01060D00FE09016602D620FFFEB1
:101BC0000BFE0AFE0D0060221969808080808080F3
:101BD000800080183363A0A0A00357675050F850CE
:101BE000F850500259692078A0A0702828F02002EF
:101BF000596948A85010204050A89002586840A049
:101C0000A040A0989068281363808080113B6B20CF
:101C100040408080808080404020113B6B8040406D
:101C2000202020202040408006556520A870A82054
:101C30000455652020F82020113363604080065150
:101C400061F811336340E040025969080810102020
:101C500040408080025969205088888888885020B8
:101C60000259692060A02020202020F802596970C4
:101C700088880810204080F8025969F80810207000
:101C800008088870025969101030505090F81010F0
:101C9000025969F88080B0C80808887002596970D4
:101CA000888080F088888870025969F808101020B0
:101CB0002040404002596970888888708888887000
:101CC00002596970888888780808887011386840D7
:101CD000E040000040E04011386840E04000006013
:101CE00040800259690810204080402010080454A8
:101CF00064F80000F8025969804020100810204064
:101D000080025969708888081020200020025969D3
:101D100070888898A8A8B08078025969205088886F
:101D200088F8888888025969F048484870484848C7
:101D3000F0025969708880808080808870025969BB
:101D4000F048484848484848F0025969F88080807F
:101D5000F0808080F8025969F8808080F08080806F
:101D600080025969708880808098888870025969DB
:101D700088888888F888888888123969E0404040D7
:101D800040404040E0025969381010101010109087
:101D900060025969888890A0C0A09088880259691B
:101DA0008080808080808080F80259698888D8A8E7
:101DB000A88888888802596988C8C8A8A898988877
:101DC000880259697088888888888888700259696B
:101DD000F0888888F080808080015A6A70888888BE
:101DE000888888A87008025969F0888888F0A090CF
:101DF0008888025969708880807008088870025944
:101E000069F8202020202020202002596988888815
:101E100088888888887002596988888888505050D6
:101E2000202002596988888888A8A8A8A850025943
:101E30006988885050205050888802596988885095
:101E4000502020202020025969F80810102040401E
:101E500080F8113B6BE0808080808080808080E013
:101E6000025969808040402010100808113B6BE047
:101E7000202020202020202020E0085363205088AC
:101E8000015161F82A226280400256667008788803
:101E90009868025969808080F088888888F00256A6
:101EA0006670888080887002596908080878888878
:101EB0008888780256667088F88088700259693080
:101EC000484040F04040404000586870888888781A
:101ED000088870025969808080B0C8888888881214
:101EE00038684000C040404040E0004A6A1000307E
:101EF0001010101090906002596980808090A0C0EE
:101F0000A09088123969C040404040404040E00203
:101F10005666D0A8A8A8A888025666B0C88888883F
:101F200088025666708888888870005868F08888AB
:101F300088F0808080005868788888887808080849
:101F4000025666B0C8808080800256667088601035
:101F500088700258684040F0404040483002566661
:101F60008888888898680256668888885050200239
:101F700056668888A8A8A850025666885020205027
:101F8000880058688888889868088870025666F8BB
:101F900010204080F8015B6B1820202020C02020FA
:101FA00020201822196980808080808080808001B4
:101FB0005B6BC0202020201820202020C008536305
:101FC00048A890FFFFFFFFFFFFFFFFFFFFFFFFFF9E
:101FD000FFFFFFFFFFFFFFFFFFFFFFFFFFFFFFFF11
:101FE000FFFFFFFF0D006022196980008080808064
:101FF0008080800358682070A8A0A0A87020025993
:102000006930484040E0404048B003566688705010
:1020100050708802596988885050F820F820202292
:102020001969808080800080808080124A6A609078
:1020300080609090601090601A3262A0A00359698D
:102040007088A8D8C8D8A88870045767700878889E
:102050007800F80356662850A0A05028045363F86F
:102060000808163161E00359697088E8D8D8E8D8C3
:1020700088700A5161F81744646090906003576754
:102080002020F8202000F807356540A02040E00718
:10209000356540A04020C02A2262408000586888F0
:1020A00088888898E8808002596978E8E8E8E868D4
:1020B000282828262161C0202262408007356540FB
:1020C000C04040E0045767708888887000F8035665
:1020D00066A050282850A0025A6A40C04040E0083C
:1020E00018283808025A6A40C04040E010280810FA
:1020F00038025A6A40A04020A048182838080259DF
:1021000069200020204080888870025A6A402000A0
:1021100020508888F88888025A6A10200020508849
:1021200088F88888025A6A30480020508888F888E1
:1021300088025A6A28500020508888F88888025AF5
:102140006A50500020508888F88888025A6A2050C7
:102150002020508888F8888802596958A0A0A0B02B
:10216000E0A0A0B8005B6B70888080808080887061
:102170002040025A6A402000F88080F08080F802F7
:102180005A6A102000F88080F08080F8025A6A3085
:102190004800F88080F08080F8025A6A505000F8B9
:1021A0008080F08080F8123A6A804000E040404031
:1021B0004040E0123A6A204000E04040404040E0A9
:1021C000124A6A609000E04040404040E0123A6AA3
:1021D000A0A000E04040404040E0025969F048487B
:1021E00048E8484848F0025A6A2850008888C8A839
:1021F000988888025A6A4020007088888888887089
:10220000025A6A10200070888888888870025A6A8A
:1022100030480070888888888870025A6A28500080
:1022200070888888888870025A6A50500070888840
:10223000888888700355658850205088015B6B083A
:10224000709898A8A8A8C8C87080025A6A40200050
:1022500088888888888870025A6A10200088888850
:1022600088888870025A6A304800888888888888F8
:1022700070025A6A50500088888888888870025A8C
:102280006A1020008888502020202002596980F0A0
:10229000888888F0808080025969609090A0A09022
:1022A0008888B002596940200070087888986802D0
:1022B0005969102000700878889868025969304878
:1022C000007008788898680259692850007008786A
:1022D0008898680259695050007008788898680298
:1022E0005A6A3048300070087888986802566670DC
:1022F0002870A0A85000586870888080887020409E
:102300000259694020007088F8808870025969106D
:1023100020007088F8808870025969304800708801
:10232000F88088700259695050007088F880887071
:10233000123969804000C040404040E012396920B5
:102340004000C040404040E0124969609000C040F9
:10235000404040E0123969A0A000C040404040E049
:10236000025A6A5020601070888888887002596903
:10237000285000B0C88888888802596940200070B9
:102380008888888870025969102000708888888839
:1023900070025969304800708888888870025969CD
:1023A00028500070888888887002596950500070E1
:1023B0008888888870035767202000F80020200153
:1023C0005868087098A8A8C8708002596940200011
:1023D00088888888986802596910200088888888C9
:1023E0009868025969304800888888889868025936
:1023F00069505000888888889868005B6B102000BE
:102400008888889868088870005A6A8080B0C88870
:1024100088C8B08080005B6B5050008888889868BE
:1024200008887000000000000000000000000000AC
:10243000000000000000000000000000000000009C
:102440000000000000000C000000000000000C0074
:102450000000000000001200000000000000230047
:1024600000000000000021000000000000004C807F
:102470000000000000005E800000000000009240AC
:10248000000000000000A140000000000001212029
:102490000000000000027F90000000000002001019
:1024A000000000000007FFF8000000000004000822
:1024B0000000000000080004000000000008000602
:1024C00000000000001000020000000000301E01AB
:1024D0000000000000207F81000000000041FFE0BC
:1024E000800000000043FCF08000000000873B7883
:1024F00040000000018EDBFC60000000010FEBCC0F
:1025000020000000021FEDB610000000021FDEB622
:10251000100000000439CD7F080000000436E0FF01
:1025200008000000087EC0BB84000000187F005D2A
:1025300086000000107FC0ED82000000203CC073C8
:1025400001000000203B337F01000000701BE77E8C
:1025500003800000C81DEEDE04C00000880FDEDC32
:1025600004400001240FDF3C092000012607DBF8AE
:10257000192000027203E7F0139000025101FFE0FE
:102580002290000489007F802448000904801E00F6
:102590004824000BFE400000DFF400100040000063
:1025A0008002001FFFFFFFFFFFFE00000000000091
:1025B000000000000000000000000000000000001B
:1025C0000000001022103C3C0E1F001022100422BC
:1025D0001104001022100822110400102210083CDF
:1025E00011040010221010221104001022102022C9
:1025F0001104001E1C1E3C3C0E04000000000000E4
:1026000000000000000000000000000000000000CA
:1026100000000000000000000000000000000000BA
:1026200000000000000000000000000000000000AA
:10263000000000000000000000000000000000009A
:10264000000000000000000000000000000000008A
:10265000000000000000000000000000000000007A
:10266000002040002042403A0020403A004D6F7662
:10267000652058004D6F76652059004D6F766520B6
:102680005A004578747275646572320045787472C8
:1026900075646572310020496E76616C69642065ED
:1026A000787472756465722000204400204900200F
:1026B000204D333034205000204400204900202099
:1026C0004D3330312050002044002049002050007C
:1026D00020204D333031204500504944207365742B
:1026E00074696E67733A0A00204600204200204851
:1026F0000020204D3134352053004D6174657269DE
:10270000616C2068656174757020706172616D65BF
:10271000746572733A0A0020590020580020204D39
:10272000323138205400486F74656E64206F6666DD
:10273000736574733A0A00205A0020590020204D16
:10274000323036205800486F6D65206F66667365BD
:10275000743A0A00204500205A00205900205800F1
:1027600020420020540020204D32303520530041BB
:102770006476616E6365643A20533C6D696E5F6692
:10278000656564726174653E20543C6D696E5F746A
:10279000726176656C5F66656564726174653E2022
:1027A000423C6D696E5F7365676D656E745F7469D9
:1027B0006D655F6D733E20583C6D61785F78795F21
:1027C0006A65726B3E205A3C6D61785F7A5F6A651C
:1027D000726B3E20453C6D61785F655F6A65726B28
:1027E0003E0A0020540020520020204D3230342078
:1027F0005000416363656C65726174696F6E202877
:10280000756E6974732F7332293A20503C70726967
:102810006E745F616363656C3E20523C72657472D6
:102820006163745F616363656C3E20543C747261E4
:1028300076656C5F616363656C3E0A00204500202D
:10284000204D323031205400205A002059002020E1
:102850004D3230312058004D6178696D756D2041E1
:102860006363656C65726174696F6E2028756E694B
:1028700074732F7332293A0A0020450020204D320C
:102880003033205400205A0020590020204D32308F
:10289000332058004D6178696D756D2066656564FB
:1028A00072617465732028756E6974732F73293A89
:1028B0000A0020450020204D3932205400205A00C3
:1028C00020590020204D3932205800537465707310
:1028D0002070657220756E69743A0A0020204D32AE
:1028E00030302044300A0020204D32303020543126
:1028F00020440020204D32303020440020446973B1
:1029000061626C65640A0046696C616D656E742075
:1029100073657474696E67733A0020204D313439E1
:102920002043203B20556E69747320696E204365F7
:102930006C736975730A00202047323120202020F3
:102940003B20556E69747320696E206D6D0A0029F5
:102950000A002062797465733B2063726320005320
:10296000657474696E67732053746F726564202890
:102970000045313A200045303A20005A3A200059AB
:102980003A2000583A20004D53312C4D53322050FC
:10299000696E730A002042002050006F6B00526580
:1029A00073656E643A200043290A0061626C6564B5
:1029B00020286D696E2074656D702000436F6C6413
:1029C00020657874727564657320617265200020DB
:1029D000643A0020693A0020703A0020643A0020EE
:1029E000693A0020703A00202863616C63756C615D
:1029F00074656429210A0020213D2000454550527C
:102A00004F4D20435243206D69736D61746368209C
:102A10002D202873746F726564292000290A002014
:102A200062797465733B2063726320002073746F56
:102A30007265642073657474696E6773207265745F
:102A4000726965766564202800204D61726C696E3C
:102A50003D563430290A0028454550524F4D3D001F
:102A6000454550524F4D2076657273696F6E206DEB
:102A700069736D617463682000526573746F726569
:102A8000206661696C73616665004D3530320A4DB0
:102A9000353030004C6F61642073657474696E6703
:102AA000730053746F72652073657474696E677315
:102AB00000416476616E6365642053657474696E69
:102AC0006773004D61696E005072696E74206162B7
:102AD0006F727465640041626F7574204669726D2F
:102AE00077617265004E6F20534420636172640009
:102AF0005072696E742066726F6D20534400537477
:102B00006F70207072696E7400526573756D652008
:102B10007072696E74005061757365207072696EB1
:102B200074004368616E67652066696C616D656EEF
:102B300074204532004368616E67652066696C6188
:102B40006D656E7420453100436F6E6669677572FE
:102B50006174696F6E0054656D7065726174757231
:102B600065004D6F76656D656E740054756E650019
:102B7000496E666F2073637265656E00506C6561A7
:102B80007365207265736574005052494E54455206
:102B90002048414C544544005072696E746572205F
:102BA00068616C7465642E206B696C6C28292063E5
:102BB000616C6C6564210A006265640A002C2073F4
:102BC000797374656D2073746F707065642120482B
:102BD00065617465725F49443A2000544845524D1E
:102BE000414C2052554E41574159204245440054D2
:102BF0006865726D616C2052756E61776179005401
:102C00004845524D414C2052554E4157415920455F
:102C10003100544845524D414C2052554E41574188
:102C2000592045300048656174696E6720666169A6
:102C30006C6564204245440048656174696E672094
:102C40006661696C65640048656174696E672066D9
:102C500061696C65640048656174696E67206661CE
:102C6000696C65642045310048656174696E672050
:102C70006661696C65642045300057726974696EDD
:102C80006720746F2066696C653A20006F70656E0E
:102C9000206661696C65642C2046696C653A200089
:102CA0006F70656E206661696C65642C2046696C86
:102CB000653A200046696C652073656C65637465D0
:102CC000640A002053697A653A200046696C6520E1
:102CD0006F70656E65643A20006F70656E20666186
:102CE000696C65642C2046696C653A200020666931
:102CF0006C653A20004E6F7720002220706F7300C1
:102D00002220706172656E743A2200535542524F10
:102D10005554494E452043414C4C207461726765BF
:102D2000743A22004B494C4C45442E200074727971
:102D3000696E6720746F2063616C6C207375622DFF
:102D400067636F64652066696C6573207769746872
:102D500020746F6F206D616E79206C6576656C7381
:102D60002E204D4158206C6576656C2069733A00C1
:102D700053442063617264206F6B0A006F70656E4C
:102D8000526F6F74206661696C65640A00766F6CBF
:102D9000756D652E696E6974206661696C65640A7B
:102DA00000534420696E6974206661696C0A007C76
:102DB0003C3E5E2B3D3F2F5B5D3B2C2A225C00435B
:102DC000616E6E6F74206F70656E207375626469DA
:102DD00072200000060900FE06018902FE20FFFEA7
:102DE00007FE06FE000000060007010606060200B8
:102DF000808080800080030303060103A0A0A0055B
:102E000007070600FF5050F850F850500509090612
:102E100000FE2070A8A07028A870200608080600F0
:102E2000FF40A84810204854080507070600FF6027
:102E300090906098906801030306020380808002EE
:102E400007070602FF408080808080400207070657
:102E500002FF804040404040800505050600008894
:102E600050F850880505050600002020F8202002B3
:102E700004040602FEC0404080050101060002F87D
:102E8000020202060200C0C004060606010010107D
:102E900020408080040606060100609090909060BB
:102EA00003060606010040C0404040E00406060656
:102EB00001006090102040F0040606060100F0209A
:102EC000601010E005060606000010305090F81063
:102ED000040606060100F080E01010E00406060675
:102EE00001006080E0909060040606060100F0108A
:102EF000102040400406060601006090609090603B
:102F00000406060601006090907010600205050638
:102F10000200C0C000C0C00207070602FEC0C00019
:102F2000C040408005050506000018608060180557
:102F30000303060001F800F8050505060000C0308F
:102F40000830C00407070601006090106040004090
:102F50000506060600007090A8B0807005060606FB
:102F60000000205088F88888050606060000F088D2
:102F7000F08888F00406060601006090808090606A
:102F8000040606060100E090909090E00406060614
:102F90000100F080E08080F0040606060100F08069
:102FA000E0808080040606060100609080B090609A
:102FB0000406060601009090F09090900306060625
:102FC0000100E040404040E00506060600003810E1
:102FD0001010906004060606010090A0C0A090901A
:102FE0000406060601008080808080F00506060643
:102FF000000088D8A8A8888804060606010090D09A
:10300000B090909005060606000070888888887049
:10301000040606060100E09090E0808004070706A1
:1030200001FF609090D0B06010040606060100E039
:103030009090E09090040606060100609040209079
:1030400060050606060000F8202020202004060661
:103050000601009090909090600406060601009092
:103060009090F060600506060600008888A8A8D841
:1030700088050606060000885020205088050606B0
:10308000060000888850202020040606060100F073
:1030900010204080F0030606060100E0808080805A
:1030A000E00406060601008080402010100306069A
:1030B000060100E020202020E00503030600032095
:1030C00050880501010600FEF80202020602048093
:1030D0004004040406010070909070040606060186
:1030E000008080E09090E00404040601007080807D
:1030F000700406060601001010709090700404041D
:1031000006010060B0C070040606060100205040B1
:10311000E040400406060601FE60909070106004D6
:1031200006060601008080E09090900306060601E6
:10313000004000C04040E00308080601FE20006097
:10314000202020A0400406060601008080A0C0A028
:1031500090030606060100C040404040E00504041C
:10316000060000D0A8A888040404060100E090909E
:1031700090040404060100609090600406060601B5
:10318000FEE09090E080800406060601FE709090BC
:10319000701010040404060100A0D0808004040410
:1031A00006010070C030E00406060601004040E061
:1031B0004050200404040601009090907004040420
:1031C0000601009090606005040406000088A8A82D
:1031D0005004040406010090606090040606060195
:1031E000FE909090709060040404060100F020406E
:1031F000F0030707060100204040804040200107FF
:10320000070602FF80808080808080030707060118
:10321000008040402040408004020206010350A08C
:10322000FFFFFFFFFFFFFFFFFFFFFFFFFFFFFFFFAE
:10323000FFFFFFFFFFFFFFFFFFFFFFFFFFFFFFFF9E
:10324000FF0000000600070106060602008000805D
:103250008080800406060601FF2070A0A070200573
:1032600007070600FF304840F04040F80505050616
:103270000000A8508850A80506060600008850F8EF
:1032800020F8200107070602FF80808000808080F0
:103290000407070601FF708060906010E0030101E1
:1032A000060105A0060707060000788494A494840C
:1032B0007803050506010160A06000E0050505062C
:1032C00000002850A05028040303060100F010104D
:1032D000040101060102F00607070600007884B425
:1032E000A4A48478040101060105F0040303060187
:1032F000026090600507070600FF2020F8202000EC
:10330000F803050506010140A02040E0030505067D
:103310000101C0204020C0020202060204408004D5
:1033200005050601FF9090B0D08005060606000056
:1033300078E8E868282801010106020280020202FA
:103340000602FE408003050506010140C04040E042
:1033500003050506010140A04000E0050505060043
:1033600000A0502850A00508080600FF40C04050AB
:10337000703078100508080600FF40C0405068080B
:1033800010380508080600FFC0204030F0307810E3
:1033900004070706010020002060809060050707F1
:1033A00006000040202050708888050707060000AE
:1033B0001020205070888805070706000020502044
:1033C0005070888805070706000028502050708834
:1033D0008805070706000050002050708888050700
:1033E0000706000020502050708888050606060059
:1033F0000078A0F0A0A0B80408080601FE60908044
:1034000080906020400407070601004020F080E023
:1034100080F00407070601002040F080E080F004FF
:1034200007070601002050F080E080F0040707063F
:1034300001005000F080E080F003070706010080E3
:1034400040E0404040E00307070601002040E04024
:103450004040E003070706010040A0E0404040E094
:10346000030707060100A000E0404040E005060613
:103470000600007048E8484870040707060100503D
:10348000A090D0B090900407070601004020609003
:1034900090906004070706010020406090909060C3
:1034A0000407070601002050609090906004070711
:1034B00006010050A060909090600407070601008C
:1034C000500060909090600505050600008850202F
:1034D00050880408080601FF1070B0B0D0D0E0801A
:1034E00004070706010040209090909060040707B1
:1034F00006010020409090909060040707060100AC
:1035000020509090909060040707060100500090B2
:10351000909090600507070600001020885020203A
:103520002004060606010080E09090E08004060674
:103530000601006090A0A090A004070706010040CB
:103540002000709090700407070601002040007072
:103550009090700407070601002050007090907052
:1035600004070706010050A0007090907004060642
:1035700006010050007090907004070706010020BB
:1035800050207090907005040406000070A8B07878
:103590000406060601FE70808070204004070706BE
:1035A000010040200060B0C0700407070601002041
:1035B000400060B0C07004070706010020500060A2
:1035C000B0C070040606060100500060B0C0700371
:1035D0000707060100804000C04040E003070706DF
:1035E0000100204000C04040E00307070601004002
:1035F000A000C04040E0030606060100A000C04055
:1036000040E00407070601003060107090906004ED
:10361000070706010050A000E090909004070706FD
:103620000100402000609090600407070601002020
:103630004000609090600407070601002050006081
:1036400090906004070706010050A0006090906011
:10365000040606060100500060909060050505060E
:1036600000002000F8002004040406010070B0D01F
:10367000E0040707060100402000909090700407C6
:103680000706010020400090909070040707060193
:103690000020500090909070040606060100500033
:1036A000909090700409090601FE204000909090CF
:1036B0007090600408080601FE8080E09090E08031
:1036C000800408080601FE50009090907090600001
:1036D000002200250028002B002E003100340002BB
:1036E000010000050108010B0100000A0B02090C92
:1036F0000D0E080703040100000000000000000098
:1037000000000000000000000000000000000000B9
:103710000000000000121110000000000000000076
:103720000000000000000000000000000000004B4E
:10373000494C4C45442E20004B494C4C206361754C
:10374000736564206279204B494C4C206275747417
:103750006F6E2F70696E0A004B494C4C45442E2009
:10376000004B494C4C20636175736564206279207D
:10377000746F6F206D75636820696E61637469761C
:10378000652074696D65202D2063757272656E7495
:1037900020636F6D6D616E643A200020746F6F203E
:1037A0006C6F6E6720657874727573696F6E2070C8
:1037B000726576656E7465640A0020636F6C6420C0
:1037C000657874727573696F6E2070726576656E58
:1037D0007465640A0000002100240027002A002DDF
:1037E000003000330001010000040107010A01015B
:1037F0000210202008081020401020408002010202
:1038000001080402010102040810204080804020C9
:103810001008040201800402018040201008040204
:103820000108040201010204081020408001020482
:10383000081020408005050505070508080808024E
:103840000202020A0A080804040404010101010139
:103850000101010303030303030303040707070C28
:103860000C0C0C0C0C0C0C020202020606060606DE
:103870000606060B0B0B0B0B0B0B0B1FFFFFFFFFC3
:10388000FFFF600000000001FF400000000000FF9B
:103890008000000000007F83CF00000C303F87FFD6
:1038A00080000C301F867980000C000F8C30C7839D
:1038B0008C30E78C30CFC7CC31F38C30DCECEC3380
:1038C000B98C30D86C6C33198C30D06C0C33198CAB
:1038D00030D86C0C33198C30DC6C0E3B198C30CF2B
:1038E0007C079F198C30C77C038F194000000000B3
:1038F0000002600000000000061FFFFFFFFFFFF84E
:103900002020506C616E6E6572427566666572420B
:10391000797465733A20002046726565204D656DA7
:103920006F72793A2000436F6D70696C65643A205C
:1039300044656320313520323031370A00207C2045
:10394000417574686F723A2028416C657068204F29
:10395000626A6563747320496E632E2C204C756C0B
:103960007A426F7420476974205265706F7369746E
:103970006F7279290A004465632031352032303175
:103980003731353A31393A313700204C6173742080
:10399000557064617465643A2000312E312E350A09
:1039A000004D61726C696E0020536F6674776172AE
:1039B000652052657365740A0020576174636864FA
:1039C0006F672052657365740A002042726F776ECC
:1039D000206F75742052657365740A0020457874F1
:1039E00065726E616C2052657365740A00506F7762
:1039F000657255700A0073746172740A00657272A0
:103A00006F722077726974696E6720746F206669BF
:103A10006C650A004572726F723A00456E64737489
:103A20006F707320256320256320256320256300A4
:103A3000205A3A0020593A0020583A00656E6473C3
:103A4000746F7073206869743A20006563686F3A18
:103A500000446F6E6520736176696E672066696CDD
:103A6000652E0A004D32390020204E6F7A7A6C653F
:103A70003A20006368616E6765006F662074686550
:103A80002066696C616D656E7400576169742066AB
:103A90006F72207374617274005052494E542050FA
:103AA00041555345440020204E6F7A7A6C653A2088
:103AB0000020004261636B004D696E696D756D2079
:103AC00054656D70206973203132302E0048656175
:103AD00074696E67206661696C65640025753A25B6
:103AE00030327500253032753A2530327500257533
:103AF0006420253032753A25303275000006090001
:103B0000FE000000000001090008FE000005080892
:103B100006000040F0C8888898781005080806005C
:103B200000C0F88888888888F80505050600012007
:103B300030F830200508080600002070F82020200A
:103B400020E00509090600FF2070A8A8B888887041
:103B5000200509090600FFE080C0B0A82830282809
:103B60000509090600FFF8A88888888888A8F8054C
:103B70000A0A0600FE205050505088A8A8887003FA
:103B8000030306000340A04000060900FE0701925F
:103B9000032120FFFF08FF07FF00000006000001CF
:103BA00007070602008080808080008003020206F2
:103BB0000105A0A00507070600005050F850F85076
:103BC000500507070600002078A07028F0200507A0
:103BD00007060000C0C81020409818050707060017
:103BE000006090A040A89068020303060104C04052
:103BF00080030707060100204080808040200307E3
:103C000007060100804020202040800505050600B1
:103C10000120A870A8200505050600012020F82035
:103C2000200203030602FFC04080050101060003D5
:103C3000F8020202060200C0C005050506000108E0
:103C40001020408005070706000070888888888853
:103C50007003070706010040C040404040E00507F0
:103C600007060000708808708080F80507070600C6
:103C700000F81020100808F00507070600001030B3
:103C80005090F81010050707060000F880F00808AB
:103C90008870050707060000708080F0888870052E
:103CA0000707060000F80810202020200507070657
:103CB000000070888870888870050707060000700B
:103CC000888878080870020505060200C0C000C098
:103CD000C00206060602FFC0C000C04080040707FD
:103CE000060000102040804020100503030600025B
:103CF000F800F804070706010080402010204080EB
:103D00000507070600007088081020002005070737
:103D100006000070880868A8A8700507070600005C
:103D2000708888F8888888050707060000F088886A
:103D3000F08888F00507070600007088808080887A
:103D400070050707060000F08888888888F0050756
:103D500007060000F88080F08080F805070706005D
:103D600000F88080F08080800507070600007088DA
:103D700080B8888870050707060000888888F8885A
:103D80008888010707060200808080808080800587
:103D9000070706000038101010109060050707068E
:103DA00000008890A0C0A09088050707060000804A
:103DB0008080808080F805070706000088D8A888E2
:103DC0008888880507070600008888C8A89888881A
:103DD000050707060000708888888888700507072F
:103DE000060000F08888F080808005070706000044
:103DF00070888888A89068050707060000F0888802
:103E0000F0A09088050707060000788080700808F9
:103E1000F0050707060000F82020202020200507D5
:103E200007060000888888888888700507070600CC
:103E30000088888888885020050707060000888841
:103E4000888888A8500507070600008888502050F9
:103E500088880507070600008888885020202005EC
:103E60000707060000F80810204080F8030707063F
:103E70000100E08080808080E0050505060001806B
:103E800040201008030707060100E0202020202022
:103E9000E005030306000420508805010106000028
:103EA000F8020202060205804005050506000070C2
:103EB000087888780507070600008080B0C88888E1
:103EC000F00505050600007080808870050707066C
:103ED00000000808689888887805050506000070C5
:103EE00088F880700507070600003048E040404031
:103EF000400506060600FF708888780870050707E9
:103F00000600008080B0C888888801070706020084
:103F1000800080808080800308080601FF20002048
:103F2000202020A040040707060000808090A0C049
:103F3000A090030707060100C04040404040E00554
:103F40000505060000D0A8A8A8A8050505060000DC
:103F5000B0C88888880505050600007088888870C4
:103F60000506060600FFF08888F080800506060634
:103F700000FF788888780808050505060000B0C8A5
:103F800080808005050506000070807008F0040739
:103F9000070600004040E0404040300505050600AF
:103FA000008888889868050505060000888888507C
:103FB000200505050600008888A8A8500505050607
:103FC000000088502050880506060600FF88888873
:103FD000780870050505060000F8102040F8030772
:103FE00007060100204040804040200107070602EC
:103FF0000080808080808080030707060100804069
:104000004020404080050202060002689000000047
:10401000060000000000060000000000060000008E
:10402000000006000000000006000000000006007E
:104030000000000006000000000006000000000074
:10404000060000000000060000000000060000005E
:10405000000006000000000006000000000006004E
:104060000000000006000000000006000000000044
:10407000060000000000060000000000060000002E
:10408000000006000000000006000000000006001E
:104090000000000006000000000006000000000014
:1040A00006000000000006000000000006000000FE
:1040B00000000600000000000600000000000600EE
:1040C00000000000060000000000060000000000E4
:1040D000060000000000060000010707060200803D
:1040E0000080808080800507070600002070A8A05F
:1040F000A87020050707060000304040E04050A8A7
:104100000505050600008870507088050707060041
:1041100000885020F820F820010707060200808060
:10412000800080808005080806000030482050503C
:10413000209060030101060107A0050707060000A3
:10414000F888B8B8B888F80507070600017008783D
:10415000887800F80505050600012850A0502805BC
:104160000303060001F80808020202060206408066
:10417000050707060000F888A88898A8F805010137
:10418000060006F80404040600036090906005072A
:10419000070600002020F8202000F804050506008E
:1041A0000360902040F0030505060003E020E020B6
:1041B000E002020206020640800508080600FF88A9
:1041C00088888898E8808005070706000078989816
:1041D00078181818020202060202C0C00202020683
:1041E00002FF408003050506000340C04040E00593
:1041F0000707060001708888887000F80505050625
:104200000001A0502850A00507070600008890A8CC
:1042100058B808080507070600008890B848982095
:1042200038050808060000C040C048D8380808050E
:104230000707060000200020408088700508080657
:1042400000004020007088F88888050808060000F3
:104250001020007088F888880508080600002050A3
:10426000007088F8888805080806000068900070CB
:1042700088F888880508080600005000708888F8CB
:1042800088880508080600002050207088F8888873
:104290000507070600003860A0B8E0A0B8050808C8
:1042A0000600FF708880808870206005080806007E
:1042B00000402000F880F080F8050808060000089B
:1042C0001000F880F080F805080806000020500073
:1042D000F880F080F80507070600005000F880F02D
:1042E00080F8030808060100804000E0404040E0FC
:1042F000030808060100204000E0404040E00308B9
:104300000806010040A000E0404040E00307070627
:104310000100A000E0404040E005070706000070F3
:104320004848E8484870050808060000689000887A
:10433000C8A898880508080600004020708888886A
:10434000887005080806000010207088888888702A
:10435000050808060000205000708888887005084D
:1043600008060000689000708888887005080806B4
:1043700000005000708888888870050505060001D7
:1043800088502050880508080600FF1070A8A8A8CB
:10439000A8704005080806000040208888888888A2
:1043A0007005080806000010208888888888700535
:1043B00008080600002050008888888870050808D2
:1043C0000600005000888888888870050808060064
:1043D0000010208850202020200509090600FFC079
:1043E00040704848704040E00408080601FF6090B3
:1043F00090A09090E0800508080600004020007022
:1044000008788878050808060000102000700878F1
:104410008878050808060000205000700878887821
:10442000050808060000689000700878887805077D
:104430000706000050007008788878050808060014
:10444000002050207008788878050606060000D005
:104450002878A0A8500506060600FF708088702006
:10446000600508080600004020007088F88070058C
:1044700008080600001020007088F8807005080801
:104480000600002050007088F880700507070600BD
:104490000050007088F88070030808060100804012
:1044A0000040C04040E003080806010020400040F2
:1044B000C04040E003080806010040A00040C040A2
:1044C00040E0030707060100A00040C04040E005AF
:1044D0000707060000A040A01078887005080806AD
:1044E0000000689000B0C8888888050808060000A9
:1044F0004020007088888870050808060000102099
:104500000070888888700508080600002050007038
:104510008888887005080806000068900070888800
:1045200088700507070600005000708888887005AD
:1045300005050600012000F800200507070600FF1A
:104540001070A8A8A87040050808060000402000C8
:104550008888889868050808060000102000888868
:104560008898680508080600002050008888889808
:1045700068050707060000500088888898680509C4
:10458000090600FF102000888888F80870040707D3
:104590000601FFC04060506040E00508080600FFCB
:1045A00050008888887808705A00590058000920FF
:1045B000000000000000000000000000007FFFE09D
:1045C0000000000000000000000000007000E0009B
:1045D000000000000000000000000061F860000022
:1045E0000000000000000000000041F82000000072
:1045F00000000000000000000040F020000000006B
:1046000000000000000000004060200000000000EA
:10461000000000000000005801A07F80003FC000A3
:104620000000004104005C63A0FBC00079E00000D2
:1046300000002082005EF7A0F3C00076E0000000DA
:10464000002082005EF7A0EBC0007EE000000000CA
:104650004104005C63A07B80003DC000000000823C
:1046600008005801A07B80003BC00000000104103E
:1046700000406020FBC00077E00000000104100053
:1046800040F020FBC00070E0000000008208004104
:10469000F820FFC0007FE00000000041040061F846
:1046A000603F00001F80000000000000007000E07C
:1046B0001E00000F0000000001FFFF807FFFE00CE4
:1046C0000000060000000001FFFF80000000000065
:1046D000000000000000000000007FFFE00000007C
:1046E0000000000000000000007000E0000000007A
:1046F0000000000000000000630C600000000000EB
:1047000000000000000000470E2000000000000034
:104710000000000000004F0F20000000000000001B
:1047200000000000005F0FA000000000000000007B
:10473000000000005E07A07F80003FC00000000076
:10474000410400406020FBC00079E0000000002030
:10475000820040F020F3C00076E0000000002082DC
:104760000040F020EBC0007EE000000000410400AB
:104770004060207B80003DC0000000008208005E99
:1047800007A07B80003BC0000000010410005F0F09
:10479000A0FBC00077E0000000010410004F0F20D4
:1047A000FBC00070E000000000820800470E20FF00
:1047B000C0007FE000000000410400630C603F0087
:1047C000001F80000000000000007000E01E0000DC
:1047D0000F0000000001FFFF807FFFE00C000006DB
:1047E0000000000001FFFF80000000656E7175652C
:1047F0007565696E672022004572726F722077724C
:104800006974696E6720746F20454550524F4D2181
:104810000A00486F6D65202573257325732066692E
:10482000727374002066697273740A005A0059002A
:104830005800486F6D6520005072696E7420706179
:1048400075736564004D313235004D36303020428D
:1048500030205431004D363030204230205430006A
:104860004D3234004D3233202573006175746F254D
:10487000692E6700004D32340045787472756465A6
:104880007232004578747275646572004D6F76659A
:10489000205A004D6F76652059004D6F766520587F
:1048A000004D6F76656D656E74004D6F76652061A5
:1048B0007869730044697361626C65207374657014
:1048C00070657273004D3834004175746F20686FE5
:1048D0006D6500473238004D61696E0043616E6E50
:1048E0006F7420656E746572207375626469723AC4
:1048F0002000022E2E004D61696E00205A3A0020E1
:10490000593A0020436F756E7420583A0020453A9A
:1049100000205A3A0020593A00583A00486F74650E
:104920006E64206F6666736574733A00202F0056BC
:10493000652D6A65726B0056652D6A65726B00564F
:10494000652D6A65726B00567A2D6A65726B00562A
:104950007A2D6A65726B0056792D6A65726B005606
:10496000792D6A65726B0056792D6A65726B0056F7
:10497000782D6A65726B0056782D6A65726B0056E9
:10498000782D6A65726B004D6F74696F6E004D36DD
:10499000303020486F74656E6420746F6F20636FD1
:1049A0006C6420746F206368616E67652066696C53
:1049B000616D656E740A00436F6F6C646F776E0093
:1049C00046616E20737065656420310046616E201B
:1049D000737065656420310042656400426564005F
:1049E0004E6F7A7A6C652032004E6F7A7A6C652051
:1049F00032004E6F7A7A6C652031004E6F7A7A6C95
:104A0000652031004D61696E00466C6F7720320081
:104A1000466C6F77203200466C6F77203100466C11
:104A20006F7720310046616E2073706565642031B8
:104A30000046616E207370656564203100426564D4
:104A400000426564004E6F7A7A6C652032004E6FCA
:104A50007A7A6C652032004E6F7A7A6C652031006C
:104A60004E6F7A7A6C65203100537065656400532F
:104A700070656564004D61696E00416D6178204527
:104A80003200416D617820453200416D61782045EA
:104A90003100416D617820453100416D6178205AC7
:104AA00000416D6178205A00416D617820590041C4
:104AB0006D6178205900416D6178205800416D6129
:104AC00078205800412D74726176656C00412D7418
:104AD000726176656C00412D726574726163740059
:104AE000412D7265747261637400416363656C008B
:104AF000416363656C004D6F74696F6E004D6F7636
:104B00006520302E316D6D004D6F766520316D6DF5
:104B1000004D6F76652031306D6D004D6F766520EC
:104B200061786973004578747275646572004D6FC1
:104B30007665205A004D6F76652059004D6F766579
:104B4000205800746F20726573756D650057616938
:104B50007420666F72207072696E74005052494EF4
:104B6000542050415553454400457874727564652E
:104B7000206D6F726500526573756D652070726986
:104B80006E7400524553554D45204F5054494F4E79
:104B9000533A0020204E6F7A7A6C653A200020004C
:104BA000506C6561736520776169742E2E2E004804
:104BB000656174696E67206E6F7A7A6C6500505219
:104BC000494E54205041555345440020204E6F7AA1
:104BD0007A6C653A2000200068656174206E6F7AF7
:104BE0007A6C652E00507265737320627574746FF1
:104BF0006E20746F005052494E5420504155534519
:104C0000440020204E6F7A7A6C653A2000200066BE
:104C1000696C616D656E7420657874727564650089
:104C20005761697420666F72005052494E5420508B
:104C300041555345440020204E6F7A7A6C653A20E6
:104C400000200066696C616D656E74206C6F616434
:104C5000005761697420666F72005052494E5420AB
:104C60005041555345440020204E6F7A7A6C653A86
:104C70002000746F20636F6E74696E75652E2E2E22
:104C800000616E6420707265737320627574746F56
:104C90006E00496E736572742066696C616D656E35
:104CA00074005052494E5420504155534544002001
:104CB000204E6F7A7A6C653A2000200066696C613C
:104CC0006D656E7420756E6C6F61640057616974F8
:104CD00020666F72005052494E5420504155534542
:104CE00044005761726E696E673A20486F6D696E55
:104CF000672042756D702044697669736F72203C3D
:104D000020310A000202040000A0400000A0400080
:104D100000004047322F4733206261642070617287
:104D2000616D65746572730A004F6666004F6E2090
:104D300000456E6473746F702061626F727400530B
:104D4000746570732F6D6D004A65726B004163630B
:104D5000656C65726174696F6E0056656C6F63692E
:104D6000747900416476616E636564205365747480
:104D7000696E6773005654726176206D696E0056D5
:104D800054726176206D696E005654726176206DA2
:104D9000696E00566D696E00566D696E00566D69DC
:104DA0006E00566D617820453200566D6178204561
:104DB0003200566D617820453200566D617820458D
:104DC0003100566D617820453100566D617820457F
:104DD0003100566D6178205A00566D6178205A0076
:104DE000566D6178205A00566D6178205900566DD5
:104DF0006178205900566D6178205900566D6178B0
:104E0000205800566D6178205800566D6178205802
:104E1000004D6F74696F6E000000904300008A437C
:104E200000007A4300004842000048420000404031
:104E300000000000FFFFFF5A2070726F6265206F54
:104E400075742E206265640A005A2070726F626564
:104E5000206F75742E2062656400486F6D65205860
:104E6000592066697273740A00486F6D652058593D
:104E7000206669727374004B642000236465666960
:104E80006E65202044454641554C545F004B6920D7
:104E90000023646566696E65202044454641554C93
:104EA000545F004B70200023646566696E652020A6
:104EB00044454641554C545F005049442041757467
:104EC0006F74756E652066696E697368656421200C
:104ED00050757420746865206C617374204B702C5D
:104EE000204B6920616E64204B6420636F6E737485
:104EF000616E74732066726F6D2062656C6F7720CF
:104F0000696E746F20436F6E66696775726174694C
:104F10006F6E2E680A00504944204175746F747595
:104F20006E65206661696C6564212074696D656FCA
:104F300075740A00504944204175746F74756E652C
:104F4000206661696C6564212054656D70657261CD
:104F50007475726520746F6F20686967680A002035
:104F60004B643A2000204B693A2000204B703A20D5
:104F7000000A20436C617373696320504944200A1E
:104F8000002054753A2000204B753A2000206D61B6
:104F9000783A2000206D696E3A200020643A2000A3
:104FA00020626961733A2000436172642072656D0A
:104FB0006F766564004361726420696E7365727414
:104FC00065640048617264636F646564204465666B
:104FD00061756C742053657474696E6773204C6FCF
:104FE000616465640A00282300002823000064002F
:104FF00000001027000000009643000096430000C8
:1050000040400000C8410000C9420000C942000001
:10501000C84400804F4400804F444E6F204C696E5E
:1050200065204E756D6265722077697468206368CB
:1050300065636B73756D2C204C617374204C696EC5
:10504000653A200053544F505045442E2000507272
:10505000696E7465722073746F7070656420647516
:105060006520746F206572726F72732E20466978A6
:1050700020746865206572726F7220616E6420759D
:105080007365204D39393920746F207265737461EE
:1050900072742E202854656D706572617475726526
:1050A0002069732072657365742E205365742069BE
:1050B00074206166746572207265737461727469BC
:1050C0006E67290A004E6F20436865636B73756DC8
:1050D0002077697468206C696E65206E756D6265F5
:1050E000722C204C617374204C696E653A20006309
:1050F0006865636B73756D206D69736D617463684A
:105100002C204C617374204C696E653A20004C6908
:105110006E65204E756D626572206973206E6F74C6
:10512000204C617374204C696E65204E756D62650C
:10513000722B312C204C617374204C696E653A20BF
:10514000004D313130004D3331004D38342058207E
:1051500059205A20450053442072656164206572CD
:10516000726F720A00446F6E65207072696E7469A6
:105170006E672066696C650A0045327374657073EA
:105180002F6D6D00453273746570732F6D6D004522
:105190003173746570732F6D6D0045317374657074
:1051A000732F6D6D005A73746570732F6D6D005A97
:1051B00073746570732F6D6D005973746570732F00
:1051C0006D6D005973746570732F6D6D0058737435
:1051D0006570732F6D6D005873746570732F6D6DEE
:1051E000004D6F74696F6E004E414E494E495459DF
:1051F000494E46CDCCCC3D0AD7233C17B7D13877A2
:10520000CC2B329595E6241FB14F0A0000204100B7
:1052100000C84200401C4620BCBE4CCA1B0E5AAE01
:10522000C59D740079FCDA5B11241FBECFEFD1E27B
:10523000DEBFCDBF00E00CBF14E0A0E0B2E0E6EAC4
:10524000F1E102E00BBF02C007900D92A831B10757
:10525000D9F725E1A8E1B4E001C01D92A834B20756
:10526000E1F712E5C6E2D2E500E006C022970109A7
:10527000FE010BBF0F945308C432D10780E008072A
:10528000A9F70E949AA60D94C2080C9400002F92D0
:105290003F924F925F926F927F928F929F92AF92C6
:1052A000BF92CF92DF92EF92FF920F931F93CF9313
:1052B000DF93CDB7DEB7CF55D1090FB6F894DEBF77
:1052C0000FBECDBF00918A1020E6029F80011124FD
:1052D000065F104F80910B0780FF1AC0EBE4FAE3E2
:1052E00084917F013FEFE31AF30A811102C0780134
:1052F00004C00E94804BF701F3CFD7018D917D014F
:10530000882319F00E94804BF8CF8AE00E94804BDE
:1053100010927806109277068FE380930A07109216
:105320000907109208071092320410923304109269
:10533000340410923504F80180810F5F1F4F8032D2
:10534000D1F38E34B1F4818190ED980F9A3020F032
:105350008D3211F08B3269F43296DF0131962C9147
:1053600020532A30D0F3CD01FC0101962081203258
:10537000D9F3F0930207E09301077F01BFEFEB1A27
:10538000FB0A10816AE270E0C7010F94930800974E
:1053900039F0DC0111978C918032E1F311961C9267
:1053A0001D3429F0143519F0173409F0CDC0F70178
:1053B0004E2F9F2F81918032D9F380538A3008F08D
:1053C000C3C010930A072091080730910907E42F02
:1053D000F92F6AE0AF014F5F5F4F629FC001639F8B
:1053E000900D1124208130E020533109820F931F4A
:1053F000218120532A3030F09093090780930807C9
:105400009A0103C09C01FA01E5CFD9012F5F3F4FFC
:105410004C914032D1F31D3449F0B09001074091D6
:1054200077065091780661E070E050C08E319105AA
:1054300091F03CF48731910571F08C31910569F759
:105440000AC0853791054CF38737910524F0803ADF
:10545000E3E09E0711F7B0937806A093770674C037
:105460002132F1F10FEB020F0A3108F05AC09F010F
:10547000F901A0812F5F3F4FA032D1F320ED2A0F19
:105480002A3008F042C09F01E02EF12CD701B595DB
:10549000A795B595A795B595A795AE5CBB4F077039
:1054A0006B01002E01C0CC0C0A94EAF7DC90DC28DA
:1054B000DC922115310599F12B19D701A85EBB4F5C
:1054C0002C93208121542A3188F5DF01FD0131968A
:1054D0002C912111C5CF509378064093770634C0A4
:1054E0001D3409F0BFCF8032910509F0BBCFF09396
:1054F0007806E093770663E270E0CF010F9493089B
:10550000009711F1DC011C921FC023ED2A0F2230FD
:1055100008F4B9CFAB3211F00C94493FB4CF20E07E
:10552000CCCF4115510569F6AD01CBCF9F01319626
:10553000D9010C9100530A30C8F3F9012F5F3F4F96
:10554000A081A032D1F3C1CF80910A078D3409F434
:1055500033C2843511F40C94233E873411F00C943B
:105560002C3F20910807309109072A31310509F4B1
:1055700059C18CF42430310544F4223031050CF04B
:1055800003C137FF25C00C94463F2430310509F490
:1055900004C10C94463F2A35310509F4CEC174F498
:1055A0002B31310509F445C12C31310511F00C9432
:1055B000463F80E00E940BEC0C94463F2B353105B2
:1055C00009F4BFC12C35310509F4C0C10C94463F24
:1055D00080916202882311F40C94463F0E94AF4EE2
:1055E00086E394E00E949D4C0E94FB5180910B0742
:1055F00083FD79C0C0904204D0904304E0904404FD
:10560000F09045042091E00E3091E10E4091E20EC1
:105610005091E30EC701B6010F942F01882309F4BE
:1056200062C0809100070E941A4F882301F1C09246
:10563000E00ED092E10EE092E20EF092E30EEBE487
:10564000FAE384918F010F5F1F4F882321F00E949E
:10565000804BF801F6CFE5EDF1E084918F010F5F0B
:105660001F4F882321F00E94804BF801F6CFC09095
:105670004204D0904304E0904404F090450420910B
:10568000E00E3091E10E4091E20E5091E30EC70121
:10569000B6010F94610520E030E048E453E40F9434
:1056A0008807181604F5C092E00ED092E10EE09241
:1056B000E20EF092E30EEBE4FAE384918F010F5FC8
:1056C0001F4F882321F00E94804BF801F6CFE6EBB4
:1056D000F1E084918F010F5F1F4F882321F00E941A
:1056E000804BF801F6CF2091360430913704409179
:1056F0003804509139046091D40E7091D50E809188
:10570000D60E9091D70E0F942F0181111DC02091BC
:105710003A0430913B0440913C0450913D04609127
:10572000D80E7091D90E8091DA0E9091DB0E0F9405
:105730002F01811109C060915E0270915F0280911A
:105740006002909161021AC060918E0270918F0286
:10575000882777FD8095982F0F94350120915E0260
:1057600030915F0240916002509161020F94940168
:105770002AE037ED43E25CE30F9494010E9403F6C4
:105780000E94FC4C0C94463F81E02230310509F028
:1057900080E00E945DE00C94463F80E50E94CF4D82
:1057A000882329F00E949E4B4B015C0103C0812C91
:1057B000912C540183E50E94CF4D882361F00E9413
:1057C000DE4B20E030E04AE754E40F9494010F945C
:1057D000AB064B015C010E9447F080910A028111E7
:1057E00005C060E080EF91E00E9493B90E94FB51F8
:1057F000C0904604D0904704E0904804F0904904DB
:10580000C80CD91CEA1CFB1C0E94C9506C197D09EC
:105810008E099F0997FD02C00C94463F80E00E94CC
:105820009C97F2CF81E0809362021092DB060C9489
:10583000463F0E9452B381110C94463F80E50E947E
:10584000CF4D882321F00E94AE4B462F01C040E08F
:105850006091DC0E7091DD0E8091DE0E9091DF0E76
:1058600000E010E020E031E409831A832B833C83BD
:1058700000E010E025E833E40D831E832F83388792
:1058800000E010E020EA31E409871A872B873C8783
:1058900000E010E020EC3FE70D871E872F87388B54
:1058A000413071F1423021F518A219A21AA21BA2AF
:1058B00020E030E040EA51E40F9462057B018C0166
:1058C00020E030E04AE753E40F948807181624F4E8
:1058D000E12CF12C0AE713E4A701B8014BAF5CAF50
:1058E0006DAF7EAFBE01605E7F4FCE01CB9611C023
:1058F00020E030E040EA51E40F942F0187FF0BC015
:1059000018A219A21AA21BA2BE01605E7F4FCE018F
:1059100009960E9433E718A219A21AA21BA29E019F
:10592000205E3F4F4CED5EE0BE016B5F7F4FCE01CE
:1059300001960E9441E60C94463F109207070C9492
:10594000463F81E0809307070C94463F85E40E9420
:10595000CF4DC82E811102C00E9447F0EFE0EE2E1D
:10596000E3E0FE2E04ED1EE0B12CD12CF701819175
:105970007F010E94CF4D882369F00E94DE4BD80141
:105980006D937D938D939C931397B3E0DB1611F089
:10599000BB24B394D3940C5F1F4FE4E0DE12E6CF38
:1059A000BB2019F00E94F6F203C0C1100E9456B449
:1059B0000E942BCA0C94463F8091080790910907DA
:1059C0008737910511F40C9442360CF0CCC08C341E
:1059D000910509F47DC50CF06CC08831910509F47E
:1059E000AAC2BCF58231910509F486C7C4F497FFB9
:1059F00002C00C94463F823091050CF4C1C141971E
:105A000011F00C94463F60E080E392E00E9493B96D
:105A1000179816981598149813980C94463F85314A
:105A2000910509F471C23CF4449711F00C94463F7F
:105A3000E8E4F2E028C28631910509F469C247978B
:105A400011F00C94463F8091770690917806FC0106
:105A500069C28E31910509F4E5C2C4F48A31910519
:105A600009F496C20CF486C28B31910509F49EC2EA
:105A70004C9711F00C94463F40E060E0809177062F
:105A8000909178060E94877F0C94463F8032910562
:105A900009F4EBC30CF434C48A32910509F4D1C47F
:105AA0008B34910511F00C94463F0E941DB40C9468
:105AB000463F8936910509F4A7C524F5833591053C
:105AC00009F415C77CF48135910509F4F1C60CF091
:105AD0000AC78D34910511F00C94463F0E948797B8
:105AE0000C94463F8535910509F43DC70CF404C775
:105AF0008C35910509F452C78836910509F4ECC438
:105B00000C94463F8F36910509F45CC584F48B36BE
:105B1000910509F416C60CF4EFC58D36910509F40C
:105B2000B6C58E36910509F43AC50C94463F8337C5
:105B3000910509F4D1C75CF48237910511F00C94FA
:105B4000463F0E9447F00E942BCA0C94463F85377F
:105B5000910511F40C94FE358637910511F40C94DF
:105B600007360C94463F8C32F1E09F0711F40C94F9
:105B700083390CF077C0893C910511F40C941A37E5
:105B800064F58C38910509F421C574F489379105C1
:105B900011F40C94AD3614F40C94A6368D3791059F
:105BA00009F4E7C50C94463F8B39910509F446C5C5
:105BB0004CF48139910511F00C94463F0E94444EFB
:105BC0000C94463F8E3B910509F47FC5883C9105B6
:105BD00011F40C94B3360C94463F833D910511F4B7
:105BE0000C94813824F58C3C910511F40C94753794
:105BF0003CF48B3C910511F40C944C370C94463FCB
:105C00008D3C910511F40C94DF378E3C910511F019
:105C10000C94463F0FE0802E03E0902E84EDA82EDA
:105C20008EE0B82E08EC1EE0712C0C944A388C3DA6
:105C3000910511F40C9419394CF48A3D910511F039
:105C40000C94463F0E94BCC90C94463F8D3D910583
:105C500011F40C942639823E910511F40C943F39CD
:105C60000C94463F843F31E0930711F40C94933A2F
:105C70000CF04DC08E3551E0950711F40C94A33D06
:105C8000C4F48E32B1E09B0711F40C94AF3914F4D4
:105C90000C94AC398F32F1E09F0711F40C94B239B7
:105CA0008033914011F00C94463F0E9463710C9434
:105CB000463F833631E0930711F40C94F83D3CF4F1
:105CC0008F35914011F40C94A63D0C94463F8039D9
:105CD000A1E09A0711F40C94B5398C3A914011F077
:105CE0000C94463FE8EC8E2EEEE09E2EF4EDAF2EA7
:105CF000FEE0BF2EABEC2A2EA6E03A2E00E010E02C
:105D0000422D409560964FAF60970C94B839883516
:105D1000E2E09E0711F40C94B53AB4F4863F21E01A
:105D2000920711F40C94993A14F40C94963A873F24
:105D300041E0940711F40C949C3A8C31924011F498
:105D40000C94AA3A0C94463F8C38A3E09A0711F4BD
:105D50000C94A03D4CF48B38934011F00C94463FCA
:105D60000E9456C90C94463F803AF3E09F0709F41D
:105D7000BAC2873E934011F40C94113E0C94463FF6
:105D8000009177061091780680E50E94CF4D882318
:105D900069F00E949E4B6B017C01BB24B39461159A
:105DA00071058105910531F4B12C04C0B12CC12CD1
:105DB000D12C760183E50E94CF4D8823F9F00E9413
:105DC000DE4B20E030E04AE754E40F9494010F9456
:105DD000AB066B017C01B11013C061157105810523
:105DE000910571F40115110559F0D8018C918823A2
:105DF00039F061E0C8010E942EB907C0BB2091F3C1
:105E000060E08DE192E00E9493B981E080935807B1
:105E10000E9447F00E94FB51C114D104E104F10437
:105E2000D1F08090460490904704A0904804B09030
:105E300049048C0C9D1CAE1CBF1C0E94C9506819E3
:105E400079098A099B0997FF1AC080915807811127
:105E50000C94533F14C080915807882321F080E0B0
:105E60000E949C97F8CF8091911260E0882319F0EE
:105E70008EE092E002C089EF91E00E9493B9109207
:105E800058070C94463F84918F010F5F1F4F882362
:105E900021F00E94804BF801F6CF10923D1540E0B2
:105EA00050E0BA0189EE92E10E9451958BE1E9EE52
:105EB000F2E1DE01159601900D928A95E1F780914D
:105EC000E7129091E8129C838B8387E093E09A839A
:105ED000898340E050E0BE016F5F7F4F8CE293E02A
:105EE0000E94718CCE0101960E946A8CE9E3F2E077
:105EF00084918F010F5F1F4F882311F40C94463F4C
:105F00000E94804BF801F4CF0E942B8A0C94463FEC
:105F100010929112109292120C94463F203209F482
:105F20001082319620812111F9CF40E061E00E947A
:105F3000877F0C94463F19821A821B821C8218A20A
:105F400019A21AA21BA28091DA06882341F040E030
:105F5000BE016F5F7F4FCE0180960E94CCCC8091B6
:105F60009212882319F081E0809391120E941DB44F
:105F70000C94463F109291120E949BB489E592E0E6
:105F80009093DD078093DC070E94BA7E0C94463F15
:105F900080919212882311F40C94463F83E50E946D
:105FA000CF4D81110C94583F0C94463F8091921232
:105FB000882351F1EEE5F2E084918F010F5F1F4FCE
:105FC000882321F00E94804BF801F6CF60913415B0
:105FD0007091351580913615909137154AE00E94E1
:105FE000916F8FE20E94804B609130157091311556
:105FF00080913215909133154AE00E94916F8AE0AA
:106000000E94804B0C94463FE0E7F2E084918F01C0
:106010000F5F1F4F882311F40C94463F0E94804B62
:10602000F801F4CF80919212882311F40C94463F2A
:1060300083E894E10E942DC483E894E10E94188AC9
:106040001092901210928F12E0907706F0907806DE
:1060500080919212882311F40C94463F0E94218A69
:106060001D8218861C821B8287E093E09A838983B5
:1060700085EE92E19093051380930413F7018081DC
:106080008F3209F06BC06FE270E0C7010F94930884
:106090008C010F5F1F4F9E012F5F3F4F590101156C
:1060A000110509F461C06FE270E0C8010F94930814
:1060B0006C01009709F459C00817190708F055C07A
:1060C0004C01801A910AA401B801CE0180960F9468
:1060D000B308E0E2F0E0EC0FFD1FE80DF91D1082BF
:1060E0008E01005E1F4FD8018D918D01882319F01C
:1060F0000E94804BF8CF8AE00E94804B609104138D
:10610000709105136115710519F06C5F7F4F02C026
:1061100060E070E021E0AE01405E5F4FCE01059689
:106120000E94758B811112C0BE01605E7F4F87EAAD
:1061300092E00E9483B58EE20E94804B8AE00E942A
:10614000804BC5010E946A8C0C94463FB0920513A7
:10615000A092041386010F5F1F4FA1CF86E093E149
:106160009093051380930413870160910413709139
:1061700005136115710519F06C5F7F4F02C060E077
:1061800070E018A21BA222E0A801CE0180960E9416
:10619000758BF82E882311F1CE0180960E945186CE
:1061A000F82E8823D9F06CA57DA58EA59FA541E08A
:1061B0000E94C891F82E882389F0E8A9B0E2EB9FED
:1061C000F0011124E65BFB4F309739F085EE8083B8
:1061D0001BA20E948A91F82E01C0F12CCE0180965C
:1061E0000E94708BFF2011F171E8E72E72E0F72E0C
:1061F000F7018491882331F0FFEFEF1AFF0A0E9424
:10620000804BF6CFD8018D918D01882319F00E9423
:10621000804BF8CF8AE00E94804B10923415109288
:106220003515109236151092371519C06FE8E62E05
:1062300062E0F62EF7018491882331F0FFEFEF1A28
:10624000FF0A0E94804BF6CFD8018D918D018823E3
:1062500019F00E94804BF8CF8EE20E94804BCE0155
:1062600001960E946A8C0C94463F80919112811194
:106270000E9447F0009177061091780680E50E9411
:10628000A14D882321F00E94CF4BF82E01C0F12CA4
:1062900080919212882311F40C94463F4F2D61E0B7
:1062A000C8010E94877F83E50E94CF4D882381F03B
:1062B0000E94AE4BAB01BC01409334155093351591
:1062C000609336157093371583E894E10E945195D9
:1062D00080919212882319F081E080939112F1103D
:1062E0000C94463F43CE809177069091780621E04A
:1062F0002093901240E060E00E94877F0C94463F1C
:106300000E94E9B35CE3C52ED12CE12CF12CA7014E
:1063100096010F940405162F072FCA01B901A70192
:1063200096010F940405D62EC72ECA01B90128E1A3
:1063300030E040E050E00F940405FB01C9016DE638
:1063400071E00F9426089B014D2D5C2DDE01119606
:106350007D012115310599F00F931F93CF92DF92A4
:10636000FF93EF939F938F933F932F9383EE92E04E
:106370009F938F93FF92AF930F94C90012C0009721
:10638000B1F00F931F93CF92DF92FF93EF939F9300
:106390008F9383ED92E09F938F93FF92AF930F942F
:1063A000C9000FB6F894DEBF0FBECDBF30C0309726
:1063B00079F00F931F93CF92DF92FF93EF9387ECC7
:1063C00092E09F938F93FF92AF930F94C900E9CF10
:1063D000452B69F00F931F93CF92DF928FEB92E0E2
:1063E0009F938F93FF92AF930F94C900DACF0F93CF
:1063F0001F938BEB92E09F938F93FF92AF930F9439
:10640000C9000F900F900F900F900F900F9060E0C9
:10641000C7010E942EB9EBE4FAE384918F010F5F6C
:106420001F4F882321F00E94804BF801F6CFB7015F
:1064300087EF92E00E9483B58AE00E94804B0C9423
:10644000463F83E50E94CF4D882311F40C94463FCC
:106450000E94BE4BE82E80E50E94CF4D882311F4A8
:106460000C94463F80E50E94CF4D882341F00E9466
:10647000AE4B77FF02C00C94463F8B0102C00DE08B
:1064800010E0802FE4E0F3E09491891739F0319621
:1064900093E0E433F907C1F70C94693FE4E1FAE3D0
:1064A00084918F010F5F1F4F882321F00E94804B42
:1064B000F801F6CFE4E3F3E084918F010F5F1F4F03
:1064C000882311F40C94463F0E94804BF801F4CFCE
:1064D0000E949BB40C94463F88E690E00E94056FB2
:1064E00081110C94463F80910B0783FF02C00C94EE
:1064F000463F83E50E94CF4D882311F40C94463F1C
:106500000E94DE4BF090B2060F2D10E0000F111F1D
:106510000F5E124F0F94A606D8016D937C938F2DBA
:106520000E941E510E94DE4B20E030E040E752E422
:106530000F942F0118163CF00E94879760E082E5C7
:1065400093E00E9493B90E94DE4B0091B20610E0E6
:10655000F801EE0FFF1FEE0FFF1FED5AF94F2081DC
:106560003181428153810F948807181614F00C94DE
:10657000463F8EED92E09F938F930F5F1F4F1F93C7
:106580000F9383E493E09F938F931F920E9438B3FD
:106590000FB6F894DEBF0FBECDBF0C94463F8EE41D
:1065A0000E94CF4D882311F40C94463F0E94AE4BBD
:1065B00060934A0670934B0680934C0690934D0669
:1065C0000C94463F0E94DB4D0C94463F80910B0794
:1065D00083FF02C00C94463F83E50E94CF4D882381
:1065E00011F40C94463F0E94DE4B0F94A6066739C7
:1065F000710514F066E970E070930E0D60930D0D57
:106600000E94D5500C94463F89E690E00E94056FA9
:1066100081110C94EE42E7E6F3E084918F010F5F65
:106620001F4F882321F00E94804BF801F6CF0E9473
:10663000AD638AE00E94804B0C94EE4283E50E9499
:10664000CF4D882311F40C94463F0E94BE4B80939B
:1066500052068D3318F08CE3809352060E94C95085
:106660006B017C012091520630E0A8EEB3E00F945C
:106670005205C60ED71EE81EF91EC0924E06D092D5
:106680004F06E0925006F09251060C94463F8DE67C
:1066900090E00E94056F81110C94463F80910B079A
:1066A00083FF02C00C94463F83E50E94CF4D609665
:1066B0008FAF609781110C94853F82E50E94CF4D8A
:1066C00081110C94853F0C94463F80910B0783FF0A
:1066D00002C00C94463F83E50E94CF4D68968FAF71
:1066E000689781110C94464182E50E94CF4D81113B
:1066F0000C9446410C94463F83E50E94CF4D88237D
:1067000039F00E94AE4B8B016F3F710519F010F00C
:106710000FEF10E080E50E94CF4D882339F00E94F2
:10672000BE4B823010F00C94463F01C080E0E82F51
:10673000F0E0EE0FFF1FE251FF4E118300830C9437
:10674000463F80E50E94CF4D882341F00E94AE4B2A
:106750006230710510F00C94463F02C060E070E0BA
:10676000FB01EE0FFF1FE251FF4E118210820C94CD
:10677000463F8CE40E94A14D882319F00E94DE4B15
:1067800004C060E070E080E090EC27966CAF7DAFD5
:106790008EAF9FAF27978AE50E94CF4D882319F0CF
:1067A0000E94DE4B03C060E070E0CB0120E030E0EF
:1067B00040E251E40F94620523966CAF7DAF8EAF3B
:1067C0009FAF239788E50E94CF4D882319F00E9440
:1067D000DE4B03C060E070E0CB0120E030E040E23F
:1067E00051E40F946205E0910007EE2359F0A4E014
:1067F000EA9FF0011124E851F94F20813181428153
:10680000538103C020E030E0A9010F9462056BAF13
:106810007CAF8DAF9EAF89E50E94CF4D882319F0E4
:106820000E94DE4B03C060E070E0CB0120E030E06E
:106830004AE853E40F94620520E030E040E251E47E
:106840000F946105E0910007EE2359F0B4E0EB9F4F
:10685000F0011124E051F94F2081318142815381AF
:1068600003C020E030E0A9010F94620568A379A37A
:106870008AA39BA319821A821B821C828091DA064A
:1068800081110C94463FC12CE12C8E010F5F1F4FEC
:106890009E01205E3F4FAE01455C5F4FBE01615CD3
:1068A0007F4FCE018D5B9F4F0E940ACE0C94463FD6
:1068B0000E94446F0E9447F00E94124C1092EF1009
:1068C0001092EE101092F1101092F01068EE73E03A
:1068D00080E090E00E942F8660E086ED93E00E94C9
:1068E00093B90C94463F109206070C94463F81E002
:1068F000809306070C94463F83E50E94CF4D882382
:10690000A1F00E94DE4B20E030E04AE754E40F940F
:1069100094010F94AB0660934D0270934E028093E6
:106920004F02909350020C94463F88E50E94A14D7F
:1069300081110C94CB4289E50E94A14D81110C94E8
:10694000CB428AE50E94A14D81110C94CB4285E493
:106950000E94A14D81110C94CB420E9447F00E94ED
:10696000124C0C94463F83E50E94A14D882311F4FC
:106970000C94463F0E94DE4B20E030E04AE754E4AE
:106980000F9494010F94AB0660935F0670936006BA
:1069900080936106909362060C94463F8CE590E0EC
:1069A0000E94056F81110C94463FEFE0F3E0619681
:1069B000FFAFEEAF619744EDA42E41E1B42E312C30
:1069C0006196AEADBFAD61978D916196BFAFAEAF31
:1069D00061970E94A14D882309F473C0B3E03B1274
:1069E00069C00E94DE4B6B017C0120E030E040EA90
:1069F00051E40F942F012090B20687FF50C0022D62
:106A000010E00D5F1F4F000F111F000F111FF80145
:106A1000EC52FE4EA70196016081718182819381C3
:106A20000F943E062B013C019B01AC016091A20634
:106A30007091A3068091A4069091A5060F949401ED
:106A40006093A2067093A3068093A4069093A50674
:106A5000F801EE57F94F4F01A30192016081718156
:106A6000828193810F949401D4016D937D938D93D2
:106A70009C9313970D59194FF801608171818281A0
:106A800093810F943301A30192010F9494010F9409
:106A9000AB06D8016D937D938D939C931397B4E0CF
:106AA0002B9EF0011124E052FE4EC082D182E28280
:106AB000F38207C00E94DE4BF501608371838283FD
:106AC00093833394F4E0AF0EB11C24E0321278CFFC
:106AD0000E942FF10C94463FE4ECF4E084918F0186
:106AE0000F5F1F4F882321F00E94804BF801F6CFE3
:106AF000E6EBF4E084918F010F5F1F4F882321F0B4
:106B00000E94804BF801F6CFEFE9F4E084918F0109
:106B10000F5F1F4F882321F00E94804BF801F6CFB2
:106B2000EFE8F4E084918F010F5F1F4F882321F07D
:106B30000E94804BF801F6CFEEE7F4E084918F01DC
:106B40000F5F1F4F882321F00E94804BF801F6CF82
:106B5000EDE6F4E084918F010F5F1F4F882321F051
:106B60000E94804BF801F6CFEEE5F4E084918F01AE
:106B70000F5F1F4F882321F00E94804BF801F6CF52
:106B8000E9E4F4E084918F010F5F1F4F882321F027
:106B90000E94804BF801F6CFE3E3F4E084918F018B
:106BA0000F5F1F4F882321F00E94804BF801F6CF22
:106BB000EEE1F4E084918F010F5F1F4F882321F0F5
:106BC0000E94804BF801F6CFE1E0F4E084918F0160
:106BD0000F5F1F4F882321F00E94804BF801F6CFF2
:106BE000E9EEF3E084918F010F5F1F4F882311F4CA
:106BF0000C94463F0E94804BF801F4CF60E08091F6
:106C00007706909178060E942EB90C94463F85E451
:106C10000E94A14D882381F00E94CF4B882361F010
:106C2000EBE4FAE384918F010F5F1F4F882321F07B
:106C30000E94804BF801F6CF81E40E94A14D882389
:106C400081F00E94CF4B882361F0ECEBF5E084915A
:106C50008F010F5F1F4F882321F00E94804BF801A6
:106C6000F6CF0091770610917806D8018D918D01AD
:106C7000882319F00E94804BF8CF8AE00E94804B55
:106C80000C94463FE8EDF5E084918F010F5F1F4FB4
:106C9000882321F00E94804BF801F6CFE0EDF5E06B
:106CA00084918F010F5F1F4F882321F00E94804B3A
:106CB000F801F6CF1E9903C009EF12E002C004EFFD
:106CC00012E0F80181918F01882319F00E94804B16
:106CD000F8CF8AE00E94804BE8ECF5E084918F01C8
:106CE0000F5F1F4F882321F00E94804BF801F6CFE1
:106CF0001D9903C009EF12E002C004EF12E0D801B1
:106D00008D918D01882319F00E94804BF8CF8AE085
:106D10000E94804BE0ECF5E084918F010F5F1F4FE4
:106D2000882321F00E94804BF801F6CF1C9903C004
:106D300009EF12E002C004EF12E0F80181918F0127
:106D4000882309F49ACF0E94804BF7CF81E080938B
:106D5000C70E8093C60E0C94463F1092C70E109239
:106D6000C60E0C94463F88EC90E00E94056F81119E
:106D70000C94463F84E40E94A14D882309F456C038
:106D80000E94DE4B11E020E030E0A9010F942F01BA
:106D9000811101C010E010938106112309F446C04F
:106DA0000091B20610E00E94DE4BF801EE0FFF1FCB
:106DB000EE0FFF1FE758F94F60837183828393833F
:106DC00020E030E0A9016091790670917A06809107
:106DD0007B0690917C060F942F0181110CC080E0FE
:106DE00090E0A0E4B0E48093790690937A06A093B3
:106DF0007B06B0937C0620E030E0A90160917D061F
:106E000070917E0680917F06909180060F942F01ED
:106E100081110CC080E090E0A0E4B0E480937D0696
:106E200090937E06A0937F06B09380060E941C4C30
:106E30000C94463F89EC90E00E94056F81110C9400
:106E4000463F9FE0E92E93E0F92ED12CD7018D919A
:106E50007D010E94A14D8823C1F0B3E0DB1203C085
:106E60000091B20601C000E00E94DE4B0D0DE4E08F
:106E70000E9F800111240D501F4E0F94AB06D801B8
:106E80006D937D938D939C931397D394B4E0DB1211
:106E9000DDCF0E94F14AFAC78BEC90E00E94056FAB
:106EA0008111F4C70FE013E0F12CF80181918F01FB
:106EB0000E94A14D8823A1F0F3E0FF1203C0E090EF
:106EC000B20601C0E12C0E94DE4BEF0C24E0E29EF2
:106ED000F0011124EE57F94F60837183828393830D
:106EE000F39434E0F312E1CFD1C783E50E94A14DC2
:106EF0008823D9F00E94DE4BAB01BC0140930F11F7
:106F00005093101160931111709312114093071157
:106F1000509308116093091170930A118CE496E064
:106F20000E94AD708AE00E94804B80E50E94A14DD6
:106F3000882399F00E94DE4BAB01BC0140930F11F6
:106F40005093101160931111709312118FE296E01B
:106F50000E94AD708AE00E94804B82E50E94A14DA4
:106F6000882399F00E94DE4BAB01BC0140930B11CA
:106F700050930C1160930D1170930E1180E196E007
:106F80000E94AD708AE00E94804B84E50E94A14D72
:106F9000882309F47BC70E94DE4BAB01BC01409300
:106FA0000711509308116093091170930A1182EF31
:106FB00095E00E94AD708AE00E94804B67C783E530
:106FC0000E94A14D882351F00E94DE4B6093AE06D3
:106FD0007093AF068093B0069093B10684E50E944B
:106FE000A14D882351F00E94DE4B6093AA06709356
:106FF000AB068093AC069093AD0682E40E94A14D4F
:10700000882351F00E949E4B6093A6067093A706BA
:107010008093A8069093A90688E50E94A14D882335
:1070200051F00E94DE4B6093960670939706809312
:1070300098069093990689E50E94A14D882351F006
:107040000E94DE4B60939A0670939B0680939C0689
:1070500090939D068AE50E94A14D882351F00E94DD
:10706000DE4B60939E0670939F068093A0069093DC
:10707000A10685E40E94A14D882309F407C70E9458
:10708000DE4B6093A2067093A3068093A4069093B0
:10709000A506FCC6D4018D914D010E94A14D882307
:1070A00011F10E94DE4B6B017C01F80120813181DE
:1070B000428153810F9461059B01AC01D5016D9113
:1070C0007D918D919C910F946205F5016083718390
:1070D00082839383D801CD92DD92ED92FC92139737
:1070E000872D0E94064D7394B4E0AB0EB11C0C5F6B
:1070F0001F4FE3E07E12CECF0E94F6F20E942BCA11
:10710000C5C6EBE4FAE384918F010F5F1F4F88231C
:1071100021F00E94804BF801F6CF83E50E94A14D3B
:10712000882321F00E94CF4B80935102ECE9F6E0D6
:1071300084918F010F5F1F4F882321F00E94804BA5
:10714000F801F6CF80915102882319F0E4E9F6E0C6
:1071500002C0E8E9F6E084918F010F5F1F4F88239A
:1071600021F00E94804BF801F6CFECE8F6E0849124
:107170008F010F5F1F4F882321F00E94804BF80181
:10718000F6CF4091BF065091C0066091C106709144
:10719000C2068AE896E00E94AD704091C306509105
:1071A000C4066091C5067091C60687E896E00E9405
:1071B000AD704091C7065091C8066091C9067091A4
:1071C000CA0684E896E00E94AD70ECE7F6E0849190
:1071D0008F010F5F1F4F882321F00E94804BF80121
:1071E000F6CF409152025091530260915402709137
:1071F00055028AE796E00E94AD7040915602509188
:107200005702609158027091590287E796E00E94F8
:10721000AD7040915A0250915B0260915C02709196
:107220005D0284E796E00E94AD708AE00E94804B88
:107230002DC683E50E94CF4D882309F427C60E94FE
:10724000AE4B70938F0260938E0220C68DED90E05E
:107250000E94056F81111AC683E50E94CF4D8823D5
:1072600009F414C60091B20610E00E94AE4BF8017A
:10727000EE0FFF1FE657FD4F7183608307C680E561
:107280000E94A14D882309F401C60E94AE4BF62E40
:10729000062F172F83E50E94CF4D882321F00E94EF
:1072A000AE4B6B0103C0CC24CA94DC2C96012F5F3B
:1072B0003F4F2330310508F0E9C517FDE7C50E94AF
:1072C00047F0FFEFCF16DF0631F0CA94CD2871F0FA
:1072D00000E010E00DC08F2D0E94665031E020E0EC
:1072E000892B09F030E0032F122F02C001E010E0DB
:1072F0008F2D0E9466508017910709F4C7C580E062
:107300000E949C97F5CF83E50E94CF4D882319F00A
:107310000E94AE4B02C064E071E079A368A380E5EF
:107320000E94CF4D882339F00E94AE4B693833E17B
:10733000730730F402C068EE73E07A83698304C097
:1073400088E893E19A838983BE01605E7F4FCE0116
:1073500001960E9442859AC50E94C97097C50E94F5
:10736000F87194C50E943AE791C50E9447F08EC516
:10737000D1018D911D01882309F4A3C0F50140803E
:10738000518062807380F801EE5AFD4F2081318177
:1073900042815381F801E154F94F6081718182810A
:1073A00093810F94620520E030E040E05FE30F94AA
:1073B00094019B01AC01C301B2010F948807181618
:1073C00044F4F801E455F94FC590D590E590F49058
:1073D00003C0C12CD12C7601F801ED54F94F208166
:1073E000318142815381C301B2010F9461059B0138
:1073F000AC01C701B6010F9461056B017C0120E06F
:1074000030E040EA51EC0F94880787FD2BC020E064
:1074100030E040EA51E4C701B6010F942F0118167D
:107420000CF1D4012D913D914D915C91C701B601B4
:107430000F9461059B01AC01C301B2010F94620579
:10744000F5016083718382839383D401CD92DD92B1
:10745000ED92FC92139760968FAD6097820D0E941B
:10746000064D2FC0E4E1FAE384918F010F5F1F4FB7
:10747000882321F00E94804BF801F6CFE6EDF6E07C
:1074800084918F010F5F1F4F882321F00E94804B52
:10749000F801F6CF61E088EC96E00E9493B90E9473
:1074A000B5BC88E290E09A83898388EC90E099A348
:1074B00088A3BE016F5F7F4FCE0180960E944285F8
:1074C000E5C4B4E08B0E911C0C5F1F4FE4E0AE0EE0
:1074D000B11C0C30110509F04BCF0E94F6F20E944E
:1074E0002BCA60E088EB96E00E9493B983E992E0B2
:1074F00099A388A304E610E01A830983BE01605EA5
:107500007F4FCE0101960E9442858AEB92E099A3BB
:1075100088A31A830983BE01605E7F4FCE01019666
:107520000E944285B3C40E947E65B0C40E94D47696
:10753000ADC40E9468F1AAC483E50E94A14D8823CE
:1075400019F00E94CF4B01C081E091E089270E9491
:10755000046A9CC483E50E94A14D882309F496C463
:107560000E94CF4B8093E80E91C40E9452B38823AF
:1075700019F081E00E940BEC84E50E94A14D81117D
:1075800003C0FF24FA94E1C00E94BE4BE82EF090A5
:107590000007F816B1F3F1E0F81718F40E94DC6E5A
:1075A000D4C020915E0230915F0240916002509100
:1075B000610263962CAF3DAF4EAF5FAF639780E043
:1075C00090E0A8ECB2E480935E0290935F02A093F7
:1075D0006002B09361020E94F24CCE2CD12C0F2D90
:1075E00010E0F601EE0FFF1FEE0FFF1FE851F94FFD
:1075F000D801AA0FBB1FAA0FBB1FA851B94F2D91CD
:107600003D914D915C9160817181828193810F9454
:1076100061054B015C01F601EE0FFF1FEE0FFF1F2E
:10762000E051F94FD801AA0FBB1FAA0FBB1FA051F1
:10763000B94F2D913D914D915C9160817181828115
:1076400093810F9461052B013C01A5019401609188
:10765000D40E7091D50E8091D60E9091D70E0F94C6
:1076600062056093D40E7093D50E8093D60E9093DE
:10767000D70EA30192016091D80E7091D90E80911E
:10768000DA0E9091DB0E0F9462056093D80E709322
:10769000D90E8093DA0E9093DB0EA50194016091D0
:1076A000DC067091DD068091DE069091DF060F9476
:1076B00062056093DC067093DD068093DE0690938E
:1076C000DF0680E00E94064DA30192016091E00672
:1076D0007091E1068091E2069091E3060F946205B5
:1076E0006093E0067093E1068093E2069093E306D0
:1076F00081E00E94064DE09200070E94F6F20E948F
:1077000047F063968CAD9DADAEADBFAD63978093F2
:107710005E0290935F02A0936002B0936102EBE47B
:10772000FAE384918F010F5F1F4F882321F00E949D
:10773000804BF801F6CF6091000770E083E097E09E
:107740000E94DF718AE00E94804B85E40E94A14D77
:10775000882319F00E94DE4B04C060E070E080E0F6
:1077600090EC2F966CAF7DAF8EAF9FAF2F978AE5D1
:107770000E94CF4D882319F00E94DE4B04C060E0C8
:1077800070E080E291E42B966CAF7DAF8EAF9FAF3F
:107790002B9788E50E94CF4D882319F00E94DE4B7D
:1077A00004C060E070E080E291E427966CAF7DAFAA
:1077B0008EAF9FAF279789E50E94CF4D882319F0A0
:1077C0000E94DE4B04C060E070E085E893E42396FD
:1077D0006CAF7DAF8EAF9FAF239785E50E94A14D23
:1077E000882319F00E94DE4B04C060E070E088EC52
:1077F00092EC6BAF7CAF8DAF9EAF8CE40E94A14D3D
:10780000882319F00E94DE4B03C060E070E0CB01DA
:1078100068A379A38AA39BA382E40E94CF4D882307
:1078200021F00E94AE4BB62E02C035E0B32ED090B0
:1078300082128091DA0681119EC0CC24C394EB2C75
:107840008E01055C1F4F9E01215C3F4FAE014D5BD9
:107850005F4FBE01695B7F4FCE01855B9F4F0E94EA
:107860000ACE882309F487C081E08093580711E08D
:1078700080915807882309F46AC060E08B2D0E942C
:10788000B8858091D8069091D906892B09F45BC000
:107890001093CF0640E050E0BA018EEC97ED0E94C5
:1078A0005DBC80915807882321F081E00E949C975D
:1078B000F8CF1092D0061092D1061092D2061092F4
:1078C000D3061092D8060E941E511092D406109230
:1078D000D5061092D6061092D7061092D90681E0EE
:1078E0000E941E510E942CA61093CF0640E050E04B
:1078F000BA0184E296ED0E945DBC0E94C9506853B3
:1079000070458F4F9F4F6093D0067093D106809340
:10791000D2069093D3061092D8060E94C95068539D
:1079200070458F4F9F4F6093D4067093D506809318
:10793000D6069093D7061092D9061093580761E0A7
:107940008B2D0E94B88581E00E949C9791CF80E0AA
:1079500090E0A8E4B2E489839A83AB83BC838091EE
:10796000DA06882341F04B2DBE016F5F7F4FCE01B9
:1079700080960E94CCCC91E09F1520F48F2D0E9420
:10798000DC6ED8C020915E0230915F0240916002AF
:107990005091610263962CAF3DAF4EAF5FAF6397DE
:1079A00080E090E0A8ECB2E480935E0290935F02E6
:1079B000A0936002B093610200910007F01609F4F1
:1079C00093C00E94F24CAF2CB12C10E0F501EE0FE9
:1079D000FF1FEE0FFF1FE851F94FD801AA0FBB1F81
:1079E000AA0FBB1FA851B94F2D913D914D915C91AC
:1079F00060817181828193810F9461052B013C012B
:107A0000F501EE0FFF1FEE0FFF1FE051F94FD801F8
:107A1000AA0FBB1FAA0FBB1FA051B94F2D913D91BB
:107A20004D915C9160817181828193810F94610598
:107A30004B015C01A30192016091D40E7091D50EAF
:107A40008091D60E9091D70E0F9462056093D40E5C
:107A50007093D50E8093D60E9093D70EA501940106
:107A60006091D80E7091D90E8091DA0E9091DB0E54
:107A70000F9462056093D80E7093D90E8093DA0E3E
:107A80009093DB0EA30192016091DC067091DD06FC
:107A90008091DE069091DF060F9462056093DC060C
:107AA0007093DD068093DE069093DF0680E00E94EF
:107AB000064DA50194016091E0067091E106809168
:107AC000E2069091E3060F9462056093E0067093DE
:107AD000E1068093E2069093E30681E00E94064D62
:107AE000F09200070E94F6F20E9447F063968CAD78
:107AF0009DADAEADBFAD639780935E0290935F0284
:107B0000A0936002B0936102EBE4FAE384918F01E9
:107B10000F5F1F4F882321F00E94804BF801F6CFA2
:107B20006091000770E083E097E00E94DF718AE0D7
:107B30000E94804B91E0D912A9C10E941DB4A6C138
:107B40000E941AC9A3C10E94CB73A0C183E50E9401
:107B5000CF4D882309F449C00E94BE4B813039F0D3
:107B6000823009F042C00FE013E0F12C23C00FE097
:107B700013E0F12CD8018D918D010E94CF4D882307
:107B800039F00E94BE4B4FEF682F8F2D0E940A499B
:107B9000F394B4E0FB12EECF82E40E94CF4D882331
:107BA00021F10E94BE4B4FEF682F1CC0F394F4E00C
:107BB000FF1679F0F80181918F010E94CF4D882343
:107BC000A9F30E94BE4B482F6FEF8F2D0E940A49E8
:107BD000EDCF82E40E94CF4D882339F00E94BE4B46
:107BE000482F6FEF84E00E940A490E941F734EC124
:107BF000E4E1FAE384918F010F5F1F4F882321F0A6
:107C00000E94804BF801F6CFE4EFF6E084918F01FB
:107C10000F5F1F4F882309F439C10E94804BF80180
:107C2000F5CF81E0809362021092DB0683E50E942B
:107C3000A14D811103C00E94B77228C10E94CF4B91
:107C4000811124C1F8CF0091080710910907F02E87
:107C500080910007081731F083E50E94A14D811142
:107C60000E94CF4B86E40E94CF4D882319F00E94DA
:107C7000DE4B03C060E070E0CB0121E02F1520F463
:107C8000802F0E94DC6E02C120E030E040E752E429
:107C90000F943E065B016C0120E030E0A9010F94D7
:107CA000880718166CF0A0905E02B0905F022090DA
:107CB00060023090610230E020E098EC82E405C080
:107CC00016013A2D2B2D9C2D832D432F522F692FDA
:107CD000782F40935E0250935F026093600270932E
:107CE0006102E0900007FE1409F493C00E94F24C78
:107CF00048019924F12CF401EE0FFF1FEE0FFF1F36
:107D0000E851F94FD701AA0FBB1FAA0FBB1FA851FB
:107D1000B94F2D913D914D915C916081718182812E
:107D200093810F9461052B013C01F401EE0FFF1FBD
:107D3000EE0FFF1FE051F94FD701AA0FBB1FAA0F8B
:107D4000BB1FA051B94F2D913D914D915C91608128
:107D50007181828193810F9461056B017C01A30184
:107D600092016091D40E7091D50E8091D60E9091B3
:107D7000D70E0F9462056093D40E7093D50E809346
:107D8000D60E9093D70EA70196016091D80E7091F0
:107D9000D90E8091DA0E9091DB0E0F9462056093FC
:107DA000D80E7093D90E8093DA0E9093DB0EA30158
:107DB00092016091DC067091DD068091DE06909163
:107DC000DF060F9462056093DC067093DD068093F6
:107DD000DE069093DF0680E00E94064DA701960123
:107DE0006091E0067091E1068091E2069091E306D1
:107DF0000F9462056093E0067093E1068093E206BB
:107E00009093E30681E00E94064D009300070E94D4
:107E1000F6F20E9447F0A501B10140935E02509333
:107E20005F026093600270936102EBE4FAE3849175
:107E30008F010F5F1F4F882321F00E94804BF801B4
:107E4000F6CF6091000770E083E097E00E94DF7159
:107E50008AE00E94804B1AC0EBE4FAE384918F0120
:107E60000F5F1F4F882321F00E94804BF801F6CF4F
:107E7000609101077091020785E197E00E9483B548
:107E800082E20E94804B8AE00E94804B0E944F72E7
:107E9000A5C34115510519F4AF014150510920E026
:107EA00030E00C94442A80E00E949C970C941D2F93
:107EB0000E94AE4BAB01BC01409334155093351575
:107EC000609336157093371583E894E10E945195BD
:107ED000DDCF802F0E94E78E6E2D802F0E948F5065
:107EE000F12CB701802F0E94068F0630110529F46E
:107EF000F092EF10E092EE10C9CF0830110531F684
:107F0000F092F110E092F010C1CF0E94DE4BF090A1
:107F1000B2060F2D10E0000F111F0F5E124F0F94CD
:107F2000A606D8016D937C938F2D0E941E510E944E
:107F3000DE4B20E030E040E752E40F942F011816AA
:107F400044F00E94879760E089E993E00E9493B92A
:107F500002C00E941DB40091B20610E0F801EE0FBD
:107F6000FF1FEF5EF24F60817181882777FD80955A
:107F7000982F0F943501F801EE0FFF1FEE0FFF1F32
:107F8000ED5AF94F20813181428153810F94880746
:107F900018160CF073C18EED92E09F938F930F5FD4
:107FA0001F4F1F930F938AE893E09F938F931F9225
:107FB0000E9438B30FB6F894DEBF0FBECDBF81E08C
:107FC0008093630267961CAE1DAE1EAE1FAE679710
:107FD0006C961CAE1DAE1EAE1FAE6C97312C6D960E
:107FE0001FAE6D973CE36E963FAF6E974CE16F9678
:107FF0004FAF6F9756E4A0965FAFA097C12CD12CDE
:1080000010E8E12E0FEBF02E812C912C5401009101
:10801000B20610E0F801EE0FFF1FEF5EF24F608135
:108020007181882777FD8095982F0F943501762EE2
:10803000672E582E492E262F372F482F592FB6013D
:10804000C7010F942F018823F9F0F801EE0FFF1FED
:10805000EE0FFF1FED5AF94F20813181428153818C
:10806000672D762D852D942D0F942F01382E331CDE
:108070003324331C60968FAD6097882349F03320FA
:1080800039F033243394E8C07C2C6D2C5E2C4F2CBB
:108090000E94C9506B017C01DC01CB016C962CADB8
:1080A0003DAD4EAD5FAD6C97821B930BA40BB50B32
:1080B000B7FD3AC0D701C60188519C4FAF4FBF4FA3
:1080C0006C968CAF9DAFAEAFBFAF6C970E94AD63A7
:1080D000E6E8F3E084918F010F5F1F4F882321F0C2
:1080E0000E94804BF801F6CF81149104A104B104E1
:1080F000A9F0C501B40168517C4F8F4F9F4F6C1997
:108100007D098E099F0928EE33E040E050E00F948E
:108110000405CA01B9010E94027003C08FE30E94E6
:10812000804B8AE00E94804B80E00E949C970E94D6
:10813000FB51E091B20694E0E99FF0011124ED5A61
:10814000F94F2080A1816896AFAF689702811381B3
:10815000222D3A2FA801672D762D852D942D0F9471
:1081600061059F7720E030E040E251E48114910402
:10817000A104B10429F40F942F0187FD05C006C0A6
:108180000F948807181614F446015701332009F498
:1081900049C067962CAD3DAD4EAD5FAD67972115DB
:1081A00031054105510541F0D701C601821B930BF2
:1081B000A40BB50BB7FD36C0222D68963FAD68976E
:1081C000A8016D966FAD6D976E967FAD6E976F96A9
:1081D0008FAD6F97A0969FADA0970F94610520E09B
:1081E00030E040EC5FE30F942F0187FD4ACFD701C9
:1081F000C601805A9541AF4FBF4F67968CAF9DAF78
:10820000AEAFBFAF67976D962FAE6D9768969FAD77
:1082100068976E969FAF6E976F960FAF6F97A09609
:108220001FAFA097809163028823B1F0811491045D
:10823000A104B10429F4C72CD62CE52CF42CE7CEEC
:10824000A8EECA1AA3E0DA0AE108F108C818D908AA
:10825000EA08FB08F7FCEFCF80916302882309F45A
:1082600015CE60E0332029F08AE693E00E9493B9AE
:108270000DCE88E793E00E9493B908CE6096BFAD1B
:108280006097B1119CCE89EE92E087CE0E94DE4BC2
:108290000F94A6066739710514F066E970E07093D3
:1082A0000E0D60930D0D0E94D5500E94DE4B20E014
:1082B00030E040EA50E40F948807181614F40E9446
:1082C0001DB460910D0D70910E0D882777FD80957E
:1082D000982F0F94350120915B0630915C064091F8
:1082E0005D0650915E060F942F0160E087FF03C08A
:1082F00089EC93E002C08CEB93E00E9493B981E09B
:1083000080936302809100078093B20667961CAE4B
:108310001DAE1EAE1FAE67976C961CAE1DAE1EAE98
:108320001FAE6C9760961FAE60976D961FAE6D97EF
:10833000BCE36E96BFAF6E97ECE16F96EFAF6F97B1
:10834000F6E4A096FFAFA097C12CD12C70E8E72EE1
:10835000EFEBFE2E812C912C540160910D0D70914C
:108360000E0D882777FD8095982F0F943501162FD5
:10837000072F782E692E262F372F482F592FB60119
:10838000C7010F942F01882331F120915B063091B2
:108390005C0640915D0650915E06612F702F872D1F
:1083A000962D0F942F01881F8827881F60968FAF06
:1083B000609768962FAD6897222389F0882379F01B
:1083C00080916302882309F461CD60E08EEA93E036
:1083D0000E9493B95BCD1C2D0D2D7E2C6F2C0E941D
:1083E000C9506B017C01DC01CB016C962CAD3DAD1D
:1083F0004EAD5FAD6C97821B930BA40BB50BB7FD15
:108400003BC0D701C60188519C4FAF4FBF4F6C9600
:108410008CAF9DAFAEAFBFAF6C970E94AD63E8EB82
:10842000F3E084912F019FEF491A590A882321F024
:108430000E94804BF201F5CF81149104A104B10494
:10844000A9F0C501B40168517C4F8F4F9F4F6C1943
:108450007D098E099F0928EE33E040E050E00F943B
:108460000405CA01B9010E94027003C08FE30E9493
:10847000804B8AE00E94804B80E00E949C970E9483
:10848000FB5120905B0630905C0640905D0650905A
:108490005E069101A201612F702F872D962D0F94FA
:1084A00061059F7720E030E040EA50E481149104B8
:1084B000A104B10429F40F942F0187FD05C006C063
:1084C0000F948807181614F4460157016096AFAD53
:1084D0006097AA2309F443C067962CAD3DAD4EAD1D
:1084E0005FAD6797211531054105510541F0D70171
:1084F000C601821B930BA40BB50BB7FD30C09101D5
:10850000A2016D966FAD6D976E967FAD6E976F966B
:108510008FAD6F97A0969FADA0970F94610520E057
:1085200030E040EC5FE30F942F0187FD49CFD70186
:10853000C601805A9541AF4FBF4F67968CAF9DAF34
:10854000AEAFBFAF67976D962FAE6D976E963FAE8D
:108550006E976F964FAE6F97A0965FAEA097809183
:108560006302882309F42CCF81149104A104B1047F
:1085700029F4C12ED02EE72CF62CEFCE98EEC91A96
:1085800093E0D90AE108F108C818D908EA08FB08FD
:10859000F7FE16CFEECF0E9447F088E50E94A14D6E
:1085A000882319F0179A1092C30E89E50E94A14DF5
:1085B000882319F0169A1092C40E8AE50E94A14DE4
:1085C000882319F0159A1092C50E85E40E94A14DDA
:1085D000882309F45BCC0E940F4C58CCC15ADF4F62
:1085E0000FB6F894DEBF0FBECDBFDF91CF911F91C4
:1085F0000F91FF90EF90DF90CF90BF90AF909F9042
:108600008F907F906F905F904F903F902F90089544
:10861000CF92DF92EF92FF920F931F93CF93DF934E
:108620007C016A01EB0100E010E00C151D0571F002
:108630006991D701ED91FC910190F081E02DC70186
:108640001995892B19F00F5F1F4FEFCFC801DF91EC
:10865000CF911F910F91FF90EF90DF90CF900895F1
:10866000089580E090E0089580E00895FC01E60F11
:10867000F11D849190E0982F88273196E4918E0F18
:10868000911D08950895DC011696ED91FC911797C0
:1086900012968C911297481B15968C91483018F0C1
:1086A000E80FF11D4770869586958695489F402D69
:1086B0001124E40FF11D362F377080E890E002C0DE
:1086C000959587953A95E2F7669566956695E60FD6
:1086D000F11D3081222311F0832B02C0809583236A
:1086E0008083089581E00895089590E0FC0131971A
:1086F000E231F10508F04CC0EE58FF4F0D944D08E3
:10870000809180008F7703C0809180008F7D80935F
:108710008000089580918000877FF9CF84B58F779E
:1087200002C084B58F7D84BD08958091B0008F779D
:1087300003C08091B0008F7D8093B0000895809138
:1087400090008F7707C0809190008F7D03C080914B
:108750009000877F8093900008958091A0008F778C
:1087600007C08091A0008F7D03C08091A000877F0B
:108770008093A0000895809120018F7707C0809199
:1087800020018F7D03C080912001877F809320018D
:1087900008953FB7F8948091F5119091F611A0914A
:1087A000F711B091F81126B5A89B05C02F3F19F01D
:1087B0000196A11DB11D3FBF6627782F892F9A2FE3
:1087C000620F711D811D911D42E0660F771F881F8A
:1087D000991F4A95D1F708952FB7F8949091050104
:1087E0009B7F909305012FBF87FD96C0A3982FB75D
:1087F000F894909105019460909305012FBF880F24
:108800002FB7F894909105019B7F909305012FBF9E
:1088100087FD8EC0A3982FB7F894909105019460BE
:10882000909305012FBF880F2FB7F8949091050101
:108830009B7F909305012FBF87FD78C0A3982FB72A
:10884000F894909105019460909305012FBF880FD3
:108850002FB7F894909105019B7F909305012FBF4E
:1088600087FD62C0A3982FB7F8949091050194609A
:10887000909305012FBF880F2FB7F89490910501B1
:108880009B7F909305012FBF87FD4CC0A3982FB706
:10889000F894909105019460909305012FBF880F83
:1088A0002FB7F894909105019B7F909305012FBFFE
:1088B00087FD36C0A3982FB7F89490910501946076
:1088C000909305012FBF982F990F2FB7F89480919F
:1088D00005018B7F809305012FBF97FD1FC0A398D3
:1088E0002FB7F894809105018460809305012FBF14
:1088F0002FB7F894809105018B7F809305012FBFDE
:1089000096FD18C0A3989FB7F894809105018460E4
:10891000809305019FBF0895A39A69CFA39AE0CFE2
:10892000A39AC9CFA39AB3CFA39A9DCFA39A87CF77
:10893000A39A71CFA39AE7CFFC0120E03EE2DB01CE
:108940004C91403241F0283011F430833196DB01F4
:108950004C91408331962F5F6F5F7F4F2B3079F7BB
:10896000108208954F925F926F927F928F929F92A2
:10897000AF92BF92CF92DF92EF92FF920F931F932D
:10898000CF93DF932C012BE338E081E090E0F901F5
:1089900045915491441655060CF062C0AC0141500B
:1089A0005109DA01AA0FBB1FAA0FBB1FA75CB74F63
:1089B000FD0165917491440F551F440F551F495C8B
:1089C000574FFA0165907490FC01EE0FFF1FEE0FF8
:1089D000FF1FE75CF74FA590B490FD01059114913E
:1089E000F901C591D491FA0185909490882777FD7B
:1089F0008095982F0F9435016B017C01B2016619A7
:108A00007709882777FD8095982F0F9435012B01E2
:108A10003C01B501601B710B882777FD8095982F6D
:108A20000F9435019B01AC01C301B2010F94940175
:108A30002B013C01BE0168197909882777FD8095D3
:108A4000982F0F9435019B01AC01C301B2010F9423
:108A50003E069B01AC01C701B6010F94620511C02F
:108A600001962C5F3F4F8A33910509F090CFEDE1DD
:108A7000F9E065917491882777FD8095982F0F9480
:108A80003501DF91CF911F910F91FF90EF90DF9013
:108A9000CF90BF90AF909F908F907F906F905F909E
:108AA0004F9008954F925F926F927F928F929F9214
:108AB000AF92BF92CF92DF92EF92FF92CF93DF936C
:108AC000CDB7DEB72C970FB6F894DEBF0FBECDBF83
:108AD00080915B0690915C06A0915D06B0915E0668
:108AE00089839A83AB83BC8360910D0D70910E0DC9
:108AF000882777FD8095982F0F94350129813A8139
:108B00004B815C810F9461056B017C01609354077C
:108B100070935507809356079093570720913D1106
:108B200030913E1140913F11509140110F949401AA
:108B30006D837E838F83988760935007709351076E
:108B4000809352079093530720914C0730914D0723
:108B500040914E0750914F07C701B6010F9462052F
:108B60004B015C0160934C0770934D0780934E0757
:108B700090934F072091391130913A1140913B1158
:108B800050913C110F94940169877A878B879C8759
:108B9000609348077093490780934A0790934B0767
:108BA00020ED3CEC4CE45DE36091351170913611A1
:108BB00080913711909138110F9494012B013C0151
:108BC000209144073091450740914607509147074F
:108BD00069817A818B819C810F9461059B01AC0135
:108BE000C301B2010F9494012B013C0123E333E351
:108BF00043E75FE36091400770914107809142072E
:108C0000909143070F9494019B01AC01C301B20101
:108C10000F9462052B013C0160934007709341075C
:108C2000809342079093430789819A81AB81BC81ED
:108C30008093440790934507A0934607B093470756
:108C400029853A854B855C856D817E818F819885EC
:108C50000F946205A30192010F9461052B013C0161
:108C600020E030E04EE453E40F94880720E030E049
:108C7000A9011816ACF4C701B6010F94880718169D
:108C80006CF5A7019601C501B4010F9461056093CD
:108C90004C0770934D0780934E0790934F071EC06B
:108CA000C301B2010F942F0187FF22C020E030E002
:108CB000A901C701B6010F942F0187FF16C0A701B4
:108CC0009601C501B4010F94610560934C07709340
:108CD0004D0780934E0790934F0707C0412C512CAE
:108CE0008EE4682E83E4782E03C0412C512C32018F
:108CF000C301B2012C960FB6F894DEBF0FBECDBFF4
:108D0000DF91CF91FF90EF90DF90CF90BF90AF9029
:108D10009F908F907F906F905F904F9008952F92CB
:108D20003F924F925F926F927F928F929F92AF92FB
:108D3000BF92CF92DF92EF92FF920F931F93CF9348
:108D4000DF93CDB7DEB72A970FB6F894DEBF0FBE1C
:108D5000CDBF082F112707FD1095F801EE0FFF1F5B
:108D6000EF5EF24F20803180C801880F991F880F75
:108D7000991F9A878987FC01ED5AF94F808091806D
:108D8000A280B380B101882777FD8095982F0F943A
:108D90003501A50194010F9461056B017C01E98502
:108DA000FA85E85CF84F608371838283938320EDBA
:108DB0003CEC4CE45DE36091291170912A118091A3
:108DC0002B1190912C110F9494012B013C01A9853A
:108DD000BA85A05DB84FBE83AD832D913D914D9175
:108DE0005C91C501B4010F9461059B01AC01C30105
:108DF000B2010F9494012B013C01E985FA85E85DED
:108E0000F84FF887EF8323E333E343E75FE36081C1
:108E10007181828193810F9494019B01AC01C30104
:108E2000B2010F94620569837A838B839C83AF813F
:108E3000B8856D937D938D939C931397ED81FE81FF
:108E400080829182A282B382F801E852F94F808138
:108E50000A5D184F81111AC020E030E040E251E471
:108E6000C701B6010F948807181624F481E0F801B1
:108E70008083A2C020E030E040E251ECC701B6019F
:108E80000F942F0187FD02C0232821F481E0D8012F
:108E90008C9399C0F8018081882351F0E985FA8587
:108EA000E25EF84F1082118212821382D8011C9266
:108EB0002091311130913211409133115091341180
:108EC000C701B6010F9494012B013C01E985FA8595
:108ED000EA5EF84F608371838283938309851A85E4
:108EE000025E184FF8012081318142815381C70110
:108EF000B6010F9462054B015C01D8016D937D931F
:108F00008D939C93139720912D1130912E114091A8
:108F10002F11509130110F9494019B01AC01E98500
:108F2000FA85E25FF84F6083718382839383C30184
:108F3000B2010F94620529813A814B815C810F94C3
:108F400061052B013C0120E030E04FE753E40F9432
:108F5000880720E030E0A901181694F4C701B60193
:108F60000F948807181644F5A7019601C501B401AE
:108F70000F946105F80160837183828393831CC021
:108F8000C301B2010F942F0187FF20C020E030E021
:108F9000A901C701B6010F942F0187FF14C0A701D3
:108FA0009601C501B4010F946105D8016D937D93BD
:108FB0008D939C93139707C0412C512C9FE7692EEA
:108FC00093E4792E03C0412C512C3201C301B2012C
:108FD0002A960FB6F894DEBF0FBECDBFDF91CF91BA
:108FE0001F910F91FF90EF90DF90CF90BF90AF90C7
:108FF0009F908F907F906F905F904F903F902F90B9
:10900000089560915B0670915C0680915D06909179
:109010005E06089594E0899FF0011124ED5AF94FFE
:10902000608171818281938108952F923F924F9246
:109030005F926F927F928F929F92AF92BF92CF92E8
:10904000DF92EF92FF920F931F93CF93DF9300D0A5
:109050001F92CDB7DEB72C0170E0FB01EE0FFF1FB2
:10906000EB5EFC4F208131813C832B83232B09F461
:10907000A2C0FB01ED5EFC4F30813A832B813C8125
:109080002C5F3F4F81E090E08983EA818E1708F0E2
:1090900077C0DC01F901459154910196B9016C5FEB
:1090A0007F4F441655060CF069C00297AC01440F7F
:1090B000551F440F551F4E5F5F4F6B817C81460FDC
:1090C000571FFA0165917491880F991F880F991F96
:1090D000EB81FC818E0F9F1FFC0165907490FD0158
:1090E000EE0FFF1FEE0FFF1F3296AB81BC81EA0F20
:1090F000FB1FA590B490FA0105911491F901859098
:109100009490FC0125903490882777FD8095982FC6
:109110000F9435016B017C01B2016619770988272C
:1091200077FD8095982F0F9435012B013C01B501F7
:10913000601B710B882777FD8095982F0F94350160
:109140009B01AC01C301B2010F9494012B013C01BE
:10915000B40162197309882777FD8095982F0F94C1
:1091600035019B01AC01C301B2010F943E069B0186
:10917000AC01C701B6010F94620506C09B0184CF04
:1091800060E070E080E090E0F9812A81F2132BC06A
:109190002B813C8144E0F49F200D311D112422508D
:1091A0003109F90165917491882777FD8095982F91
:1091B0000F94350118C0BC01882777FD8095982F42
:1091C0000F94350120E030E04AEF5EE30F94940104
:1091D00020E030E040E85DE30F94940120E030E0CF
:1091E000A9010F9462050F900F900F900F90DF91DF
:1091F000CF911F910F91FF90EF90DF90CF90BF9094
:10920000AF909F908F907F906F905F904F903F9026
:109210002F90089567FD5CC0823021F128F48823E7
:1092200049F0813069F054C0833071F1843009F421
:109230003DC04EC0662311F0A19A8FC0A1988DC089
:109240009FB7662329F0F89480910801806804C0D4
:10925000F894809108018F77809308019FBF47FFA2
:109260004CC07FC09FB7662329F0F8948091080115
:10927000806404C0F894809108018F7B809308017A
:109280009FBF47FF40C06FC09FB7662329F0F89487
:1092900080910801886004C0F89480910801877F5C
:1092A000809308019FBF47FF3EC05AC09FB7662307
:1092B00029F0F89480910801826004C0F8948091AC
:1092C00008018D7F809308019FBF47FF39C04AC0C6
:1092D00047FD49C08230B9F028F4882341F081303D
:1092E00061F008958330F9F0843051F108954423FA
:1092F00011F0A09A0895A0980895442311F0A29A1D
:109300000895A29808959FB7442329F0F894809176
:109310000801806204C0F894809108018F7D8093D9
:1093200008019FBF08959FB7442329F0F8948091C6
:1093300008018061F4CFF894809108018F7EEFCF0F
:109340009FB7442329F0F894809108018460E7CF07
:10935000F894809108018B7FE2CF47FFC8CF089532
:109360000895089508950895643079F028F46130DF
:1093700041F0623041F00895683051F0603141F0C1
:10938000089540E003C040E004C041E060E002C056
:1093900041E061E03FCF24E08202C0011124FC01E2
:1093A000EE52F34F4081518162817381FC01E350A1
:1093B000F14F4083518362837383E091050DF091F7
:1093C000060D82899389A489B5898093E20C9093D4
:1093D000E30CA093E40CB093E50C0895CF93DF93D6
:1093E0002FB7F89494E08902E0011124FE01EE52B7
:1093F000F34F60817181828193812FBF0F9435017A
:10940000C751D14F288139814A815B810F949401E2
:10941000DF91CF9108958091040D9FB780FF09C01F
:10942000F89480910B018D7F80930B019FBF8FEF8C
:1094300008C0F89480910B01826080930B019FBF5C
:1094400081E0809364028091040D9FB781FF09C081
:10945000F89480910B01816080930B019FBF8FEF87
:1094600008C0F89480910B018E7F80930B019FBF01
:1094700081E0809365028091040D9FB782FF09C04F
:10948000F89480910B018B7F80930B019FBF8FEF2E
:1094900008C0F89480910B01846080930B019FBFFA
:1094A00081E0809366028091040DE091050DF091BA
:1094B000060D83FF12C081819FB7811105C0F8940A
:1094C00080910B01806404C0F89480910B01806846
:1094D00080930B019FBF8FEF11C081819FB78111D6
:1094E00005C0F89480910B018F7B04C0F8948091A3
:1094F0000B018F7780930B019FBF81E08093670200
:1095000008954F925F926F927F92AF92BF92CF92E7
:10951000DF92EF92FF920F931F93CF93DF938C0113
:10952000EB01FC0147A050A461A472A4AFA0B8A4B1
:10953000C9A4DAA49501A601C301B2010F942F01B9
:1095400087FF40C0A3019201C301B2010F949401AF
:109550002B013C01F80183A994A9A5A9B6A9BC01D6
:10956000CD0190589B01AC010F946205F80127A52D
:1095700030A941A952A90F9494019B01AC01C301E8
:10958000B2010F9461050F94CD077B018C019B0103
:10959000AC01B501C6010F942F0187FF02C0750110
:1095A00086019701A801B501C6010F942F018823F8
:1095B00049F0A701B8014FA358A769A77AA78881E6
:1095C00081608883DF91CF911F910F91FF90EF9081
:1095D000DF90CF90BF90AF907F906F905F904F9053
:1095E00008954F925F926F927F928F929F92AF9267
:1095F000BF92CF92DF92EF92FF920F931F93CF9380
:10960000DF9300D01F92CDB7DEB70091000710E0C6
:109610000D5F1F4F83EFE82E80E1F82E94ED692E49
:1096200091E1792E23E6C22E26E0D22E412C512C38
:10963000812C912C54018394F70161917191819156
:1096400091917F01F30121913191419151913F011C
:1096500029833A834B835C830F94330129813A81B8
:109660004B815C810F9494010F94AB06F6016193DA
:109670007193819391936F01F2E0F41518F4401601
:10968000510639F486169706A806B90610F44B0160
:109690005C012FEF421A520A85E04816510461F628
:1096A0006FEF7FEFCB01A50194010F940405209388
:1096B000AA0E3093AB0E4093AC0E5093AD0E0F90AC
:1096C0000F900F900F90DF91CF911F910F91FF900E
:1096D000EF90DF90CF90BF90AF909F908F907F9052
:1096E0006F905F904F9008958EBD0DB407FEFDCF33
:1096F00008958FEF8EBD0DB407FEFDCF8EB5089592
:109700009091C00095FFFCCF8093C60008953FB7AD
:10971000F8942091DB078091DA07821759F0E22F45
:10972000F0E0E65AF84F808190E02F5F2F7720938A
:10973000DB0702C08FEF9FEF3FBF089580910C07BA
:1097400090910D07009731F04AE050E060E070E042
:109750000C946FFF60E070E0CB01089580910C07DE
:1097600090910D07009731F04AE050E060E070E022
:109770000C943EFE60E070E0CB010895EFDF97FDB2
:109780000CC0ECDF6F3F71058105910509F014F401
:10979000E5DF01C06FEF862F089580E00895809186
:1097A0000C0790910D07892B39F0E8DF91E08111CA
:1097B00001C090E0892F089581E008951F93CF9311
:1097C000DF9380910C0790910D070097E1F0FC0169
:1097D000EF011191212F2F7D79F0153411F01536FD
:1097E000B9F7188260E070E00E94D6FC1883562F0B
:1097F000472F382F292F0BC060E070E0DF91CF9109
:109800001F910C94D6FC50E040E030E020E0652F42
:10981000742F832F922FDF91CF911F910895149A67
:10982000139A0895179A1092C30E169A1092C40EA6
:10983000159A1092C50EF3CFCF92DF92EF92FF925E
:10984000CF93C0918106C0907906D0907A06E090BF
:109850007B06F0907C06CC2321F120E030E0A901CA
:10986000C701B6010F942F018823D9F020E030E022
:1098700040E05FE3C701B6010F9494019B01AC0186
:109880000F9494012BED3FE049E450E40F949401D0
:109890009B01AC0160E070E080E89FE30F943E061E
:1098A00004C060E070E080E89FE36093B00E7093C6
:1098B000B10E8093B20E9093B30EC0907D06D090FF
:1098C0007E06E0907F06F0908006CC2321F120E018
:1098D00030E0A901C701B6010F942F018823D9F008
:1098E00020E030E040E05FE3C701B6010F9494014F
:1098F0009B01AC010F9494012BED3FE049E450E44F
:109900000F9494019B01AC0160E070E080E89FE35C
:109910000F943E0604C060E070E080E89FE360932F
:10992000B40E7093B50E8093B60E9093B70ECF9190
:10993000FF90EF90DF90CF900895CF92DF92EF925B
:10994000FF92CF93DF93EC0180915102882309F4B9
:1099500042C0C0905202D0905302E0905402F09066
:109960005502A7019601688179818A819B810F94B4
:109970008807181624F4C882D982EA82FB82C09034
:109980005602D0905702E0905802F0905902A70179
:1099900096016C817D818E819F810F9488071816B6
:1099A00024F4CC82DD82EE82FF82C0905A02D090F5
:1099B0005B02E0905C02F0905D02A7019601688571
:1099C00079858A859B850F948807181624F4C886A4
:1099D000D986EA86FB86DF91CF91FF90EF90DF90EA
:1099E000CF90089580E1E4EDFEE0A6E3B4E00190BD
:1099F0000D928A95E1F7089580E1E6E3F4E0A4EDA5
:109A0000BEE001900D928A95E1F70895AF92BF9262
:109A1000CF92DF92EF92FF920F931F93CF93DF933A
:109A2000C82FDD27C7FDD0958E01000F111F000F35
:109A3000111FF801E853F14F20E030E0A9016081E7
:109A40007181828193810F946205F801E452F94F8C
:109A500020813181428153810F9462056B017C0129
:109A6000F801ED54F94F6083718382839383085129
:109A7000184FF80165917591859194918E01000FB1
:109A8000111F000F111F98012154394F5901A701CF
:109A900096010F946205F50160837183828393833D
:109AA0000C50184FF8016591759185919491CC0FE8
:109AB000DD1FCC0FDD1FCE5ADD4FA70196010F949D
:109AC0006205688379838A839B83DF91CF911F919D
:109AD0000F91FF90EF90DF90CF90BF90AF900895DF
:109AE0009091540DE92FF0E0EC51F14F80839F5F8E
:109AF000943018F49093540D02C01092540D80913C
:109B00008B108F5F80938B100895CF93FC01C62F2D
:109B100080818B3399F080918B10843078F4209180
:109B2000540D30E6239FC0011124BF01865F904F82
:109B30000F949E088C2FD4DF81E001C080E0CF918C
:109B4000089581548A3148F5482F50E0FA01A3E086
:109B5000F595E795AA95E1F7EE5CFB4F208130E0A3
:109B6000877002C0359527958A95E2F720FF15C0CA
:109B7000FA01E85EFB4F2081222339F08091010732
:109B800090910207820F911D02C080E090E09093B7
:109B90000D0780930C0781E0089580E00895D1DFE0
:109BA000882339F081E020910C0730910D07232B99
:109BB00009F480E00895DF92EF92FF920F931F93D4
:109BC000CF93DF9383E5EBDF882311F0D7DD01C06E
:109BD00080E080930B07EBE4FAE38491EF01219698
:109BE000882319F08DDDFE01F8CFE0E3F8E08491E1
:109BF000EF012196882319F083DDFE01F8CF8091D3
:109C00000B07882371F102E218E0C0E0D0E020E009
:109C100080910B0790E00C2E02C0959587950A94D1
:109C2000E2F780FF15C0DD24D394D20E222311F079
:109C30008CE266DDF80125913491F9018491790176
:109C4000FFEFEF1AFF0A882321F05ADD9701F5CFC5
:109C5000D22E21960E5F1F4FC530D10561F02D2DFC
:109C6000D7CFECE2F8E08491EF012196882319F038
:109C700047DDFE01F8CF8AE0DF91CF911F910F9170
:109C8000FF90EF90DF903CCDCF93DF9383E587DFAC
:109C9000882311F063DD02C060E070E0EB01DD2796
:109CA000C230D105A8F0E4E1FAE38491EF012196F6
:109CB000882319F025DDFE01F8CFE0E0F8E084917B
:109CC000EF012196882309F447C01ADDFE01F7CF82
:109CD00088E465DF8823A1F041DD683771053CF039
:109CE000633281E078072CF062E271E002C068E73D
:109CF00070E0FE01EE0FFF1FED5BF24F718360839A
:109D000086E44DDF882391F029DD6F3F710519F05E
:109D100014F06FEF70E0FE01EE0FFF1FE55CF24FF5
:109D200077FF02C060E070E07183608382E437DF18
:109D3000882391F013DD6530710534F068387105C2
:109D40002CF067E870E002C065E070E0CC0FDD1F2A
:109D5000C15CD24F79836883DF91CF910895CF9210
:109D6000DF92EF92FF920F931F93CF93DF932FE039
:109D7000E22E23E0F22E06E314E0C4EDDEE033E051
:109D8000C32E37E0D32EF70181917F01DADE8823DD
:109D9000C9F014DDF6012081211104C020910707CC
:109DA000222329F0288139814A815B8103C020E088
:109DB00030E0A9010F946205F8016083718382830A
:109DC000938309C088819981AA81BB81F80180832E
:109DD0009183A283B3830C5F1F4F2496FFEFCF1AAA
:109DE000DF0A83E1E81683E0F80669F686E4D7DE49
:109DF0008823B9F0E3DC20E030E0A9010F94880764
:109E000018167CF4DBDC20E030E040E752E40F94ED
:109E10003E0660935E0270935F02809360029093AF
:109E20006102DF91CF911F910F91FF90EF90DF9032
:109E3000CF900895CF93DF939091DB1091111CC0C8
:109E400094E0899FE0011124CD5AD94F6091880296
:109E500070918902882777FD8095982F0F9435019E
:109E60009B01AC01688179818A819B810F942F01CC
:109E7000881F8827881F01C080E0DF91CF91089557
:109E80008091621290916312891B8F7008950B96D6
:109E9000FC01849108950A96FC018491089568E07C
:109EA0000C94364366E00C943643FC01849108958B
:109EB000FCDF882311F0823011F486E0089583E0FE
:109EC0000895FB014181DC0112962C9112974217F3
:109ED00068F013962C911397241740F06081159623
:109EE0002C91621718F424810C9443430895FC01CB
:109EF00020818281820F82839181891760F484811D
:109F00008F5F84838381820F891710F08FEF890F11
:109F1000838381E0089580E00895FC0112828081AE
:109F2000815083831482089588E290E00197F1F7CD
:109F300008952EE93FE0009729F0F9013197F1F7F4
:109F40000197F9CF08950F93FC010150040F84A9E4
:109F500096A9941718F0081728F402C0081750F0B3
:109F6000041740F42150260F83A995A9961720F4D1
:109F7000281720F480E007C0281720F481E0261776
:109F800010F0F8CF81E00F910895DB01ED91FC9185
:109F90001994EF92FF920F931F93CF93DF931F9229
:109FA000CDB7DEB78C01DC011296ED90FC901397D3
:109FB000D196ED91FC91D29782E0199520E030E0A6
:109FC0004AE0B701C801E1DFF82ED801D196ED9142
:109FD000FC91D29783E01995D801D196ED91FC912F
:109FE000D29780E01995FF2081F1F8016281738199
:109FF0009E012F5F3F4F46E4C801C7DF8981D8012A
:10A000008C9312966D917C9113979E012F5F3F4F19
:10A0100047E4C801BADF8981F801818362817381D5
:10A0200020E030E048E4C801B0DFD8011B968C93F3
:10A030001B9798012D5C3F4F12966D917C91139761
:10A0400047E1C801A2DF81E001C080E00F90DF910D
:10A05000CF911F910F91FF90EF9008958F929F9253
:10A06000AF92BF92CF92DF92EF92FF926B017C0191
:10A070000E94C9434B015C01C114D104E104F10405
:10A08000E1F00E94C943681979098A099B09683E71
:10A0900073408105910580F321E0C21AD108E108DF
:10A0A000F10888EE880E83E0981EA11CB11CC11433
:10A0B000D104E104F10429F7DFCFFF90EF90DF90A6
:10A0C000CF90BF90AF909F908F900895CF93DF93E4
:10A0D000282F30E0F901E751F94C8491F901E15161
:10A0E000F84CD491F901EB5CF74CC491CC2391F07E
:10A0F00081110E947543EC2FF0E0EE0FFF1FE25339
:10A10000F84FA591B4912C912D2381E090E021F49A
:10A1100080E002C080E090E0DF91CF9108950F933E
:10A120001F93CF93DF931F92CDB7DEB7282F30E078
:10A13000F901E751F94C8491F901E151F84C14917E
:10A14000F901EB5CF74C04910023C9F0882321F05E
:10A1500069830E9475436981E02FF0E0EE0FFF1FD5
:10A16000E153F94CA591B4919FB7F8948C9161118A
:10A1700003C01095812301C0812B8C939FBF0F904A
:10A18000DF91CF911F910F91089561E0FC018081D3
:10A19000C6CF2FB7F8946091FA117091FB1180919E
:10A1A000FC119091FD112FBF0895CF92DF92EF9295
:10A1B000FF92C0905B06D0905C06E0905D06F09048
:10A1C0005E0660910D0D70910E0D68507109882723
:10A1D00077FD8095982F0F9435019B01AC01C70145
:10A1E000B6010F942F0187FF1CC020E030E040E053
:10A1F00050E4C701B6010F9462050F94AB0670934B
:10A20000690E6093680EC5DF605A75418F4F9F4F8E
:10A2100060936A0E70936B0E80936C0E90936D0E2C
:10A2200008C010926A0E10926B0E10926C0E109273
:10A230006D0EFF90EF90DF90CF900895CF92DF9258
:10A24000EF92FF920F931F93CF93DF93082F10E0AD
:10A25000E801CC0FDD1FCC0FDD1FFE01ED5AF94FD9
:10A26000C080D180E280F380000F111FF801EF5E03
:10A27000F24F6081718165517109882777FD809562
:10A28000982F0F9435019B01AC01C701B6010F94C3
:10A290002F01CE58D14F87FF19C00259114F20E02E
:10A2A00030E040E251E4C701B6010F9462050F941B
:10A2B000AB06F801718360836CDF605C73468F4F7F
:10A2C0009F4F688379838A839B8304C01882198295
:10A2D0001A821B82DF91CF911F910F91FF90EF9017
:10A2E000DF90CF9008950F931F93CF93DF93EB01EF
:10A2F00050DF8B01FED98F3F41F04BDF601B710BAC
:10A300006C177D07B8F380E001C081E0DF91CF9149
:10A310001F910F910895CF92DF92FF920F931F9399
:10A32000CF93DF9300D01F92CDB7DEB76C01F62E2E
:10A33000FC018281982F906A96959CBD80FD06C095
:10A3400091E0863009F490E0892F01C080E08DBD56
:10A3500060E0F601808129833A834B835C83DFDEF2
:10A360006CE271E0C601BFDF8F2D8064BDD908E1CA
:10A3700010E05C814B813A812981DA01C901002E0C
:10A3800004C0B695A795979587950A94D2F7298327
:10A390003A834B835C83A8D90850110929813A81FB
:10A3A0004B815C81083FFFEF1F0739F7FF2029F041
:10A3B00088E0F81621F08FEF03C085E901C087E837
:10A3C00093D9ECE0FE1201C094D910E092D9F601C5
:10A3D000838387FF04C01F3F11F01F5FF7CF0F90EB
:10A3E0000F900F900F90DF91CF911F910F91FF90E1
:10A3F000DF90CF900895CDDE6093460470934704BC
:10A40000809348049093490408951F920F920FB6C9
:10A410000F9211240BB60F922F933F934F935F939C
:10A420006F937F938F939F93AF93BF93EF93FF931C
:10A430008091320D9091330DA091340DB091350D76
:10A44000892B8A2B8B2B59F19091310DE0912F0D97
:10A45000F091300D8081892780838091320D909119
:10A46000330DA091340DB091350D181619061A064A
:10A470001B060CF055C08091320D9091330DA091C8
:10A48000340DB091350D0197A109B1098093320DBA
:10A490009093330DA093340DB093350D41C080914E
:10A4A0006C02EAEBF1E1E4919FEF90936C02E230F1
:10A4B000C9F050F4EE2399F0E13081F590916F00EE
:10A4C0009D7F90936F002AC0E43019F1E0F0E530F1
:10A4D00029F5909173009D7F909373001FC0109297
:10A4E0006E001CC0909170009D7F9093700091E071
:10A4F0009093B0009091B100987F94609093B100D8
:10A500001092B3000BC0909171009D7F90937100E9
:10A5100005C0909172009D7F9093720060E0FFDD16
:10A52000FF91EF91BF91AF919F918F917F916F912B
:10A530005F914F913F912F910F900BBE0F900FBEE7
:10A540000F901F9018951F920F920FB60F92112423
:10A550000BB60F921F932F933F934F935F936F937D
:10A560007F938F939F93AF93BF93CF93DF93EF939B
:10A57000FF9380912E0D8111BBC181E080932E0D40
:10A5800080916E008B7F80936E00789480916B0237
:10A590008F3778F18F5790912C0D90932B0D2FB70B
:10A5A000992329F0F89490910201906404C0F894E2
:10A5B000909102019F7B909302012FBF90912D0DEE
:10A5C00090932A0D2FB7992329F0F89490910201C6
:10A5D000906104C0F894909102019F7E90930201D3
:10A5E0002FBF9091290D9093280D9923F1F0759A22
:10A5F0001DC090912B0D891740F02FB7F8949091C2
:10A6000002019F7B909302012FBF90912A0D891721
:10A6100040F02FB7F894909102019F7E9093020131
:10A620002FBF9091280D891708F075988F5F809340
:10A630006B028091270D91E089278093270D81116E
:10A640000E943EB980916A0290E08730910508F03F
:10A6500057C0FC01EC57FF4F0D944D088091260D1B
:10A66000811103C084E08093260D8091260D8150D6
:10A670008093260D882309F443C085E080936A0205
:10A680003FC010927B0080E412C02091780030918E
:10A69000790080911C0D90911D0D820F931F909356
:10A6A0001D0D80931C0D2CC010927B0082E48093C2
:10A6B0007C0080917A00806480937A0021C0209190
:10A6C00078003091790080911A0D90911B0D820FC6
:10A6D000931F90931B0D80931A0D12C010927B0054
:10A6E00081E4E5CF209178003091790080911E0DB2
:10A6F00090911F0D820F931F90931F0D80931E0D3D
:10A7000010916A02111182C0809169028F5F80935B
:10A71000690280310CF47AC0109269028091190D9F
:10A7200081111BC080911C0D90911D0D9093160DF1
:10A730008093150D80911E0D90911F0D9093180D13
:10A740008093170D80911A0D90911B0D9093100D11
:10A7500080930F0D81E08093190D8AE0ECE1FDE01C
:10A76000DF011D928A95E9F710921B0D10921A0DC8
:10A77000C091150DD091160DD195C195D10980913B
:10A78000BA0E9091BB0E9195819591098C179D07FA
:10A790000CF44EC080917F0290918002919581953A
:10A7A0009109C817D9070CF453C0C091170DD09167
:10A7B000180DD195C195D1098091BC0E9091BD0E17
:10A7C0009195819591098C179D070CF451C080914A
:10A7D000810290918202919581959109C817D907BC
:10A7E0000CF456C0C0910F0DD091100D2091B80EF1
:10A7F0003091B90E2C173D070CF05AC020917D0204
:10A8000030917E02C217D3070CF062C0812F90E016
:10A81000019667E070E00F943A0880936A02F8941A
:10A8200010922E0D80916E00846080936E0060C047
:10A830008091110D9091120D181619060CF0AACFE7
:10A840004AEA51E168E871E180E00E94E181A2CF2B
:10A850008091110D9091120D181619060CF0A5CFCC
:10A8600047E651E165E471E180E00E94E1819DCF1E
:10A870008091130D9091140D181619060CF0A7CFA6
:10A880004AE951E168E871E181E00E94E1819FCFEE
:10A890002091130D3091140D121613060CF0A2CF57
:10A8A00047E551E165E471E181E00E94E1819ACFE1
:10A8B00020910D0D30910E0D121613060CF09ECF47
:10A8C00047E751E168E871E18FEF0E94E18196CF9F
:10A8D00020910D0D30910E0D121613060CF096CF2F
:10A8E00044E351E165E471E18FEF0E94E1818ECF95
:10A8F000FF91EF91DF91CF91BF91AF919F918F9198
:10A900007F916F915F914F913F912F911F910F9088
:10A910000BBE0F900FBE0F901F9018951F920F92B5
:10A920000FB60F9211240BB60F92BF92CF92DF9207
:10A93000EF92FF920F931F932F933F934F935F9349
:10A940006F937F938F939F93AF93BF93EF93FF93F7
:10A95000CF93DF9300D01F92CDB7DEB780916E000A
:10A960008B7F80936E0080916F008D7F80936F004E
:10A970007894C090090DD0900A0DE0900B0DF090E6
:10A980000C0DC114D104E104F104F1F18091C70E62
:10A990008823D1F10E948AB809EBC0160BE0D006DB
:10A9A000E104F10488F018EBC11A1BE0D10AE108B8
:10A9B000F108C092090DD0920A0DE0920B0DF092B1
:10A9C0000C0D88EB9BE009C0C6011092090D109296
:10A9D0000A0D10920B0D10920C0D9093890080932C
:10A9E00088002091880030918900809184009091A6
:10A9F000850040962817390708F00EC6809184001C
:10AA0000909185004096D7C18091070D9091080DD7
:10AA10000097D1F08C01015011091093080D00939B
:10AA2000070D1092060D1092050D0E94ADC6012B68
:10AA300041F488E291E19093DD078093DC070E9466
:10AA4000BA7E88EC90E0B7C18091050D9091060D1B
:10AA5000892B09F0B5C19091621280916312981709
:10AA600049F1909163124FE4949F900111242E516B
:10AA7000384F8091DE079091DF07A091E007B091F9
:10AA8000E107F901E55BFF4F4081518162817381EC
:10AA9000841B950BA60BB70B8093DE079093DF0703
:10AAA000A093E007B093E107D9018C9188608C9363
:10AAB00069010DC08FB7F8941092DE071092DF077E
:10AAC0001092E0071092E1078FBFC12CD12CD092D9
:10AAD000060DC092050DC114D10409F46AC1F60136
:10AAE00052A18091040D418158130AC0242F30E0F7
:10AAF00080916802992787FD90952817390731F0D2
:10AB00005093040D409368020E940B4A1092000D6E
:10AB10001092010D1092020D1092030DD601D796DE
:10AB20008D919C91D8978134BCE99B0728F48132A0
:10AB3000EEE49E0748F002C080E49CE99695879574
:10AB40009695879524E007C08131F7E29F0730F0A2
:10AB50009695879522E02093FF0C08C021E0209372
:10AB6000FF0C8032910510F480E290E08C010052DD
:10AB70001109011528E01207D0F0812F9927880FBD
:10AB8000991F880F991F885D924FFC01329645915D
:10AB90005491AA27059F9001049F210D3A1F069406
:10ABA0002A1F3A1F1124FC01859194911DC0C801F0
:10ABB000969587958C7F885D964FFC0145915491C1
:10ABC0000296FC0185919491B80167707727869F62
:10ABD0009001879F300D969F300D112463E03695CC
:10ABE00027956A95E1F7CA01821B930B843691057C
:10ABF00088F489E1E82E83E0F82ED7018D917D015C
:10AC0000882319F00E94804BF8CFC8010E94D16EB2
:10AC100084E690E09093FE0C8093FD0C8091FF0CF5
:10AC20008093FC0CF60183AD94AD9093FB0C809364
:10AC3000FA0C8134FCE99F0728F481320EE4900776
:10AC400048F002C080E49CE9969587959695879593
:10AC500024E007C0813117E2910730F0969587957F
:10AC600022E02093FF0C08C021E02093FF0C8032EB
:10AC7000910510F480E290E08C0100521109011559
:10AC800028E01207E0F0812F9927880F991F880F7D
:10AC9000991F885D924FFC01329625913491AA2725
:10ACA000039FA001029F410D5A1F06944A1F5A1F7D
:10ACB0001124FC0125913491241B350B1EC0C801C1
:10ACC000969587958C7F885D964FFC0125913491F0
:10ACD0000296FC0145915491B80167707727469F11
:10ACE000C001479F900D569F900D1124E3E096956B
:10ACF0008795EA95E1F7281B390B2436310588F44E
:10AD000069E1E62E63E0F62ED7018D917D0188235F
:10AD100019F00E94804BF8CFC8010E94D16E24E642
:10AD200030E0C901A0E0B0E08093F60C9093F70CFE
:10AD3000A093F80CB093F90C30938900209388000D
:10AD4000F60182899389A489B589B695A7959795C7
:10AD50008795B095A095909581959F4FAF4FBF4F28
:10AD60008093F20C9093F30CA093F40CB093F50C39
:10AD70008093EE0C9093EF0CA093F00CB093F10C39
:10AD80008093EA0C9093EB0CA093EC0CB093ED0C39
:10AD90008093E60C9093E70CA093E80CB093E90C39
:10ADA0001092E20C1092E30C1092E40C1092E50C5D
:10ADB00007C080ED97E090938900809388002CC4B1
:10ADC0008091C70E81110E948AB82091FF0C222326
:10ADD00009F4ABC1E091050DF091060D8091E60CF0
:10ADE0009091E70CA091E80CB091E90C428153815D
:10ADF00064817581840F951FA61FB71F8093E60C91
:10AE00009093E70CA093E80CB093E90C1816190680
:10AE10001A061B060CF4409AE091050DF091060D00
:10AE20008091EA0C9091EB0CA091EC0CB091ED0CA0
:10AE30004681578160857185840F951FA61FB71FB6
:10AE40008093EA0C9093EB0CA093EC0CB093ED0C78
:10AE5000181619061A061B060CF4419AE091050D06
:10AE6000F091060D8091EE0C9091EF0CA091F00CFA
:10AE7000B091F10C4285538564857585840F951FCB
:10AE8000A61FB71F8093EE0C9093EF0CA093F00CCD
:10AE9000B093F10C181619061A061B060CF4429A08
:10AEA000E091050DF091060D8091F20C9091F30C5C
:10AEB000A091F40CB091F50C468557856089718995
:10AEC000840F951FA61FB71F8093F20C9093F30C6D
:10AED000A093F40CB093F50C181619061A061B066D
:10AEE00034F48181811102C0439A01C0449A809157
:10AEF000E60C9091E70CA091E80CB091E90C1816C3
:10AF000019061A061B0684F5E091050DF091060D51
:10AF10004289538964897589841B950BA60BB70BED
:10AF20008093E60C9093E70CA093E80CB093E90CA7
:10AF3000409164028091D20C9091D30CA091D40CDA
:10AF4000B091D50C552747FD5095652F752F840F6F
:10AF5000951FA61FB71F8093D20C9093D30CA0937C
:10AF6000D40CB093D50C40988091EA0C9091EB0CE6
:10AF7000A091EC0CB091ED0C181619061A061B06E0
:10AF800084F5E091050DF091060D4289538964899D
:10AF90007589841B950BA60BB70B8093EA0C9093D5
:10AFA000EB0CA093EC0CB093ED0C409165028091FA
:10AFB000D60C9091D70CA091D80CB091D90C5527F4
:10AFC00047FD5095652F752F840F951FA61FB71F3E
:10AFD0008093D60C9093D70CA093D80CB093D90C37
:10AFE00041988091EE0C9091EF0CA091F00CB091F3
:10AFF000F10C181619061A061B0684F5E091050DCA
:10B00000F091060D4289538964897589841B950BDB
:10B01000A60BB70B8093EE0C9093EF0CA093F00C63
:10B02000B093F10C409166028091DA0C9091DB0CA8
:10B03000A091DC0CB091DD0C552747FD5095652F94
:10B04000752F840F951FA61FB71F8093DA0C90935E
:10B05000DB0CA093DC0CB093DD0C42988091F20CD9
:10B060009091F30CA091F40CB091F50C1816190600
:10B070001A061B06ACF5E091050DF091060D42890C
:10B08000538964897589841B950BA60BB70B809334
:10B09000F20C9093F30CA093F40CB093F50C409148
:10B0A00067028091DE0C9091DF0CA091E00CB091D2
:10B0B000E10C552747FD5095652F752F840F951F7F
:10B0C000A61FB71F8093DE0C9093DF0CA093E00CBB
:10B0D000B093E10C8181811102C0439801C0449872
:10B0E0008091E20C9091E30CA091E40CB091E50CFE
:10B0F0000196A11DB11D8093E20C9093E30CA093E7
:10B10000E40CB093E50C2150E091050DF091060D93
:10B11000428953896489758984179507A607B707FB
:10B1200008F455CEBB24B39401C0B12C4091E20C7D
:10B130005091E30C6091E40C7091E50CE090050DEA
:10B14000F090060DF70186899789A08DB18D84173F
:10B150009507A607B70708F400C14091F60C509177
:10B16000F70C6091F80C7091F90C068D178D20A1E9
:10B1700031A1AA27419FB12D529FC001629F900D1E
:10B18000619F800D911D429FB00D811D9A1F519F9F
:10B19000B00D811D9A1F609FB00D811D9A1F509F99
:10B1A000B10D8A1F9A1FB6958A1F9A1F349F800D72
:10B1B000911D359F900D112443AD54AD480F591F7B
:10B1C0005093FB0C4093FA0C87A990ADA1ADB2ADA2
:10B1D00060E070E084179507A607B70720F4909306
:10B1E000FB0C8093FA0C8091FA0C9091FB0C81344B
:10B1F000BCE99B0728F48132EEE49E0748F002C0C8
:10B2000080E49CE9969587959695879524E007C0FC
:10B210008131F7E29F0730F09695879522E02093E1
:10B22000FF0C08C021E02093FF0C8032910510F440
:10B2300080E290E08C0100521109011528E012070C
:10B24000E0F0812F9927880F991F880F991F885D3B
:10B25000924FFC01329625913491AA27039FA001B9
:10B26000029F410D5A1F06944A1F5A1F1124FC01C8
:10B2700025913491241B350B1EC0C80196958795E6
:10B280008C7F885D964FFC01259134910296FC01DC
:10B2900045915491B80167707727469FC001479F39
:10B2A000900D569F900D1124B3E096958795BA9511
:10B2B000E1F7281B390B2436310588F4F9E1EF2E2C
:10B2C000F3E0FF2ED7018D917D01882319F00E94B4
:10B2D000804BF8CFC8010E94D16E24E630E0809107
:10B2E000C70E882301F1C901293BBBE03B07E0F011
:10B2F00068EB7BE00F942608883EE3E09E0718F495
:10B300008854944F02C088EB9BE0A901481B590B5D
:10B3100060E070E04093090D50930A0D60930B0DAF
:10B3200070930C0D01C0C90190938900809388002F
:10B330004091F60C5091F70C6091F80C7091F90C5B
:10B34000420F531F611D711D4093F60C5093F70C73
:10B350006093F80C7093F90C42C14091E20C50914B
:10B36000E30C6091E40C7091E50CF701828D938DF4
:10B37000A48DB58D84179507A607B70708F0FFC001
:10B380000091000D1091010D2091020D3091030DDF
:10B3900009831A832B833C83468D578D60A171A14D
:10B3A000AA27059FB12D169F6001269FD00C259FCF
:10B3B000C00CD11C069FB00DC11CDA1E159FB00D2C
:10B3C000C11CDA1E249FB00DC11CDA1E149FB10DE2
:10B3D000CA1EDA1EB695CA1EDA1E709FC00CD11C9A
:10B3E000719FD00C11248091FA0C9091FB0CFF9668
:10B3F000C816D90680F48C199D094081518162815B
:10B4000073818C0120E030E0041715072607370709
:10B4100020F4CA0102C08081918181341CE9910726
:10B4200028F481322EE4920748F002C080E49CE9BF
:10B43000969587959695879524E007C0813137E2E8
:10B44000930730F09695879522E02093FF0C08C073
:10B4500021E02093FF0C8032910510F480E290E00F
:10B460008C0100521109011548E01407E0F0812F0A
:10B470009927880F991F880F991F885D924FFC01AB
:10B48000329625913491AA27039FA001029F410D76
:10B490005A1F06944A1F5A1F1124FC01259134910A
:10B4A000241B350B1EC0C801969587958C7F885D3F
:10B4B000964FFC01259134910296FC0145915491DF
:10B4C000B80167707727469FC001479F900D569F30
:10B4D000900D112443E0969587954A95E1F7281B36
:10B4E000390B2436310588F489E1E82E83E0F82E03
:10B4F000D7018D917D01882319F00E94804BF8CFF0
:10B50000C8010E94D16E24E630E08091C70E8823E6
:10B5100001F1C901293BBBE03B07E0F068EB7BE0B0
:10B520000F942608883EE3E09E0718F48854944F51
:10B5300002C088EB9BE0A901481B590B60E070E05A
:10B540004093090D50930A0D60930B0D70930C0DF1
:10B5500001C0C901909389008093880089819A81F4
:10B56000AB81BC81820F931FA11DB11D8093000D83
:10B570009093010DA093020DB093030D30C0209164
:10B58000FD0C3091FE0C8091C70E882301F1293B00
:10B59000FBE03F07E0F0C90168EB7BE00F94260871
:10B5A000883E03E0900718F48854944F02C088EB5B
:10B5B0009BE0A901481B590B60E070E04093090D26
:10B5C00050930A0D60930B0D70930C0D9C013093FA
:10B5D0008900209388008091FC0C8093FF0C2091BF
:10B5E0008800309189008091840090918500409678
:10B5F0002817390748F4809184009091850040967F
:10B600009093890080938800BB2031F01092060D42
:10B610001092050D0E94ADC6F89480912E0D8823DE
:10B6200021F080916E008B7F03C080916E0084605A
:10B6300080936E0080916F00826080936F000F9006
:10B640000F900F900F90DF91CF91FF91EF91BF91ED
:10B65000AF919F918F917F916F915F914F913F91AA
:10B660002F911F910F91FF90EF90DF90CF90BF909F
:10B670000F900BBE0F900FBE0F901F9018951F924A
:10B680000F920FB60F9211240BB60F922F933F9388
:10B690004F935F936F937F938F939F93AF93BF93DA
:10B6A000EF93FF932091C6009FB7F894E091DA07DB
:10B6B00081E08E0F8F773091DB07831731F0F0E058
:10B6C000E65AF84F20838093DA079FBF30915907DD
:10B6D000832F90E08C30910508F044C0FC01E557C1
:10B6E000FF4F0D944D082D3441F02E34B9F481E014
:10B6F00005C02A3330F02D3481F582E0809359075C
:10B7000046C0203308F043C0203209F440C02D3237
:10B7100021F53DC0213329F0243329F02032E9F40A
:10B7200036C083E0EBCF88E0E9CF203321F021332E
:10B73000A1F486E0E3CF84E0E1CF283371F485E023
:10B74000DDCF223351F487E0D9CF213331F489E0C2
:10B75000D5CF203311F48AE0D1CF8BE0CFCF2A3080
:10B76000B1F413C02A3099F4373049F03A3059F027
:10B77000353059F4109263021092580706C08FE1D9
:10B7800099E00E941C7F0E943C7410925907FF911F
:10B79000EF91BF91AF919F918F917F916F915F9149
:10B7A0004F913F912F910F900BBE0F900FBE0F90B6
:10B7B0001F901895CF93DF938FE794E10E946A8CD6
:10B7C00085E293E1892B51F486E093E10E946A8C33
:10B7D00085EE92E1DF91CF910C946A8CCBE5D4E1B8
:10B7E0006F97CE010E946A8C83E1C532D807C1F7FA
:10B7F000EBCFBF92CF92DF92EF92FF920F931F9306
:10B80000CF93DF937C018B0120E030E0F701E20F62
:10B81000F31FE491EE2319F02F5F3F4FF7CFF801AC
:10B82000CF01801B910B41914111FACFC4E1D0E0CF
:10B83000C81BD1093327C217D3071CF492E0C92EC5
:10B8400002C0CC24C3948091051290E06C2D70E06E
:10B850006F5F7F4F0F943A08B62E86E0D82ED60E33
:10B8600080913812D81650F080913A1290E02D2D28
:10B8700030E02B5031098217930794F5F12C011514
:10B880001105C1F18AE30E94709082E0C8120FC0D6
:10B89000DB0C80913812D81668F120913A1230E012
:10B8A0008D2D90E00B97281739071CF423C0FF203B
:10B8B00009F18C2F880F8C0F880F80933B12D09248
:10B8C0003C1280E20E947090C801DF91CF911F91DD
:10B8D0000F91FF90EF90DF90CF90BF900C94AE90BF
:10B8E00010923B12D0923C12C7010E94A190FF24FB
:10B8F000F394C5CFDF91CF911F910F91FF90EF90FF
:10B90000DF90CF90BF900895CF92DF92EF92FF9299
:10B910001F93CF93DF9300D01F92CDB7DEB78091F6
:10B92000F0119091F111A091F211B091F311B7FFC4
:10B9300008C01092F0111092F1111092F2111092B1
:10B94000F3118091C5119091C611A091C711B091CA
:10B95000C8114091F0115091F1116091F211709164
:10B96000F31184179507A607B70744F48093F011E5
:10B970009093F111A093F211B093F311809194027E
:10B98000882351F16091F0117091F1118091F211C1
:10B990009091F311C090C911D090CA11E090CB11D1
:10B9A000F090CC116C0D7D1D8E1D9F1D0F943301E9
:10B9B00020E030E048EC52E40F94940169837A83EC
:10B9C0008B839C83CE0101960E9401B7BC018091BC
:10B9D000CF119091D0110DDF8091EC111091D11108
:10B9E000811106C01123C1F1809194028823A1F135
:10B9F0006091F0117091F1118091F2119091F31119
:10BA0000C090C911D090CA11E090CB11F090CC1128
:10BA10006C0D7D1D8E1D9F1D0F94330120E030E0C5
:10BA200048EC52E40F9494010F94AB06E091CD11D1
:10BA3000F091CE11309721F06083718382839383DC
:10BA4000112329F0E091D211F091D3111995809131
:10BA5000EC1181110E94BBBC8091EC11882329F06C
:10BA6000E091D211F091D31119950F900F900F9092
:10BA70000F90DF91CF911F91FF90EF90DF90CF90CB
:10BA80000895CF92DF92EF92FF921F93CF93DF93AF
:10BA900000D01F92CDB7DEB78091F0119091F111D7
:10BAA000A091F211B091F311B7FF08C01092F011FC
:10BAB0001092F1111092F2111092F3118091C511B0
:10BAC0009091C611A091C711B091C8114091F01189
:10BAD0005091F1116091F2117091F3118417950753
:10BAE000A607B70744F48093F0119093F111A09347
:10BAF000F211B093F31180919402882351F1609177
:10BB0000F0117091F1118091F2119091F311C090A8
:10BB1000C911D090CA11E090CB11F090CC116C0DEE
:10BB20007D1D8E1D9F1D0F9435012AE037ED43E2E8
:10BB30005CE30F94940169837A838B839C83CE01A9
:10BB400001960E94CBB5BC018091CF119091D0118C
:10BB500050DE8091EC111091D111811106C011239A
:10BB6000B1F180919402882391F16091F01170916C
:10BB7000F1118091F2119091F311C090C911D09000
:10BB8000CA11E090CB11F090CC116C0D7D1D8E1D73
:10BB90009F1D0F9435012AE037ED43E25CE30F94DB
:10BBA0009401E091CD11F091CE11309721F0608396
:10BBB000718382839383112329F0E091D211F09154
:10BBC000D31119958091EC1181110E94BBBC809119
:10BBD000EC11882329F0E091D211F091D31119953D
:10BBE0000F900F900F900F90DF91CF911F91FF90CA
:10BBF000EF90DF90CF900895CF92DF92EF92FF9277
:10BC00001F93CF93DF9300D01F92CDB7DEB7809103
:10BC1000F0119091F111A091F211B091F311B7FFD1
:10BC200008C01092F0111092F1111092F2111092BE
:10BC3000F3118091C5119091C611A091C711B091D7
:10BC4000C8114091F0115091F1116091F211709171
:10BC5000F31184179507A607B70744F48093F011F2
:10BC60009093F111A093F211B093F311809194028B
:10BC7000882351F16091F0117091F1118091F211CE
:10BC80009091F311C090C911D090CA11E090CB11DE
:10BC9000F090CC116C0D7D1D8E1D9F1D0F943501F4
:10BCA0002AE037ED43E25CE30F94940169837A83E1
:10BCB0008B839C83CE0101960E9480B6BC0180914B
:10BCC000CF119091D01195DD8091EC111091D1118F
:10BCD000811106C01123B1F180919402882391F162
:10BCE0006091F0117091F1118091F2119091F31126
:10BCF000C090C911D090CA11E090CB11F090CC1136
:10BD00006C0D7D1D8E1D9F1D0F9435012AE037EDB2
:10BD100043E25CE30F949401E091CD11F091CE11D8
:10BD2000309721F06083718382839383112329F0FC
:10BD3000E091D211F091D31119958091EC118111FC
:10BD40000E94BBBC0F900F900F900F90DF91CF918E
:10BD50001F91FF90EF90DF90CF900895CF92DF92E8
:10BD6000EF92FF921F93CF93DF9300D01F92CDB736
:10BD7000DEB78091F0119091F111A091F211B09184
:10BD8000F311B7FF08C01092F0111092F111109248
:10BD9000F2111092F3118091C5119091C611A091EA
:10BDA000C711B091C8114091F0115091F1116091FB
:10BDB000F2117091F31184179507A607B70744F4A1
:10BDC0008093F0119093F111A093F211B093F311BD
:10BDD00080919402882351F16091F0117091F111DA
:10BDE0008091F2119091F311C090C911D090CA11B5
:10BDF000E090CB11F090CC116C0D7D1D8E1D9F1D20
:10BE00000F94350120E030E048EC52E40F949401A7
:10BE100069837A838B839C83CE0101960E9401B74C
:10BE2000BC018091CF119091D011E3DC8091EC1195
:10BE30001091D111811106C01123B1F180919402AA
:10BE4000882391F16091F0117091F1118091F211BC
:10BE50009091F311C090C911D090CA11E090CB110C
:10BE6000F090CC116C0D7D1D8E1D9F1D0F94350122
:10BE700020E030E048EC52E40F949401E091CD11C1
:10BE8000F091CE11309721F0608371838283938388
:10BE9000112329F0E091D211F091D31119958091DD
:10BEA000EC1181110E94BBBC0F900F900F900F906E
:10BEB000DF91CF911F91FF90EF90DF90CF90089589
:10BEC0000F931F93CF938091F0119091F111A09156
:10BED000F211B091F311B7FF08C01092F011109257
:10BEE000F1111092F2111092F3118091C5119091FD
:10BEF000C611A091C711B091C8114091F011509195
:10BF0000F1116091F2117091F31184179507A60752
:10BF1000B70744F48093F0119093F111A093F211BC
:10BF2000B093F31180919402882309F16091F0118C
:10BF30007091F1118091F2119091F3110091C9115A
:10BF40001091CA112091CB113091CC11600F711F4B
:10BF5000821F931F0F9435010F94A606CB010E94F8
:10BF600054B8BC018091CF119091D01142DC8091E6
:10BF7000EC11C091D111811106C0CC2381F18091C7
:10BF80009402882361F16091F0117091F111809118
:10BF9000F2119091F3110091C9111091CA112091E1
:10BFA000CB113091CC11600F711F821F931F0F9422
:10BFB0003501E091CD11F091CE11309721F06083E1
:10BFC000718382839383CC2329F0E091D211F09185
:10BFD000D31119958091EC1181110E94BBBC809105
:10BFE000EC11CF911F910F9108956ADF882329F0FA
:10BFF000E091D211F091D3111994089561CF8091FD
:10C00000F0119091F111A091F211B091F311B7FFDD
:10C0100008C01092F0111092F1111092F2111092CA
:10C02000F3118091C5119091C611A091C711B091E3
:10C03000C8114091F0115091F1116091F21170917D
:10C04000F31184179507A607B70744F48093F011FE
:10C050009093F111A093F211B093F3118091940297
:10C06000882391F02091C9113091CA118091F0116B
:10C070009091F111820F931F0E9454B8BC018091DE
:10C08000CF119091D011B5DB8091EC114091D1117D
:10C09000811106C0442311F1809194028823F1F0AC
:10C0A0008091C9119091CA112091F0113091F11134
:10C0B000820F931FE091CD11F091CE11309711F0C6
:10C0C00091838083442329F0E091D211F091D31120
:10C0D00019958091EC1181110E94BBBC8091EC11EB
:10C0E00008958DDF882329F0E091D211F091D311CA
:10C0F0001994089584CFCF93DF93C82F8091EC11CA
:10C10000882321F0DF91CF910C94BBBC6091F0119A
:10C110007091F1118091F2119091F31161157105F7
:10C120008105910579F10F9435012091360D3091FB
:10C13000370D4091380D5091390D0F9494019B01AA
:10C14000AC016091E00E7091E10E8091E20E909151
:10C15000E30E0F9462056093E00E7093E10E8093FE
:10C16000E20E9093E30E1092F0111092F1111092E2
:10C17000F2111092F3116C2F83E00E94E8B981E074
:10C180008093940280919402882381F0C13019F049
:10C19000CCE8D6E202C0C2E8D6E280EE9EE00E9481
:10C1A000A3B7BC01CE01DF91CF9123CBDF91CF911B
:10C1B000089581E0A0CF8FEF9ECF3F924F925F9284
:10C1C0006F927F928F929F92AF92BF92CF92DF92A7
:10C1D000EF92FF920F931F93CF93DF9300D000D085
:10C1E000CDB7DEB78C01362E8091EC118823C9F0D3
:10C1F00026960FB6F894DEBF0FBECDBFDF91CF916C
:10C200001F910F91FF90EF90DF90CF90BF90AF9074
:10C210009F908F907F906F905F904F903F900C9485
:10C22000BBBC8091F0119091F111A091F211B091ED
:10C23000F311892B8A2B8B2B09F493C00E94FB519D
:10C24000932DA4E09A02C00111249E838D83FC01EA
:10C25000EC52F14F40805180628073808091510296
:10C2600081110BC020E030E04AE754E4C301B20181
:10C270000F9462056B017C0108C0ED81FE81EE5ACE
:10C28000FD4FC080D180E280F3808091F0119091C9
:10C29000F111A091F211B091F31189839A83AB83CC
:10C2A000BC83BC01CD010F9435012091360D309136
:10C2B000370D4091380D5091390D0F9494019B0129
:10C2C000AC01C301B2010F9462054B015C01AD8169
:10C2D000BE81AC52B14FBE83AD83FD0160837183DB
:10C2E0008283938389819A81AB81BC81B7FF13C01C
:10C2F00020E030E04AE754E4C301B2010F94610545
:10C300006B017C019B01AC01C501B4010F942F01AD
:10C3100087FF18C010C089819A81AB81BC81892BAD
:10C320008A2B8B2B79F0A7019601C501B4010F94DC
:10C33000880718163CF4AD81BE81CD92DD92ED9256
:10C34000FC9213976FEF832D0E94E8B91092F011C1
:10C350001092F1111092F2111092F31181E080937A
:10C36000940280919402882309F4A0C02DEC3CEC47
:10C370004CEC5DE36091360D7091370D8091380D76
:10C380009091390D0F948807E32DFF27E7FDF09575
:10C3900087FD0AC0CF01880F991F880F991F8C5203
:10C3A000914F0E94A3B768C0EE0FFF1FEE0FFF1F53
:10C3B000EC52F14F20E030E04AE754E460817181B3
:10C3C000828193810F9494010F94A6066B017C01E6
:10C3D000611571058105910561F097FF0AC0F09420
:10C3E000E094D094C094C11CD11CE11CF11C8DE2DE
:10C3F00001C080E280939010C701B60128EE33E0BF
:10C4000040E050E00F9426056AE0862E912CA12C86
:10C41000B12CCA01B901A50194010F942605605DF4
:10C42000609391108EE280939210C701B60124E6CA
:10C4300030E040E050E00F942605CA01B901A501A3
:10C4400094010F942605605D60939310C701B601B7
:10C45000A50194010F942605F62ECA01B901A50184
:10C4600094010F942605605D6093941080E38F0D16
:10C470008093951080E990E1BC01C80126960FB623
:10C48000F894DEBF0FBECDBFDF91CF911F910F910A
:10C49000FF90EF90DF90CF90BF90AF909F908F90E4
:10C4A0007F906F905F904F903F90A3C926960FB6F4
:10C4B000F894DEBF0FBECDBFDF91CF911F910F91DA
:10C4C000FF90EF90DF90CF90BF90AF909F908F90B4
:10C4D0007F906F905F904F903F90089562E08BE760
:10C4E00096E26BCE61E084E796E267CE60E08DE68F
:10C4F00096E263CE5F926F927F928F929F92AF92FD
:10C50000BF92CF92DF92EF92FF920F931F93CF9340
:10C51000DF93EC01C62ED42EB22EEC80FD80C70135
:10C520000E94554F182F8C819D810E94584F982E44
:10C53000113011F00FEF01C00FE08C819D810E943E
:10C540004B4F182F8C819D810E94474FA82E8C81C4
:10C550009D810E944F4F20E62B1530F4009721F06B
:10C56000E80EF91E11E610C08C819D810E94524F89
:10C57000E0E4EB1530F4009721F0E80EF91E11E429
:10C5800003C0F1E1EF0EF11CAB1430F4188A1B8AE2
:10C590001C8A198A1A8A99C0A116C0F3A92DB0E085
:10C5A000F70184918F3F21F4FFEFEF1AFF0A3FC09C
:10C5B0001B1135C08C819D810E94554F97012F5FC3
:10C5C0003F4FF701882311F0823091F484918B8BD7
:10C5D000F90124912C8BF7013396E491E88BF70154
:10C5E0003496E491E98BF7013596E491EA8B24C007
:10C5F0009491892F8F7082508A8B92959F70998B1E
:10C60000F9012491822F8F708C8B22952F702B8BA8
:10C61000F7013296E491E295EF70E88B0DC0F701D7
:10C620003296E491E023EE0EF11CEA0EFB1E1A1581
:10C6300009F4ACCF1F5FB4CFE114F10409F445C095
:10C640008C819D810E94584FA82E6B88BC88798868
:10C650007C0C9A899B0D1D2D191B0B2D262D412F0E
:10C66000672DCE010E94A34F882369F1EA0CF11CCB
:10C67000F7E06F0E669466946694512E5B0C5E0133
:10C680002CE1A20EB11C862C912C1515E1F0072D82
:10C6900067018C2D8E19861590F4F60184916A81BC
:10C6A0007B810C8F1D8F1F8E8E8F95014BE3CE01EA
:10C6B0000E94C54FFFEFCF1ADF0A085FEACFE80CF0
:10C6C000F91C1F5FE2CF888901C080E0DF91CF9124
:10C6D0001F910F91FF90EF90DF90CF90BF90AF90A0
:10C6E0009F908F907F906F905F900895CF92DF9290
:10C6F000EF92FF920F931F93CF93DF931F92CDB7CB
:10C70000DEB76C01DC01DC96EC90DC97DB96FC90EC
:10C71000DB978C010C5F1F4F5996ED91FC915A9756
:10C72000C80169831995482F4E0D29816F2DC801C5
:10C73000E1DEF60123AD992787FD9095820F911DCB
:10C7400083AF81E090E00F90DF91CF911F910F9127
:10C75000FF90EF90DF90CF9008950F931F93CF93AA
:10C76000DF93CDB7DEB728970FB6F894DEBF0FBEC4
:10C77000CDBF0091B20610E0F801EE0FFF1FEF5E93
:10C78000F24F60817181882777FD8095982F0F94F3
:10C7900035016D837E838F839887F801EE0FFF1F2D
:10C7A000EE0FFF1FED5AF94F80819181A281B38175
:10C7B00089839A83AB83BC834EEFBE016B5F7F4F4F
:10C7C000CE0101960E9482C960910D0D70910E0DEF
:10C7D000882777FD8095982F0F9435016D837E8390
:10C7E0008F83988780915B0690915C06A0915D068F
:10C7F000B0915E0689839A83AB83BC834FEFBE0101
:10C800006B5F7F4FCE0101960E9482C96091110D2E
:10C810007091120D882777FD8095982F0F94350120
:10C820006D837E838F839887809153069091540601
:10C83000A0915506B091560689839A83AB83BC8339
:10C8400040E0BE016B5F7F4FCE0101960E9482C91E
:10C850006091130D7091140D882777FD8095982FA6
:10C860000F9435016D837E838F839887809157065F
:10C8700090915806A0915906B0915A0689839A83DF
:10C88000AB83BC8341E0BE016B5F7F4FCE0101965D
:10C890000E9482C9E9E6F6E284918F010F5F1F4F83
:10C8A000882321F00E94804BF801F6CFE091B20678
:10C8B000F0E0E45DF24F608170E080E090E00E9483
:10C8C0000270E4E6F6E284918F010F5F1F4F882328
:10C8D00021F00E94804BF801F6CF6091290D70E0A5
:10C8E00080E090E00E94027060E070E081E696E2F5
:10C8F0000E94DF718AE30E94804B60912C0D70E0F2
:10C9000080E090E00E94027061E070E081E696E2D3
:10C910000E94DF718AE30E94804B60912D0D70E0D0
:10C9200080E090E00E94027028960FB6F894DEBF77
:10C930000FBECDBFDF91CF911F910F910895CF9280
:10C94000DF92FF920F931F93CF93DF931F921F925B
:10C95000CDB7DEB7082F162FE0911912F0911A12F9
:10C9600084E092E149835A831995180F4981C42EB6
:10C970005A81D52EF12CD6012D916D01222341F043
:10C98000412F602F84E092E1B5DD080FF80EF3CF60
:10C990008F2D0F900F90DF91CF911F910F91FF90EE
:10C9A000DF90CF9008950F931F930E9478C603E203
:10C9B00014E220E448E060E080E00E94C4C583EB1C
:10C9C0009BE10E9404904DE253E061E18DE3B7DF0B
:10C9D00088E598E10E94049043E353E06CE18EE324
:10C9E000AEDF8BEB91E10E94049042E453E069E2F8
:10C9F0008FE3A5DF8BEB91E10E9404904EE453E0BE
:10CA00006EE38EE39CDF40E553E06EE383E497DF63
:10CA10000E94CA8F8111CBCF1F910F9108958091F1
:10CA2000EC11882321F01092CF060C94BBBCBBCF35
:10CA3000CF93DF931F92CDB7DEB780913D12811166
:10CA400007C081E080933D1284E092E10E94C94FCB
:10CA5000609106127091071219829E012F5F3F4F5D
:10CA60004FE084E092E10E94C54F9DDF0F90DF917F
:10CA7000CF910895DDDFE4E0F1E080818F7D808358
:10CA80009FB7F894E5E0F1E08081806280839FBFEA
:10CA9000E4E0F1E080818F7B80839FB7F894E5E04C
:10CAA000F1E08081806480839FBF6A98729A549875
:10CAB0005C9A82E0809358110E943EB91092521104
:10CAC0000895CF92DF92EF92FF92CF93DF936A01A6
:10CAD0007B01FC018491EF012196882321F00E94C3
:10CAE000804BFE01F7CF4AE0C701B601DF91CF913D
:10CAF000FF90EF90DF90CF900C94916F8F929F9268
:10CB0000AF92BF92CF92DF92EF92FF920F931F935B
:10CB1000CF93DF93CDB7DEB7C155D1090FB6F894E7
:10CB2000DEBF0FBECDBF19AE1AAE1BAE1CAE80E38A
:10CB300090E3A0E3B0E08DAB9EABAFABB8AF259672
:10CB40001FAE1EAE259784E690E029969FAF8EAF6C
:10CB5000299710923A0D9E012D5B3F4F44E050E023
:10CB6000BE016B5C7F4FCE01895B9F4F0E94DBB49F
:10CB700029968EAD9FAD2997029629969FAF8EAFCD
:10CB8000299725961FAE1EAE259782E062968FAF3D
:10CB900062979E012D5B3F4F41E050E0BE016F5A0E
:10CBA0007F4FCE01895B9F4F0E94DBB49E012D5BBE
:10CBB0003F4F44E150E064ED71E1CE01895B9F4F4E
:10CBC0000E94DBB49E012D5B3F4F44E150E062E8E0
:10CBD00076E0CE01895B9F4F0E94DBB49E012D5B06
:10CBE0003F4F44E150E063EF70E1CE01895B9F4F1E
:10CBF0000E94DBB49E012D5B3F4F44E050E06FE0AC
:10CC000071E1CE01895B9F4F0E94DBB49E012D5BD9
:10CC10003F4F44E050E06BE071E1CE01895B9F4FF4
:10CC20000E94DBB49E012D5B3F4F44E050E067E083
:10CC300071E1CE01895B9F4F0E94DBB49E012D5BA9
:10CC40003F4F44E050E06EEA76E0CE01895B9F4FB3
:10CC50000E94DBB49E012D5B3F4F44E050E06AEA46
:10CC600076E0CE01895B9F4F0E94DBB49E012D5B75
:10CC70003F4F44E050E066EA76E0CE01895B9F4F8B
:10CC80000E94DBB49E012D5B3F4F40E150E066E91E
:10CC900076E0CE01895B9F4F0E94DBB49E012D5B45
:10CCA0003F4F4CE050E068EC7EE0CE01895B9F4F47
:10CCB0000E94DBB400E010E0B8016451794F9E019E
:10CCC0002D5B3F4F44E050E0CE01895B9F4F0E94B7
:10CCD000DBB4085F1F4F0831110571F780E090E069
:10CCE000A0E2B1E489AB9AABABABBCAB9E012D5BD0
:10CCF0003F4F44E050E0BE016F5C7F4FCE01895B47
:10CD00009F4F0E94DBB461961FAE619719AE1AAEB9
:10CD10001BAE1CAE83E060968FAF60972F968FAFEF
:10CD20002F979E012D5B3F4F41E050E0BE01605BBD
:10CD30007F4FCE01895B9F4F0E94DBB49E012D5B2C
:10CD40003F4F44E050E0BE01675C7F4FCE01895BFE
:10CD50009F4F0E94DBB49E012D5B3F4F41E050E0AE
:10CD6000BE01615B7F4FCE01895B9F4F0E94DBB4A8
:10CD70009E012D5B3F4F41E050E0BE01625B7F4F63
:10CD8000CE01895B9F4F0E94DBB41AE0115071F015
:10CD90009E012D5B3F4F44E050E0BE01675C7F4F3A
:10CDA000CE01895B9F4F0E94DBB4F0CF1DA61EA66B
:10CDB0001FA618AA9E012D5B3F4F44E050E0BE0124
:10CDC000635D7F4FCE01895B9F4F0E94DBB419AE3C
:10CDD0001AAE1BAE1CAE1AE0115071F09E012D5B15
:10CDE0003F4F44E050E0BE01675C7F4FCE01895B5E
:10CDF0009F4F0E94DBB4F0CF83E02E968FAF2E972B
:10CE00002D968FAF2D9719A61AA61BA61CA61DA29C
:10CE10001EA21FA218A619AE1AAE1BAE1CAE9E0112
:10CE20002D5B3F4F41E050E0BE01635B7F4FCE0181
:10CE3000895B9F4F0E94DBB49E012D5B3F4F41E019
:10CE400050E0BE01645B7F4FCE01895B9F4F0E9423
:10CE5000DBB49E012D5B3F4F44E050E0BE016B5DB3
:10CE60007F4FCE01895B9F4F0E94DBB49E012D5BFB
:10CE70003F4F44E050E0BE01675D7F4FCE01895BCC
:10CE80009F4F0E94DBB40AE010E001501109011528
:10CE9000110571F09E012D5B3F4F44E050E0BE0153
:10CEA000675C7F4FCE01895B9F4F0E94DBB4EDCF63
:10CEB0002C961FAE2C9719AE1AAE1BAE1CAE8FEF80
:10CEC0002B968FAF2B979E012D5B3F4F41E050E09B
:10CED000BE01655B7F4FCE01895B9F4F0E94DBB433
:10CEE0009E012D5B3F4F44E050E0BE01675C7F4FE9
:10CEF000CE01895B9F4F0E94DBB49E012D5B3F4FAB
:10CF000041E050E0BE01665B7F4FCE01895B9F4FE1
:10CF10000E94DBB419AE1AAE1BAE1CAE1DE0115060
:10CF20009E012D5B3F4F44E050E0112349F0BE01CC
:10CF3000675C7F4FCE01895B9F4F0E94DBB4EFCFD0
:10CF400063E47DE0CE01895B9F4F0E94DBB49E01CC
:10CF50002D5B3F4F44E050E06FE37DE0CE01895B05
:10CF60009F4F0E94DBB49E012D5B3F4F44E050E099
:10CF70006BE37DE0CE01895B9F4F0E94DBB4C12C47
:10CF800080E8D82E8BE3E82E85E4F82E812C912CB6
:10CF900090E8A92E9FE3B92E1230B0F59E012D5BCB
:10CFA0003F4F44E050E061E371E1CE01895B9F4F68
:10CFB0000E94DBB49E012D5B3F4F44E050E06DE2E8
:10CFC00071E1CE01895B9F4F0E94DBB49E012D5B16
:10CFD0003F4F44E050E069E271E1CE01895B9F4F31
:10CFE0000E94DBB489AE9AAEABAEBCAE9E012D5BA7
:10CFF0003F4F44E050E0BE01675C7F4FCE01895B4C
:10D000009F4F0E94DBB426C0C9AEDAAEEBAEFCAED9
:10D010009E012D5B3F4F44E050E0BE01675C7F4FB7
:10D02000CE01895B9F4F0E94DBB419AE1AAE1BAED6
:10D030001CAE04E0015071F09E012D5B3F4F44E0B7
:10D0400050E0BE01675C7F4FCE01895B9F4F0E941D
:10D05000DBB4F0CF1F5F153009F09ECF84E190E084
:10D0600023969FAF8EAF23979E012D5B3F4F42E0EB
:10D0700050E0BE016F5B7F4FCE01895B9F4F0E94E6
:10D08000DBB49E012D5B3F4F44E050E06DE371E166
:10D09000CE01895B9F4F0E94DBB49E012D5B3F4F09
:10D0A00044E050E069E371E1CE01895B9F4F0E944B
:10D0B000DBB49E012D5B3F4F44E050E065E371E13E
:10D0C000CE01895B9F4F0E94DBB480E290E0219605
:10D0D0009FAF8EAF21979E012D5B3F4F42E050E006
:10D0E000BE01615C7F4FCE01895B9F4F0E94DBB424
:10D0F0002A961FAE2A9780E090E0A0E4B0E489A3CE
:10D100009AA3ABA3BCA380E090E0A4E3B2E48D8F2C
:10D110009E8FAF8FB8A3198E1A8E1B8E1C8E1D8A00
:10D120001E8A1F8A188E198A1A8A1B8A1C8A80E016
:10D1300090E0A0E5B1E48D879E87AF87B88B198614
:10D140001A861B861C8680E090E0A0E0B1E48D8307
:10D150009E83AF83B8879E012D5B3F4F41E050E037
:10D16000BE01675B7F4FCE01895B9F4F0E94DBB49E
:10D170009E012D5B3F4F44E050E0BE016F5D7F4F4D
:10D18000CE01895B9F4F0E94DBB49E012D5B3F4F18
:10D1900044E050E0BE01635E7F4FCE01895B9F4F4C
:10D1A0000E94DBB49E012D5B3F4F44E050E0BE0186
:10D1B000675E7F4FCE01895B9F4F0E94DBB49E016B
:10D1C0002D5B3F4F44E050E0BE016B5E7F4FCE01D0
:10D1D000895B9F4F0E94DBB49E012D5B3F4F44E073
:10D1E00050E0BE016F5E7F4FCE01895B9F4F0E9472
:10D1F000DBB49E012D5B3F4F44E050E0BE01635F16
:10D200007F4FCE01895B9F4F0E94DBB49E012D5B57
:10D210003F4F44E050E0BE01675F7F4FCE01895B26
:10D220009F4F0E94DBB49E012D5B3F4F44E050E0D6
:10D23000BE016B5F7F4FCE01895B9F4F0E94DBB4C5
:10D240009E012D5B3F4F41E050E061E876E0CE016A
:10D25000895B9F4F0E94DBB409E716E0F12C81E067
:10D260008F1548F0F80180819181A281B38189AF47
:10D270009AAFABAFBCAF9E012D5B3F4F44E050E097
:10D28000BE01675C7F4FCE01895B9F4F0E94DBB47C
:10D29000F3940C5F1F4FF5E0FF12E1CF1EAE1DAE01
:10D2A0001CE0115071F09E012D5B3F4F42E050E0B9
:10D2B000BE01635C7F4FCE01895B9F4F0E94DBB450
:10D2C000F0CF19AE1AAE1BAE1CAE9E012D5B3F4FC8
:10D2D00044E050E0BE01675C7F4FCE01895B9F4F09
:10D2E0000E94DBB49E012D5B3F4F44E050E0BE0145
:10D2F000675C7F4FCE01895B9F4F0E94DBB4198230
:10D300001A821B821C8214E0115071F09E012D5B69
:10D310003F4F44E050E0BE016F5F7F4FCE01895B1D
:10D320009F4F0E94DBB4F0CF80913A0D811154C021
:10D3300029960EAD1FAD299725968EAD9FAD2597E9
:10D3400027969FAF8EAF279784E690E029969FAFF0
:10D350008EAF29979E012D5B3F4F44E050E066E879
:10D3600073E0CE01895B9F4F0E94DBB49E012D5B71
:10D370003F4F42E050E0BE016B5B7F4FCE01895BC7
:10D380009F4F0E94DBB4EBE4FAE384917F019FEFAF
:10D39000E91AF90A882321F00E94804BF701F5CFA2
:10D3A000B801645671098FE599E20E94DF712796F2
:10D3B0004EAD5FAD279760E070E082E599E281DBDA
:10D3C000EFE4F9E284918F010F5F1F4F882321F072
:10D3D0000E94804BF801F6CF90913A0D81E08927A9
:10D3E000CF5ADF4F0FB6F894DEBF0FBECDBFDF912F
:10D3F000CF911F910F91FF90EF90DF90CF90BF9052
:10D40000AF909F908F900895AF92BF92CF92DF928E
:10D41000EF92FF920F931F93CF93DF93C82F882330
:10D4200019F0E7E3F9E20CC0EBE4FAE384918F0131
:10D430000F5F1F4F8823A9F30E94804BF801F6CF9E
:10D4400084918F010F5F1F4F882321F00E94804B32
:10D45000F801F6CFCC2319F0EAE1F9E20CC0EBE4D5
:10D46000FAE384918F010F5F1F4F8823A9F30E9475
:10D47000804BF801F6CF84918F010F5F1F4F8823F7
:10D4800021F00E94804BF801F6CF8AE00E94804B89
:10D49000C1112DC0EBE4FAE384918F010F5F1F4FA0
:10D4A000882321F00E94804BF801F6CFE7E0F9E2F3
:10D4B00084918F010F5F1F4F882321F00E94804BC2
:10D4C000F801F6CF80918106882321F08AE00E943E
:10D4D000804B5AC4ECEFF8E284918F010F5F1F4F2D
:10D4E000882309F451C40E94804BF801F5CF409184
:10D4F000790650917A0660917B0670917C0683EFE5
:10D5000098E22BD68AE00E94804BC1110CC0EBE45C
:10D51000FAE384918F010F5F1F4F882321F00E944F
:10D52000804BF801F6CF40917D0650917E066091C8
:10D530007F067091800687EE98E20FD68AE00E94FF
:10D54000804B8091810681111BC0CC2319F0ECED3A
:10D55000F8E20CC0EBE4FAE384918F010F5F1F4FF8
:10D560008823A9F30E94804BF801F6CF84918F01A4
:10D570000F5F1F4F882321F00E94804BF801F6CFE8
:10D58000C11124C0EBE4FAE384918F010F5F1F4FB8
:10D59000882321F00E94804BF801F6CFEBECF8E2F3
:10D5A00084918F010F5F1F4F882321F00E94804BD1
:10D5B000F801F6CFEBE4FAE384918F010F5F1F4F80
:10D5C000882321F00E94804BF801F6CF4091D411BE
:10D5D0005091D5116091D6117091D71183EC98E2DA
:10D5E000BCD54091D8115091D9116091DA11709148
:10D5F000DB1180EC98E2B1D54091DC115091DD1146
:10D600006091DE117091DF118DEB98E2A6D58AE072
:10D610000E94804BCC2359F160E070E085EB98E2EA
:10D62000CED64091E0115091E1116091E2117091DC
:10D63000E31182EB98E291D58AE00E94804B61E091
:10D6400070E085EB98E2BBD64091E4115091E51172
:10D650006091E6117091E71182EB98E27ED58AE045
:10D660000E94804BC11131C0EBE4FAE30CC0EBE443
:10D67000FAE384918F010F5F1F4F882369F20E94A4
:10D68000804BF801F6CF84918F010F5F1F4F8823E5
:10D6900021F00E94804BF801F6CFE4E9F8E2849192
:10D6A0008F010F5F1F4F882321F00E94804BF801EC
:10D6B000F6CFEBE4FAE384918F010F5F1F4F8823CD
:10D6C00021F00E94804BF801F6CF409182065091E4
:10D6D000830660918406709185068BE898E23DD5BB
:10D6E0004091860650918706609188067091890660
:10D6F00088E898E232D540918A0650918B06609175
:10D700008C0670918D0685E898E227D58AE00E9404
:10D71000804BCC2359F160E070E08CE798E24FD663
:10D7200040918E0650918F066091900670919106FF
:10D7300089E798E212D58AE00E94804B61E070E0B0
:10D740008CE798E23CD64091920650919306609106
:10D7500094067091950689E798E2FFD48AE00E94CA
:10D76000804BC11131C0EBE4FAE30CC0EBE4FAE307
:10D7700084918F010F5F1F4F882369F20E94804BB5
:10D78000F801F6CF84918F010F5F1F4F882321F09E
:10D790000E94804BF801F6CFE7E5F8E284918F0113
:10D7A0000F5F1F4F882321F00E94804BF801F6CFB6
:10D7B000EBE4FAE384918F010F5F1F4F882321F080
:10D7C0000E94804BF801F6CF4091F3105091F41075
:10D7D0006091F5107091F6108EE498E272D9409144
:10D7E000F7105091F8106091F9107091FA108BE4D5
:10D7F00098E267D94091FB105091FC106091FD10A8
:10D800007091FE1088E498E25CD98AE00E94804B17
:10D81000CC2359F160E070E08FE398E2D0D54091DD
:10D82000FF105091001160910111709102118CE371
:10D8300098E247D98AE00E94804B61E070E08FE374
:10D8400098E2BDD5409103115091041160910511EA
:10D85000709106118CE398E234D98AE00E94804BE3
:10D86000C11131C0EBE4FAE30CC0EBE4FAE38491BC
:10D870008F010F5F1F4F882369F20E94804BF801D0
:10D88000F6CF84918F010F5F1F4F882321F00E94F4
:10D89000804BF801F6CFE2EFF7E284918F010F5F42
:10D8A0001F4F882321F00E94804BF801F6CFEBE454
:10D8B000FAE384918F010F5F1F4F882321F00E94AC
:10D8C000804BF801F6CF40910F11509110116091EB
:10D8D00011117091121189EE97E23FD440910B1112
:10D8E00050910C1160910D1170910E1186EE97E21E
:10D8F00034D4409107115091081160910911709131
:10D900000A1183EE97E229D48AE00E94804BC1116C
:10D9100024C0EBE4FAE384918F010F5F1F4F88234B
:10D9200021F00E94804BF801F6CFEFE6F7E28491F8
:10D930008F010F5F1F4F882321F00E94804BF80159
:10D94000F6CFEBE4FAE384918F010F5F1F4F88233A
:10D9500021F00E94804BF801F6CF4091AE06509125
:10D96000AF066091B0067091B10686E697E2F5D3F6
:10D970004091AA065091AB066091AC067091AD063D
:10D9800083E697E2EAD34091A6065091A7066091FC
:10D99000A8067091A90680E697E293D84091960672
:10D9A0005091970660919806709199068DE597E2DF
:10D9B000D4D340919A0650919B0660919C06709139
:10D9C0009D068AE597E2C9D340919E0650919F0635
:10D9D0006091A0067091A10687E597E2BED34091C1
:10D9E000A2065091A3066091A4067091A50684E555
:10D9F00097E2B3D38AE00E94804BC11124C0EBE4CC
:10DA0000FAE384918F010F5F1F4F882321F00E945A
:10DA1000804BF801F6CFE6E4F7E284918F010F5FC7
:10DA20001F4F882321F00E94804BF801F6CFEBE4D2
:10DA3000FAE384918F010F5F1F4F882321F00E942A
:10DA4000804BF801F6CF4091C80E5091C90E6091FD
:10DA5000CA0E7091CB0E8DE397E27FD34091CC0E2E
:10DA60005091CD0E6091CE0E7091CF0E8AE397E269
:10DA700074D34091D00E5091D10E6091D20E70911E
:10DA8000D30E87E397E269D38AE00E94804BCC23D0
:10DA900009F161E070E08DE197E291D44091EC06EC
:10DAA0005091ED066091EE067091EF068AE197E2E3
:10DAB00054D34091F4065091F5066091F6067091AA
:10DAC000F70687E197E249D38AE00E94804BC111B3
:10DAD00026C034C0EBE4FAE384918F010F5F1F4F3F
:10DAE000882321F00E94804BF801F6CFE6E2F7E2AE
:10DAF00084918F010F5F1F4F882321F00E94804B7C
:10DB0000F801F6CFEBE4FAE384918F010F5F1F4F2A
:10DB1000882309F4BECF0E94804BF801F5CF23E49F
:10DB2000A22E2DE0B22E3FE3C32E3DE0D32E4BE3D9
:10DB3000E42E4DE0F42E00E010E024C0EBE4FAE324
:10DB400084918F010F5F1F4F882321F00E94804B2B
:10DB5000F801F6CFEAEFF6E284918F010F5F1F4FD5
:10DB6000882321F00E94804BF801F6CFEBE4FAE322
:10DB700084918F010F5F1F4F882389F20E94804B91
:10DB8000F801F6CFB80181EF96E219D4F501619161
:10DB900071915F018EEE96E212D4F601619171915E
:10DBA0006F018BEE96E20BD4F701619171917F01C9
:10DBB00088EE96E204D48AE00E94804B0F5F1F4FEC
:10DBC00002301105F9F6C11117C0EBE4FAE38491B4
:10DBD000EF012196882321F00E94804BFE01F7CFB0
:10DBE000E9EDF6E28491EF012196882309F444C01F
:10DBF0000E94804BFE01F6CFC0E0D0E0BE0180ED78
:10DC000096E2DDD340913111509132116091331180
:10DC1000709134118DEC96E2A0D22CEA35EC47E2FB
:10DC20005EE360912D1170912E1180912F119091D2
:10DC300030110F943E06AB01BC018AEC96E271D222
:10DC40002CEA35EC47E25EE36091291170912A11CC
:10DC500080912B1190912C110F949401AB01BC0178
:10DC600087EC96E25ED28AE00E94804B2196C23019
:10DC7000D10509F0C3CF4AC0EBE4FAE38491EF0188
:10DC80002196882321F00E94804BFE01F7CF40911E
:10DC900031115091321160913311709134118EEB2A
:10DCA00096E25BD22CEA35EC47E25EE360912D11FF
:10DCB00070912E1180912F11909130110F943E068A
:10DCC000AB01BC018BEB96E22CD22CEA35EC47E29F
:10DCD0005EE36091291170912A1180912B1190912E
:10DCE0002C110F949401AB01BC0188EB96E219D280
:10DCF0008AE00E94804BEBE4FAE38491EF012196E5
:10DD0000882321F00E94804BFE01F7CF40913D1106
:10DD100050913E1160913F11709140118FEA96E24F
:10DD20001CD22CEA35EC47E25EE360913911709128
:10DD30003A1180913B1190913C110F943E06AB013A
:10DD4000BC018CEA96E2EDD12CEA35EC47E25EE3C9
:10DD50006091351170913611809137119091381181
:10DD60000F949401AB01BC0189EA96E2DAD18AE012
:10DD7000DF91CF911F910F91FF90EF90DF90CF90A7
:10DD8000BF90AF900C94804BEBE4FAE384918F0149
:10DD90000F5F1F4F882309F4AACB0E94804BF80124
:10DDA000F5CFBC0180E090E04AE0BBD08DE00E945E
:10DDB000804B8AE00C94804B1F93CF93DF93182FF6
:10DDC000EBE4FAE38491EF012196882321F00E948D
:10DDD000804BFE01F7CF84E50E94804B612F70E0FD
:10DDE00080E090E04AE09DD080E20E94804BC1E755
:10DDF000D3E08991882319F00E94804BFACF8AE002
:10DE0000DF91CF911F910C94804BFF920F931F9342
:10DE1000CF93DF93EC0184E50E94CF4D882349F135
:10DE20000E94BE4BF82E81E08F1504F5EBE4FAE377
:10DE300084918F010F5F1F4F882321F00E94804B38
:10DE4000F801F6CF8DE40E94804BBE0180E090E0A7
:10DE50004AE067D06F2D772767FD709586E996E2D7
:10DE6000AED28AE00E94804B81E008C0F092B206F8
:10DE700004C0809100078093B20680E0DF91CF91CB
:10DE80001F910F91FF900895CF93DF93C1E1DDE0E3
:10DE90001982188280E00E941E511092140D109277
:10DEA000130D81E00E941E5110920E0D10920D0D67
:10DEB0000E94D5500E9487971982188280E00E94A4
:10DEC0001E5110922C0D9FB7F894E2E0F1E0808192
:10DED0008F7B80839FBF1092140D1092130D81E0F1
:10DEE0000E941E5110922D0D9FB7F894E2E0F1E0D0
:10DEF00080818F7E80839FBF10920E0D10920D0D3A
:10DF00001092290D7598DF91CF9108951092EF101E
:10DF10001092EE101092F1101092F010B5DF0C94E8
:10DF2000B5BCAF92BF92CF92DF92EF92FF920F9368
:10DF30001F93CF93DF93CDB7DEB7A0970FB6F894BA
:10DF4000DEBF0FBECDBF6115710581059105B1F131
:10DF5000B12CC42ED12CE12CF12CAA24A394AB0C0F
:10DF600001E010E00C0F1D1F0B0D111DB7FC1A95E1
:10DF7000A70196010F940405F8016083B901CA0155
:10DF8000611571058105910511F41B2D12C0BA2C84
:10DF9000E4CFE1E0F0E0EC0FFD1FE10FF11D17FD14
:10DFA000FA9580818A3040F490E3890F0E94804B7B
:10DFB00011501F3F71F715C097E3F7CF80E3A0968C
:10DFC0000FB6F894DEBF0FBECDBFDF91CF911F918A
:10DFD0000F91FF90EF90DF90CF90BF90AF900C9497
:10DFE000804BA0960FB6F894DEBF0FBECDBFDF9179
:10DFF000CF911F910F91FF90EF90DF90CF90BF9046
:10E00000AF900895CF92DF92EF92FF926B017C0167
:10E0100097FF0BC08DE20E94804BF094E094D09467
:10E02000C094C11CD11CE11CF11C4AE0C701B6011F
:10E03000FF90EF90DF90CF9074CF8F929F92AF922E
:10E04000BF92CF92DF92EF92FF92CF936B017C0150
:10E05000B42E20E030E0A9010F942F0187FF07C004
:10E060008DE20E94804BF7FAF094F7F8F094C0E04C
:10E0700060E070E080E09FE3CB1541F02DEC3CECDC
:10E080004CEC5DE30F949401CF5FF6CF9B01AC01A4
:10E09000C701B6010F9462056B017C010F94AB06BA
:10E0A0004B015C014AE03DDFCC2389F1C501B4019D
:10E0B0000F9433019B01AC01C701B6010F946105B8
:10E0C0006B017C018EE20E94804B20E030E040E258
:10E0D00051E4C701B6010F9494016B017C010F94C8
:10E0E000A6064B01AA2497FCA094BA2CC501B40142
:10E0F00089DFC501B4010F9435019B01AC01C70153
:10E10000B6010F9461056B017C01C150F1F6CF910E
:10E11000FF90EF90DF90CF90BF90AF909F908F9047
:10E120000895CF92DF92EF92FF92CF93DF936A012F
:10E130007B01FC018491EF012196882321F00E944C
:10E14000804BFE01F7CF42E0C701B601DF91CF91CE
:10E15000FF90EF90DF90CF9070CFCF92DF92EF9251
:10E16000FF92CF93DF936A017B01FC018491EF0161
:10E170002196882321F00E94804BFE01F7CF42E0D8
:10E18000C701B601DF91CF91FF90EF90DF90CF9064
:10E1900054CFCF93DF9385E40E94CF4D811110C0FF
:10E1A00080E50E94A14D882391F00E94DE4B609390
:10E1B000311170933211809333119093341107C051
:10E1C0000E94BE4B823060F3E4E1FAE36AC089E466
:10E1D0000E94A14D882381F00E94DE4B2CEA35EC91
:10E1E00047E25EE30F94940160932D1170932E111A
:10E1F00080932F119093301184E40E94A14D8823C5
:10E2000081F00E94DE4B2CEA35EC47E25EE30F948E
:10E210003E066093291170932A1180932B119093DD
:10E220002C11EBE4FAE38491EF012196882321F08D
:10E230000E94804BFE01F7CF409131115091321175
:10E24000609133117091341183EE99E286DF2CEAEC
:10E2500035EC47E25EE360912D1170912E118091B3
:10E260002F11909130110F943E06AB01BC018FED40
:10E2700099E257DF2CEA35EC47E25EE36091291121
:10E2800070912A1180912B1190912C110F9494016F
:10E29000AB01BC018BED99E244DF10C00E94804BC2
:10E2A000FE018491EF0121968111F8CFC1E7D3E0FF
:10E2B0008991882319F00E94804BFACF8AE0DF9180
:10E2C000CF910C94804BCF93DF9380E50E94A14DBA
:10E2D000882351F00E94DE4B60933D1170933E11F4
:10E2E00080933F119093401189E40E94A14D8823AF
:10E2F00081F00E94DE4B2CEA35EC47E25EE30F949E
:10E3000094016093391170933A1180933B1190936B
:10E310003C1184E40E94A14D882381F00E94DE4BD1
:10E320002CEA35EC47E25EE30F943E06609335112C
:10E33000709336118093371190933811EBE4FAE320
:10E340008491EF012196882321F00E94804BFE01E9
:10E35000F7CF40913D1150913E1160913F11709166
:10E36000401187ED99E2F9DE2CEA35EC47E25EE3F5
:10E370006091391170913A1180913B1190913C114B
:10E380000F943E06AB01BC0183ED99E2CADE2CEA94
:10E3900035EC47E25EE36091351170913611809162
:10E3A0003711909138110F949401AB01BC018FEC9F
:10E3B00099E2B7DE8AE0DF91CF910C94804B0F9306
:10E3C0001F93CF93DF938B01FC018491EF01219682
:10E3D000882321F00E94804BFE01F7CFB8018827E7
:10E3E00077FD8095982FDF91CF911F910F910ACEE5
:10E3F000CF93DF9383E50E94A14DC82F882371F04E
:10E400000E94DE4B0F94A6067093890260938802E7
:10E4100021E0672B09F020E02093DB1080E50E94CB
:10E42000A14D882369F08091880290918902892BFF
:10E4300019F00E94CF4B01C081E08093DB102CC00B
:10E44000C1112AC0EBE4FAE38491EF0121968823FD
:10E4500021F00E94804BFE01F7CF8091DB108823D2
:10E4600019F066EF72E002C062E873E08CEB99E2AB
:10E470000E9483B560918802709189028BEA99E2CB
:10E480009EDFE7EAF9E28491EF012196882321F0EB
:10E490000E94804BFE01F7CFDF91CF910895CF937B
:10E4A000DF930E94FB51E0918A10F0E0EC51F14FB4
:10E4B0008081882309F458C0EBE9F9E28491EF01E7
:10E4C0002196882321F00E94804BFE01F7CFC09156
:10E4D0008A1080E6C89FE0011124C65FD04F888172
:10E4E0008E3419F0E8E9F9E210C080E20E94804B16
:10E4F00089910E94804B899190ED980F9A30C8F3D2
:10E500008D32B9F38B32A9F3EDCF8491EF012196CF
:10E51000882321F00E94804BFE01F7CF0E94404FDC
:10E520006FE070E0681B7109882777FD8095982F50
:10E5300069DDE5E9F9E28491EF012196882321F074
:10E540000E94804BFE01F7CF80918B1064E070E059
:10E55000681B7109882777FD8095982F53DD8AE025
:10E56000DF91CF910C94804BDF91CF910895CF93A1
:10E57000DF938FB7F8949091DB079093DA078FBF02
:10E58000EEE9F9E28491EF012196882321F00E94BF
:10E59000804BFE01F7CF60914A0670914B06809147
:10E5A0004C0690914D066F5F7F4F8F4F9F4F2ADD36
:10E5B0008AE00E94804BDF91CF9171CFEF92FF9262
:10E5C0000F931F93CF93DF931F92CDB7DEB7082F22
:10E5D000162FE4E1FAE384917F012FEFE21AF20AA9
:10E5E000882331F099830E94804BF7019981F3CF02
:10E5F000E02FF92F84917F019FEFE91AF90A882310
:10E6000021F00E94804BF701F5CF60914A0670918E
:10E610004B0680914C0690914D06F4DC8AE00E94F6
:10E62000804B1111A4DF1092C1111092C0110F90F4
:10E63000DF91CF911F910F91FF90EF900895CF93AD
:10E64000DF93E7E8F9E28491EF012196882321F036
:10E650000E94804BFE01F7CFE3E8F9E28491EF01DD
:10E660002196882321F00E94804BFE01F7CF62B3F0
:10E670006695617070E080E090E0C4DC62B3617028
:10E6800070E080E090E0BEDC8AE00E94804BEFE723
:10E69000F9E28491EF012196882321F00E94804BBA
:10E6A000FE01F7CF60910601772767FD7095872FF0
:10E6B000972F662797FD6395772788279927A2DCF0
:10E6C00062B362FB662760F970E080E090E09ADC5C
:10E6D0008AE00E94804BEBE7F9E28491EF012196FA
:10E6E000882321F00E94804BFE01F7CF6091060144
:10E6F00066FB662760F970E080E090E083DC609163
:10E70000060165FB662760F970E080E090E07ADC46
:10E710008AE00E94804BE6E7F9E28491EF012196BE
:10E72000882321F00E94804BFE01F7CF6091060103
:10E7300063FB662760F970E080E090E063DC609145
:10E7400006016295617070E080E090E05BDC8AE039
:10E750000E94804BE1E7F9E28491EF012196882342
:10E7600021F00E94804BFE01F7CF60910601669573
:10E77000617070E080E090E045DC6091060162FB32
:10E78000662760F970E080E090E03CDC8AE0DF9191
:10E79000CF910C94804B1F93CF93DF9383E50E941E
:10E7A000A14D811104C0CFE0D3E010E00EC0C0E065
:10E7B0000E94BE4B682F8C2F0E94B449CF5FC5309A
:10E7C000B9F7F1CF1F5F143061F089910E94A14D1C
:10E7D0008823C1F30E94BE4B682F812F0E94B44949
:10E7E000F1CF82E40E94A14D882331F00E94BE4BFC
:10E7F000682F84E00E94B449DF91CF911F911FCF11
:10E8000080910007813011F40C942FF12091E411D4
:10E810003091E5114091E6115091E71160E070E010
:10E8200080E89FE30F943E066093F90E7093FA0E12
:10E830008093FB0E9093FC0E089580910007811148
:10E8400002C00C942FF12091E0113091E111409120
:10E85000E2115091E31160E070E080E89FE30F94D3
:10E860003E066093F50E7093F60E8093F70E90932C
:10E87000F80E08950C942FF188E893E19093080D19
:10E880008093070D80916F008D7F80936F00909132
:10E89000621280916312981719F00E94ADC6F7CFEB
:10E8A0001092060D1092050D80916F00826080938A
:10E8B0006F008FB7F8941092DE071092DF07109266
:10E8C000E0071092E1078FBF0E9447F080E00E94AE
:10E8D000EE496093480D7093490D80934A0D9093D3
:10E8E0004B0D81E00E94EE4960934C0D70934D0DED
:10E8F00080934E0D90934F0D82E00E94EE496093FD
:10E90000500D7093510D8093520D9093530D8CE0E8
:10E91000E8E4FDE0A4EDBEE001900D928A95E1F7F8
:10E920000C94F6F20E94218A8091540D80938A10F3
:10E9300010928B10A1DF0E948797A6DA1092EF1039
:10E940001092EE101092F1101092F01010926302DB
:10E950006FEF88EC9AE20E9493B90C94B5BCFF92D9
:10E960000F931F93CF93DF931092F4118091F011C6
:10E970009091F111A091F211B091F3118130904872
:10E98000A105B10540F01092F0111092F111109212
:10E99000F2111092F311C091F0114091550D14161F
:10E9A000D4F4842F992787FD909501972C2F332736
:10E9B00027FD30952817390774F0CFEFC40F8C2F3F
:10E9C00090E0A0E0B0E08093F0119093F111A0935B
:10E9D000F211B093F3111092EE118091ED11C8175E
:10E9E00014F4C093ED118091ED11992787FD909556
:10E9F00004962C2F332727FD30958217930724F494
:10EA00008CEF8C0F8093ED11D091ED1100E0D111BE
:10EA10001BC08091EC11811105C080919402882364
:10EA200099F009C0C111F9CF0E94BBBC8091EE11D1
:10EA3000882399F3B3C181E0C11180E024E040E76D
:10EA40005BE2602F0E94E0BE0E94404F811182C1B4
:10EA50008091911281117EC180919212882321F0C0
:10EA600080918614811176C1D130E9F48091EC1146
:10EA7000811106C080919402882309F452C00BC012
:10EA8000C130C1F78FEE90EC0E9480BC8091EE11F6
:10EA9000882381F383C181E0C13009F080E023E065
:10EAA00042E65BE23BC0D230E1F48091EC1181118F
:10EAB00005C0809194028823A1F10BC0C230C9F730
:10EAC00083EB93ED0E9480BC8091EE11882389F343
:10EAD00065C181E0C23009F080E023E046E55BE2F9
:10EAE0001DC0D330F1F48091EC11811105C08091EB
:10EAF00094028823B1F00BC0C330C9F788EF9BE7BD
:10EB00000E9480BC8091EE11882389F347C181E087
:10EB1000C33009F080E023E048E45BE2602F0E940C
:10EB2000E0BEF12C14E080E00E941A4F81111EC05B
:10EB3000D1131BC08091EC11811105C0809194020A
:10EB4000882399F009C0CD13F9CF0E9482BD80912E
:10EB5000EE11882399F322C181E0CD1380E020E2F9
:10EB600045E35BE2602F0E94E0BE1F5F81E00E94F0
:10EB70001A4F81111EC0D1131BC08091EC1181115D
:10EB800005C080919402882399F009C0CD13F9CF74
:10EB90000E9480BD8091EE11882399F3FFC081E02F
:10EBA000CD1380E020E242E25BE2602F0E94E0BEF3
:10EBB0001F5F80919212882309F482C0809186148D
:10EBC000882309F45EC0809191128823D9F0D11373
:10EBD00036C08091EC11811105C080919402882388
:10EBE00071F109C0CD13F9CF0E9484BD8091EE115F
:10EBF000882399F3D3C081E0CD1380E020E246E181
:10EC00005BE21AC0D1131BC08091EC11811105C0C9
:10EC100080919402882399F009C0CD13F9CF0E9406
:10EC2000DEBC8091EE11882399F3B8C081E0CD134A
:10EC300080E020E249E05BE2602F0E94E0BE1F5FBF
:10EC4000D1131AC08091EC11811105C080919402FA
:10EC5000882391F008C0CD13F9CF64DE8091EE11C6
:10EC60008823A1F39BC081E0CD1380E020E24EEF2A
:10EC70005AE2602F0E94E0BE1F5FFF2009F442C0ED
:10EC800061C0F1105FC0D1133CC08091EC118111C3
:10EC900005C0809194028823A1F10BC0CD13F9CF58
:10ECA0008FE19FEB0E9480BC8091EE11882389F355
:10ECB00075C081E0CD1380E023E040EF5AE21EC032
:10ECC000F11040C0D1131DC08091EC11811105C01D
:10ECD000809194028823A9F00BC0CD13F9CF8FE166
:10ECE0009FEB0E9480BC8091EE11882389F356C06F
:10ECF00081E0CD1380E023E045EE5AE2602F0E94D0
:10ED0000E0BE1F5FD1131DC08091EC11811105C0C1
:10ED1000809194028823A9F00BC0CD13F9CF8FE026
:10ED200095E60E9480BC8091EE11882389F336C05D
:10ED300081E0CD1380E023E046ED5AE2602F0E948F
:10ED4000E0BE1F5F0F5FDF5F053009F060CE1093FC
:10ED5000550D24C0D130F1F48091EC11811105C022
:10ED6000809194028823B1F00BC0C130C9F78FECB9
:10ED700091ED0E9480BC8091EE11882389F30EC032
:10ED800081E0C13009F080E023E04BE65BE2602FD8
:10ED90000E94E0BEFF24F39412E0C5CEDF91CF9134
:10EDA0001F910F91FF9008952F923F924F925F9283
:10EDB0006F927F928F929F92AF92BF92CF92DF928B
:10EDC000EF92FF920F931F93CF93DF93CDB7DEB7F0
:10EDD000CE55D1090FB6F894DEBF0FBECDBF2DB70B
:10EDE0003EB76D963FAF2EAF6D9763961FAE1EAECA
:10EDF000639784E690E061969FAF8EAF61979E0126
:10EE00002F5A3F4F44E050E0BE016B5B7F4FCE0175
:10EE1000815B9F4F0E9447B59E012F5A3F4F42E0B2
:10EE200050E0BE01635B7F4FCE01815B9F4F0E942C
:10EE300047B543E050E0BE016B5B7F4F86E893E04F
:10EE40000F94A508892B09F43AC026968FAD269712
:10EE5000863539F08FE326968FAF269727961FAE1B
:10EE60002797EBE4FAE384918F010F5F1F4F88230C
:10EE700021F00E94804BF801F6CFE0E6FAE284919F
:10EE80008F010F5F1F4F882321F00E94804BF801F4
:10EE9000F6CFBE016B5B7F4F87E59AE20E9483B598
:10EEA000E9E4FAE284918F010F5F1F4F882321F07C
:10EEB0000E94804BF801F6CF0E9468F16CC46DB6D9
:10EEC0007EB625961CAE1DAE1EAE1FAE2597639670
:10EED0001FAE1EAE63979E012F5A3F4F41E050E098
:10EEE000BE01675A7F4FCE01815B9F4F0E9447B59D
:10EEF00084E1E5EAF2E09E012F5F3F4F7901D901FD
:10EF000001900D928A95E1F780E1E9EBF2E0DE01F4
:10EF1000959601900D928A95E1F780E1E9ECF2E097
:10EF2000DE01559601900D928A95E1F76A96CFAC75
:10EF30006A97D12C33E0C30ED11CCC0CDD1CCC0C59
:10EF4000DD1C8DB79EB78C199D090FB6F8949EBF36
:10EF50000FBE8DBFEDB7FEB731964F012DB73EB74F
:10EF60002C193D090FB6F8943EBF0FBE2DBF8DB7CB
:10EF70009EB701965C01EDB7FEB7EC19FD090FB61F
:10EF8000F894FEBF0FBEEDBF0DB71EB70F5F1F4F4A
:10EF90009E012F5A3F4FA601B401CE01815B9F4FC6
:10EFA0000E9447B59E012F5A3F4FA601B501CE01E1
:10EFB000815B9F4F0E9447B59E012F5A3F4FA6018C
:10EFC000B801CE01815B9F4F0E9447B56A964FAD55
:10EFD0006A9750E04E5F5F4F23EF30E16F963FAF8F
:10EFE0002EAF6F97B2E8CB2EB6E0DB2E64ED71E169
:10EFF00020E030E080E090E0D7014817590714F096
:10F00000740101C07D01E20EF31EF7012080318002
:10F0100042805380FB012192319241925192BF0173
:10F02000481759074CF07501E20EF31EF7012080D6
:10F0300031804280538012C0843011F07C0103C0C3
:10F04000F3E0EF2EF12CEE0CFF1CEE0CFF1CEA0E91
:10F05000FB1EF70124A035A046A057A0F60121927F
:10F060003192419251926F01481759074CF0780143
:10F07000E20EF31EF701208031804280538012C0DF
:10F08000843011F07C0103C0F3E0EF2EF12CEE0C84
:10F09000FF1CEE0CFF1CEA0EFB1EF70124883588CE
:10F0A000468857886F96EEADFFAD6F9721923192EB
:10F0B000419251926F96FFAFEEAF6F9701962C5F22
:10F0C0003F4F8530910509F098CF9E012F5A3F4F51
:10F0D00044E050E06FE071E1CE01815B9F4F0E9400
:10F0E00047B59E012F5A3F4F44E050E06BE071E17D
:10F0F000CE01815B9F4F0E9447B59E012F5A3F4F23
:10F1000044E050E067E071E1CE01815B9F4F0E94D7
:10F1100047B59E012F5A3F4F44E050E06EEA76E03B
:10F12000CE01815B9F4F0E9447B59E012F5A3F4FF2
:10F1300044E050E06AEA76E0CE01815B9F4F0E9496
:10F1400047B59E012F5A3F4F44E050E066EA76E013
:10F15000CE01815B9F4F0E9447B59E012F5A3F4FC2
:10F1600040E150E066E976E0CE01815B9F4F0E946E
:10F1700047B59E012F5A3F4F4CE050E068EC7EE0CF
:10F18000CE01815B9F4F0E9447B500E010E0B801BF
:10F190006451794F9E012F5A3F4F44E050E0CE0119
:10F1A000815B9F4F0E9447B5085F1F4F08311105D3
:10F1B00071F79E012F5A3F4F44E050E0BE016F5B54
:10F1C0007F4FCE01815B9F4F0E9447B59E012F5A12
:10F1D0003F4F41E050E0BE01685A7F4FCE01815B56
:10F1E0009F4F0E9447B59E012F5A3F4F44E050E089
:10F1F000BE016F5B7F4FCE01815B9F4F0E9447B581
:10F200009E012F5A3F4F41E050E0BE01695A7F4FA7
:10F21000CE01815B9F4F0E9447B59E012F5A3F4F01
:10F2200041E050E0BE016A5A7F4FCE01815B9F4FA3
:10F230000E9447B56896EFAC689767968FAD679761
:10F24000E89E7001112400E010E09E012F5A3F4F0C
:10F2500044E050E0BE010E151F0551F06F5B7F4F7B
:10F26000CE01815B9F4F0E9447B50F5F1F4FEDCFCF
:10F27000635C7F4FCE01815B9F4F0E9447B51AE0D0
:10F2800011509E012F5A3F4F112359F044E050E096
:10F29000BE016F5B7F4FCE01815B9F4F0E9447B5E0
:10F2A000EFCF41E050E0BE016B5A7F4FCE01815B52
:10F2B0009F4F0E9447B59E012F5A3F4F41E050E0BB
:10F2C000BE016C5A7F4FCE01815B9F4F0E9447B5B4
:10F2D0009E012F5A3F4F44E050E0BE01675C7F4FD4
:10F2E000CE01815B9F4F0E9447B59E012F5A3F4F31
:10F2F00044E050E0BE016B5C7F4FCE01815B9F4FCD
:10F300000E9447B56696EFAC669765968FAD659798
:10F31000E89E7001112400E010E09E012F5A3F4F3B
:10F320000E151F0569F044E050E0BE016F5B7F4F92
:10F33000CE01815B9F4F0E9447B50F5F1F4FEDCFFE
:10F3400041E050E0BE01665A7F4FCE01815B9F4F86
:10F350000E9447B59E012F5A3F4F44E050E0BE0146
:10F360006F5B7F4FCE01815B9F4F0E9447B59E012F
:10F370002F5A3F4F41E050E0BE016D5A7F4FCE0102
:10F38000815B9F4F0E9447B525961CAE1DAE1EAEF9
:10F390001FAE25971DE011509E012F5A3F4F44E0AC
:10F3A00050E0112349F0BE016F5B7F4FCE01815BBE
:10F3B0009F4F0E9447B5EFCF63E47DE0CE01815BB4
:10F3C0009F4F0E9447B59E012F5A3F4F44E050E0A7
:10F3D0006FE37DE0CE01815B9F4F0E9447B59E01A8
:10F3E0002F5A3F4F44E050E06BE37DE0CE01815B5C
:10F3F0009F4F0E9447B59E012F5A3F4F44E050E077
:10F40000BE016F5B7F4FCE01815B9F4F0E9447B56E
:10F41000123010F004E03EC02596CCACDDACEEAC72
:10F42000FFAC259720E030E84BE355E4C701B60177
:10F430000F942F01882371F3C0923111D0923211B1
:10F44000E0923311F09234119E012F5A3F4F44E065
:10F4500050E06DE271E1CE01815B9F4F0E9447B5A4
:10F460009E012F5A3F4F44E050E069E271E1CE0126
:10F47000815B9F4F0E9447B59E012F5A3F4F44E04A
:10F4800050E0BE016F5B7F4FCE01815B9F4F0E94BA
:10F4900047B510C0015071F09E012F5A3F4F44E014
:10F4A00050E0BE016F5B7F4FCE01815B9F4F0E949A
:10F4B00047B5F0CF1F5F153009F09DCF9E012F5A41
:10F4C0003F4F42E050E0BE01655B7F4FCE01815B64
:10F4D0009F4F0E9447B59E012F5A3F4F44E050E096
:10F4E000BE016F5B7F4FCE01815B9F4F0E9447B58E
:10F4F0002596CCACDDACEEACFFAC259720E030E837
:10F500004BE355E4C701B6010F942F01882301F1A5
:10F51000C0923D11D0923E11E0923F11F092401105
:10F520009E012F5A3F4F44E050E069E371E1CE0164
:10F53000815B9F4F0E9447B59E012F5A3F4F44E089
:10F5400050E065E371E1CE01815B9F4F0E9447B5BA
:10F550009E012F5A3F4F42E050E0BE01675B7F4F54
:10F56000CE01815B9F4F0E9447B59E012F5A3F4FAE
:10F5700041E050E0BE01665A7F4FCE01815B9F4F54
:10F580000E9447B519E011509E012F5A3F4F112399
:10F5900059F044E050E0BE016F5B7F4FCE01815BCC
:10F5A0009F4F0E9447B5EFCF41E050E061E876E021
:10F5B000CE01815B9F4F0E9447B509E716E0F12C11
:10F5C0009E012F5A3F4F44E050E0BE016F5B7F4FDA
:10F5D000CE01815B9F4F0E9447B5F1E0FF1558F0C7
:10F5E00025968CAD9DADAEADBFAD2597F80180835E
:10F5F0009183A283B383F3940C5F1F4FF5E0FF1256
:10F60000DFCF1BE09E012F5A3F4F42E050E0BE018A
:10F61000675C7F4FCE01815B9F4F0E9447B51150C1
:10F6200089F79E012F5A3F4F44E050E0BE016F5BC7
:10F630007F4FCE01815B9F4F0E9447B59E012F5A9D
:10F640003F4F44E050E0BE016F5B7F4FCE01815BD6
:10F650009F4F0E9447B514E0115071F09E012F5A40
:10F660003F4F44E050E0BE016B5C7F4FCE01815BB9
:10F670009F4F0E9447B5F0CF63962EAD3FAD639785
:10F680002F968EAD9FAD2F972817390709F03AC0F6
:10F690000E945AF1EBE4FAE384918F010F5F1F4F50
:10F6A000811103C006E813E004C00E94804BF801FA
:10F6B000F3CFF80181918F01882319F00E94804BCC
:10F6C000F8CF61966EAD7FAD6197645671098CE29B
:10F6D0009AE20E94DF7163964EAD5FAD639760E082
:10F6E00070E08FE19AE20E946165ECE1FAE28491B8
:10F6F0008F010F5F1F4F882309F448C00E94804B81
:10F70000F801F5CFE4E1FAE384918F010F5F1F4F19
:10F71000882321F00E94804BF801F6CFECEFF9E24C
:10F7200084918F010F5F1F4F882321F00E94804B2F
:10F73000F801F6CF2F966EAD7FAD2F9780E090E069
:10F740004AE00E94916FE7EFF9E284918F010F5F29
:10F750001F4F882321F00E94804BF801F6CF63965B
:10F760006EAD7FAD639780E090E04AE00E94916FBC
:10F77000E7EEF9E284918F010F5F1F4F882321F09C
:10F780000E94804BF801F6CF0E9468F10FB6F89402
:10F790007EBE0FBE6DBE80E00E94046A90913A0D5D
:10F7A00081E089276D962EAD3FAD6D970FB6F89429
:10F7B0003EBF0FBE2DBFC25ADF4F0FB6F894DEBF5B
:10F7C0000FBECDBFDF91CF911F910F91FF90EF90B2
:10F7D000DF90CF90BF90AF909F908F907F906F9071
:10F7E0005F904F903F902F900895DEDA0C947685CD
:10F7F000FF920F931F93CF93DF931092F411809198
:10F80000F0119091F111A091F211B091F3118130AA
:10F810009048A105B10540F01092F0111092F1113D
:10F820001092F2111092F3111091F0114091470DC6
:10F830001416D4F4842F992787FD90950197212FD2
:10F84000332727FD30952817390774F01FEF140F61
:10F85000812F90E0A0E0B0E08093F0119093F1113F
:10F86000A093F211B093F3111092EE118091ED116B
:10F87000181714F41093ED118091ED11992787FD5D
:10F8800090950496212F332727FD309582179307F3
:10F8900024F48CEF810F8093ED11F090ED1100E0D6
:10F8A000CAE8DAE2F1101AC08091EC11811106C0A9
:10F8B00080919402882309F48DC009C01111F8CFFA
:10F8C0000E94BBBC8091EE11882391F38AC081E035
:10F8D000111180E024E043EC5AE279C081E0F81293
:10F8E0001DC08091EC11811106C080919402882383
:10F8F00009F470C00BC01130C1F78BE29FED0E947C
:10F9000080BC8091EE11882381F36BC081E01130BF
:10F9100009F080E023E041EB5AE259C022E0F21204
:10F920001BC08091EC11811106C080919402882344
:10F9300009F450C009C01230C1F70E94B58580910A
:10F94000EE11882391F34DC081E0123009F080E080
:10F9500020E242EA5AE23BC083E0F81219C08091EB
:10F96000EC11811105C080919402882399F108C09F
:10F970001330C9F73ADF8091EE118823A1F331C02B
:10F9800081E0133009F080E020E244E95AE21FC030
:10F9900024E0F2121FC08091EC11811105C080910A
:10F9A00094028823B9F00CC01430C9F7D093DD0756
:10F9B000C093DC07DFD18091EE11882381F311C061
:10F9C00081E0143009F080E020E249E75AE2602F3C
:10F9D0000E94E0BE0F5FF394053009F063CF0093FF
:10F9E000470DDF91CF911F910F91FF900895CF9216
:10F9F000DF92FF920F931F93CF93DF931F921F927B
:10FA0000CDB7DEB76901DB0112960D911C911397FA
:10FA1000423309F471C0B8F4453109F47AC0473172
:10FA200009F48BC0443109F0A1C0D80115962C917E
:10FA300015971696ED91FC911797CF01820F911DA6
:10FA4000820F911D5EC0463409F487C0473409F423
:10FA500088C04B3309F08AC0F901818193819130CC
:10FA600029F0933031F4282F885004C028E0280F63
:10FA700001C0282F31E0D80113964C91481708F4A3
:10FA800030E051E0F8014281241708F450E041E0F1
:10FA9000281708F040E0832F842B85233423832B01
:10FAA00009F464C0D6011296FC90913039F070F0E0
:10FAB000923039F0933041F020E001C021E030E095
:10FAC00007C020E03FEF04C02FEFF9CF20E031E086
:10FAD000F7FE08C0B601C8012A8339830E94614F2E
:10FAE00039812A81F6018081830F80838181820F91
:10FAF0008183FF0C69F73AC0B901C8010E94614FC8
:10FB000035C01192E817F907E1F7C8010E948D4F3F
:10FB10002DC0C8010E94774F882351F1F80125813B
:10FB20000680F781E02DCF01820F911D820F911D7C
:10FB30001192E817F907E1F719C0D9011C92F801F1
:10FB4000828111968C9311978581815012968C93A6
:10FB50001297838113968C9309C0D80115968C91C6
:10FB600003C0D80111968C91F601808381E001C019
:10FB700080E00F900F90DF91CF911F910F91FF9038
:10FB8000DF90CF9008956F927F928F929F92AF9265
:10FB9000BF92CF92DF92EF92FF920F931F93CF937A
:10FBA000DF935C017B01942E69018AE0481709F418
:10FBB00071C0A5E14A134AC0DB011296ED91FC9198
:10FBC00013978280C681D781A49A0E94944F80EEB9
:10FBD000782E780C90E1692E680C88EF0E94EC4337
:10FBE0000E94944FBFE1B81508F443C0882D807778
:10FBF00080680E94EC43882D8295807F0E94EC43B0
:10FC00000E94944F80E80E94EC4380E00E94EC4305
:10FC10000E94944F8AEF0E94EC430E94944F8E0101
:10FC2000005F1F4F8881807F0E94EC4389918295FD
:10FC3000807F0E94EC430C171D07A1F7E8010E948A
:10FC4000944F839473948610C8CFA4989601492D3D
:10FC5000B701C501DF91CF911F910F91FF90EF90F8
:10FC6000DF90CF90BF90AF909F908F907F906F90DC
:10FC7000BECE872D807780680E94EC43872D8295C9
:10FC8000807F0E94EC430E94944F80E80E94EC43E6
:10FC900080E8BCCF9C9AA4989B9AA3988091040179
:10FCA0008460809304019FB7F8948091050184607B
:10FCB000809305019FBFA49A0E94944F88E790E02B
:10FCC0000E94994F88EF0E94EC430E94944F80E07D
:10FCD0000E94EC4380E80E94EC430E94944F80E035
:10FCE0000E94EC4380E10E94EC430E94944F8FE01D
:10FCF00090E00E94994F80E30E94EC4380EE0E94C6
:10FD0000EC430E94944FD0E08D2F807780680E9452
:10FD1000EC438D2F8295807F0E94EC430E94944F8C
:10FD200080E80E94EC4380E00E94EC430E94944FE4
:10FD30008AEF0E94EC430E94944FC0E280E00E9450
:10FD4000EC4380E00E94EC430E94944FC150B1F715
:10FD500088EF0E94EC430E94944FDF5FD032A1F6FF
:10FD600080E00E94EC4380EC0E94EC430E94944FA0
:10FD7000A4986CCFDF92EF92FF920F931F93CF93D3
:10FD8000DF93CDB7DEB76E970FB6F894DEBF0FBE28
:10FD9000CDBF6091DC077091DD076115710511F130
:10FDA0004DE150E08E010F5F1F4FC8010F94A0007E
:10FDB0001E8EF8017F01E01AF10AD190DD2019F0C2
:10FDC0008AE0D812F7CFF801EE0DFF1D108260E037
:10FDD000C8010E94854D882329F0C8010E94ABB557
:10FDE000811109C081E02091DC073091DD07232BD0
:10FDF000A9F480E013C0DD2051F08FEFE81AF80A73
:10FE00008091DC079091DD078E0D9F1D02C080E080
:10FE100090E09093DD078093DC07E4CF6E960FB6F9
:10FE2000F894DEBF0FBECDBFDF91CF911F910F9130
:10FE3000FF90EF90DF900895EC01E4E1FAE3849104
:10FE40008F010F5F1F4F882321F00E94804BF80124
:10FE5000F6CFE8E9FBE284918F010F5F1F4F882303
:10FE600021F00E94804BF801F6CF0E94446F0E945F
:10FE7000124C0E943A6561E0CE010E9493B90E9443
:10FE8000B5BC0E9478C684E00E945890809105120B
:10FE90008695869510923B1280933C120E940F919A
:10FEA0008091051286958695880F10923B1280935B
:10FEB0003C1289E89BE20E94A190809105128695F0
:10FEC0008695982F990F980F10923B1290933C12A1
:10FED0008CE79BE20E94A1900E94CA8F8111D3CF30
:10FEE0002FEF8BE49DE1215080409040E1F700C06E
:10FEF0000000F8942FEF84E39CE021508040904074
:10FF0000E1F700C000000E94446FA895FECF6F92F9
:10FF10007F928F929F92AF92BF92DF92EF92FF9269
:10FF20000F931F93CF93DF93CDB7DEB7AD970FB687
:10FF3000F894DEBF0FBECDBF7C01D62E8091921209
:10FF4000882309F4F7C180918614882309F49DC0A1
:10FF5000442309F4C4C180919E14882321F1E4E173
:10FF6000FAE384918F010F5F1F4F882321F00E94D5
:10FF7000804BF801F6CFEDE2FDE284918F010F5F37
:10FF80001F4F882321F00E94804BF801F6CF61E0DB
:10FF900070E080E090E00E9402708AE00E94804B56
:10FFA00084E29DE249DF8FE28093A314B12C21E02B
:10FFB00004EA14E13FE1A32E80915B14B816B8F473
:10FFC000AB9CC0011124B801875D9C4E2DA70E94F7
:10FFD0002FC6C8012DA58C010196F801308133236D
:10FFE00021F02D3810F42F5FF6CFB394E5CF27FD25
:10FFF00006C0B80183E894E10E942FC602C0F80150
:020000021000EC
:100000001082EBE4FAE384918F010F5F1F4F882386
:1000100021F00E94804BF801F6CFB7018BE09DE202
:100020000E9483B560919E14FDE86F9FB00111247A
:100030006D557B4E80E09DE20E9483B54091341562
:100040005091351560913615709137158AEF9CE205
:100050000E9461658AE00E94804B80919E1494E02A
:10006000899FF0011124E156FB4E409134155091C7
:100070003515609136157091371540835183628331
:1000800073838F5F80939E140DC010929E1422E0A4
:10009000B22E27C1B7018DEE9CE20E9483B58AE0A3
:1000A0000E94804B0E94218A1D8218861C821B821E
:1000B00087E093E09A83898385EE92E1909305131C
:1000C00080930413F70180818F3209F06DC087019E
:1000D0000F5F1F4FCE0101963C010115110509F478
:1000E00069C06FE270E0C8010F9493085C0100974B
:1000F00009F461C00817190708F05DC04C01801AA7
:10010000910AA401B801CE0180960F94B308E0E2F1
:10011000F0E0EC0FFD1FE80DF91D10828E01005E6E
:100120001F4FF80181918F01882319F00E94804BA5
:10013000F8CF8AE00E94804B609104137091051300
:100140006115710519F06C5F7F4F02C060E070E0CF
:1001500021E0AE01405E5F4FCE0105960E94758B97
:1001600081111AC0E9EDFCE284918F010F5F1F4FEE
:10017000811104C08E01005E1F4F04C00E94804B9D
:10018000F801F2CFF80181918F01882319F00E94C4
:10019000804BF8CF8EE28CC07092051360920413EE
:1001A00085010F5F1F4F99CF86E093E19093051370
:1001B0008093041387016091041370910513DD206F
:1001C00009F45DC06115710519F06C5F7F4F02C0C5
:1001D00060E070E021E0A80183E894E10E94758B63
:1001E000882309F448C08091941490919514A091AB
:1001F0009614B09197148093301590933115A09375
:100200003215B0933315B8018BEC9CE20E9483B594
:100210004091301550913115609132157091331520
:1002200083EC9CE20E9461658AE00E94804B109200
:100230003415109235151092361510923715E4EBDF
:10024000FCE284917F019FEFE91AF90A882321F0EB
:100250000E94804BF701F5CFB80180E090E00E944A
:100260002F8E8091A112811102C0C80102C081EAC3
:1002700092E160E02DC0B80180EA9CE213C06115F4
:10028000710519F06C5F7F4F02C060E070E026E5F9
:10029000A80183E894E10E94758B81110CC0B8011C
:1002A0008CE89CE20E9483B58EE20E94804B8AE03B
:1002B0000E94804B0FC081E080938F12B7018AE7C4
:1002C0009CE20E9483B58AE00E94804B60E0C801F6
:1002D0000E942EB9CE0101960E946A8C2BC0BB24CD
:1002E000B394EBE4FAE384918F010F5F1F4F8823EF
:1002F00021F00E94804BF801F6CFE5EFFCE28491FB
:100300008F010F5F1F4F882321F00E94804BF8015F
:10031000F6CFE1E0BE1203C000E913E002C00AE834
:1003200013E0F80181918F01882309F4B3CE0E9474
:10033000804BF7CFAD960FB6F894DEBF0FBECDBFA2
:10034000DF91CF911F910F91FF90EF90DF90BF90C1
:10035000AF909F908F907F906F90089560E0809114
:10036000150D9091160D0E941548609353067093D9
:100370005406809355069093560661E08091170DC0
:100380009091180D0E941548609357067093580677
:100390008093590690935A0680910F0D9091100DFD
:1003A0000E94B24460935B0670935C0680935D0686
:1003B00090935E06A8958FB7F8941092190D8FBF91
:1003C0000895CF92DF92FF920F931F93CF93DF9305
:1003D0001F921F92CDB7DEB7F82E6A01809162029C
:1003E000882309F441C0E4E1FAE384918F010F5FAF
:1003F0001F4F882341F069837A830E94804BF80164
:1004000069817A81F2CFFB0184918F010F5F1F4FC9
:10041000882321F00E94804BF801F6CFEDEBFBE240
:1004200084918F010F5F1F4F882321F00E94804B22
:10043000F801F6CFF7FC0CC06F2D772767FD70959C
:10044000872F972F0E9402708AE00E94804B0CC079
:10045000E8EBFBE284918F010F5F1F4F882321F0AF
:100460000E94804BF801F6CF8091560E811107C093
:100470001092620281E08093560EC601DDDC0F907F
:100480000F90DF91CF911F910F91FF90DF90CF9050
:100490000C94446F2F923F924F925F926F927F9293
:1004A0008F929F92AF92BF92CF92DF92EF92FF9284
:1004B0000F931F93CF93DF9300D01F92CDB7DEB77A
:1004C0004C011B0129833A834B835C83270138014C
:1004D000D7FE12C080918E10882309F4A7C0F401C2
:1004E000108210925F0E1092600E1092610E1092A8
:1004F000620E02E010E015C0F601E852F94F80816B
:10050000882309F4BEC0F4011082F601EE0FFF1F2C
:10051000EE0FFF1FE95AF14F1082118212821382EF
:100520008601F40180818230E1F0833009F455C006
:10053000813009F0A8C0F801EE0FFF1FEE0FFF1F7A
:10054000E95AF14F208131814281538169817A8159
:100550008B819C810F942F0187FD95C082E0F4016F
:100560008083000F111F000F111F095A114FB50191
:10057000882777FD8095982F0F9435019B01AC015A
:10058000F80160817181828193810F9461059B01E3
:10059000AC0169817A818B819C810F94880787FDEA
:1005A0000CC00E94C9506856754C8F4F9F4FF10187
:1005B000608371838283938366C00E94C950F10176
:1005C0000081118122813381601B710B820B930B9F
:1005D00097FD59C083E0F4018083FFEFCF16DF065B
:1005E00031F0C114D10431F442E15CE205C04BEDBD
:1005F0005BE202C04FEF5BE26FEE7BE28C2D0F906F
:100600000F900F900F90DF91CF911F910F91FF905E
:10061000EF90DF90CF90BF90AF909F908F907F90A2
:100620006F905F904F903F902F90CBCE02E010E004
:100630007801EE0CFF1CEE0CFF1CC701895A914F8C
:100640007C01A3019201FC0160817181828193810F
:100650000F942F01882309F464CFF701408251825F
:1006600062827382FF24F39420E030E0A901C30189
:10067000B2010F94880718160CF0F12CF401F082E7
:1006800050CF8601D5CF0F900F900F900F90DF9134
:10069000CF911F910F91FF90EF90DF90CF90BF907F
:1006A000AF909F908F907F906F905F904F903F9012
:1006B0002F9008958F3F29F0811106C047E651E140
:1006C00005C044E351E102C047E551E165E471E151
:1006D00078CE8F3F29F0811106C04AEA51E105C06A
:1006E00047E751E102C04AE951E168E871E169CEAA
:1006F0002F923F924F925F926F927F928F929F9232
:10070000AF92BF92CF92DF92EF92FF920F931F931F
:10071000CF93DF93CDB7DEB728970FB6F894DEBF3F
:100720000FBECDBF8091190D811119C028960FB64B
:10073000F894DEBF0FBECDBFDF91CF911F910F9117
:10074000FF90EF90DF90CF90BF90AF909F908F90F1
:100750007F906F905F904F903F902F900895FEDDB7
:100760000E94C9506B837C838D839E83312C22240D
:10077000239480917B0290917C02181619060CF04C
:100780002BC1019790937C0280937B02232D30E054
:1007900038872F834901880C991C880C991CF40117
:1007A000ED5AF94F4080518062807380EF81F88567
:1007B000E852F94F8081811116C0D401A053B94F7E
:1007C000CD90DD90ED90FC90C114D104E104F104D2
:1007D00051F02B813C814D815E812C193D094E09E0
:1007E0005F0957FF20824F815885440F551F5A8358
:1007F0004983FA01EF5EF24F60817181882777FDAE
:100800008095982F0F9435010EE1A02EB12CCF804A
:10081000D8847B018C01A3019201B4016458714F0B
:10082000C6018658914F36DEF401ED5AF94F4080EB
:10083000518062807380E981FA81E254F14F6081D6
:100840007181882777FD8095982F0F9435019B0142
:10085000AC01C301B2010F9488071816A4F4E98112
:10086000FA81ED57FD4F60817181882777FD809572
:10087000982F0F9435019B01AC01C301B2010F9475
:100880002F0187FDE2C060E0EF81F885E45DF24F63
:100890006083F401EE58F14F80819181A281B38190
:1008A0000097A105B10551F12B813C814D815E81FD
:1008B000281B390B4A0B5B0B57FD20C0832D0E9470
:1008C0000A482B013C01E981FA81E259F14F60812C
:1008D000718180E090E00F9433019B01AC01C30172
:1008E000B2010F942F0187FFC3C0332009F4C7C0A2
:1008F00046E55CE267E47CE2832D63DD832D33947F
:10090000813009F036CF80916A0E90916B0EA091E4
:100910006C0EB0916D0E0097A105B10521F12B81F0
:100920003C814D815E81281B390B4A0B5B0B57FDC7
:100930001AC00E9401482B013C016091680E709121
:10094000690E80E090E00F9433019B01AC01C3017C
:10095000B2010F942F0187FF8FC045E25CE268E38C
:100960007CE28FEF2EDD60910D0D70910E0D8827CA
:1009700077FD8095982F0F94350120915B0630917B
:100980005C0640915D0650915E06FAE0AF2EB12CF8
:10099000CC24CA94DC2C7B018C0163E67EE087E6E4
:1009A0009EE078DD80918E1081115FC040905B06E3
:1009B00050905C0660905D0670905E0620E030E02E
:1009C00040EA50E4C301B2010F94880787FF2CC0AE
:1009D00060E06093290DAACE432D50E058874F83E5
:1009E0004A01880C991C880C991C84010D5A194FD6
:1009F000D8014D905D906D907C9020E030E848E902
:100A000053E4C301B2010F948807181634F120E0B3
:100A100030E040EA50E4C301B2010F942F0187FF98
:100A2000C5CE80E047DEBBCE20E030E046E153E4B7
:100A3000C301B2010F942F01181654F20E945245BF
:100A40000F94A60675956795C4CF832D0E948F4697
:100A50000F94A6067595679517CF80E03ADEF801EA
:100A60004080518062807380D2CF1092290D5ECE7B
:100A7000832D0E941E5142CF0E94D55074CF48E66C
:100A80005CE238CF0F931F93CF93DF93EC018B0180
:100A90006091701240917112641306C084E692E175
:100AA0000E94D8C325DEF4CF28813981F8018081E6
:100AB000918150916F1274E0579FF0011124E85911
:100AC000FD4E33872287958784876F5F609370120E
:100AD00081E0850F841719F080936F1202C0109285
:100AE0006F12DF91CF911F910F9108950F931F9374
:100AF000CF93DF93CDB7DEB728970FB6F894DEBF5C
:100B00000FBECDBF8823C1F083E992E098878F8321
:100B100004E610E01A830983BE01695F7F4FCE01AE
:100B20000196B0DF8AEB92E09E838D831A8309835E
:100B3000BE016B5F7F4F0BC088EB91E09C838B8382
:100B400084E190E09A838983BE016D5F7F4FCE017F
:100B5000019698DF28960FB6F894DEBF0FBECDBF82
:100B6000DF91CF911F910F9108950E947E65BECFB6
:100B7000AF92BF92CF92DF92FF920F931F93CF93CA
:100B8000DF9300D01F92CDB7DEB7F82E662351F069
:100B90001092880E1092840E1092850E1092860E7E
:100BA0001092870E0E94C9500091840E1091850EFC
:100BB0002091860E3091870E5B016C01A01AB10A5C
:100BC000C20AD30AD7FC3DC0F7FE05C004EC19E009
:100BD00020E030E015C0E091880E2F2D332727FD4F
:100BE00030952C5F3F4F4E2F552747FD50952417CA
:100BF00035073CF1EF1554F300E911E020E030E057
:100C0000DC01CB01800F911FA21FB31F8093840EC4
:100C10009093850EA093860EB093870E80ED97E09B
:100C20009C838B838CE291E09A838983BE016D5F04
:100C30007F4FCE01019626DF8091880E8F5F8093D3
:100C4000880E0F900F900F900F90DF91CF911F9112
:100C50000F91FF90DF90CF90BF90AF900895CF920B
:100C6000DF92EF92FF926B017C0183E3C816D104FF
:100C7000E104F10468F082E3C81AD108E108F10840
:100C800062E370E080E090E00E942E5031DDEDCF15
:100C9000C701B6010E942E50FF90EF90DF90CF90D9
:100CA00027CDCF93DF93EC018B81813099F489813B
:100CB00081FF10C049895A896B897C89452B462B55
:100CC000472B61F140E050E0BA01CE010E945195FE
:100CD000811102C080E023C04D895E896F89788DC3
:100CE000898D9A8D0E9430978823A1F31D8A1E8AD0
:100CF0001F8A188E198A1A8A1B8A1C8A8981806821
:100D00008983CE010E942DC4882321F340E050E066
:100D1000BA01CE01DF91CF910C94519581E0DF9122
:100D2000CF9108956F927F928F929F92AF92BF92D0
:100D3000CF92DF92EF92FF920F931F93CF93DF93A7
:100D40001F92CDB7DEB78C015B014A01722EDB0129
:100D500059968D919C915A97F801928F818F40E01E
:100D600050E0BA01C5010E945195E12CF501808542
:100D70009185A285B38541895289638974898417D5
:100D80009507A607B70708F0CEC025E0B695A7954A
:100D9000979587952A95D1F7F82FFF70FF2ED501EB
:100DA00013968C91823008F49CC141E050E0BE0162
:100DB0006F5F7F4FC5010E94D793019719F4898116
:100DC00090E002C08FEF9FEF019609F48AC1F50110
:100DD00080859185A285B3854F96A11DB11D808721
:100DE0009187A287B387F0E2FF9EB0011124665B72
:100DF0007B4F6115710509F474C1DB018C91882367
:100E000011F0853EB9F4E1100EC080918C0E9091E6
:100E10008D0EA0918E0EB0918F0EF801848795876C
:100E2000A687B787F08ADB018C91EE24E3948111C9
:100E30009DCF79C04BE050E0C4010F945F08892B2F
:100E400009F094CF77FC4DC120E2F29EF00111240D
:100E5000E65BFB4F8385817121F0872D827109F05C
:100E60005EC040918C0E50918D0E60918E0E7091EF
:100E70008F0ED8011C964D935D936D937C931F97B5
:100E80005096FC924489558960E070E0BA0155277C
:100E90004427828D938DA0E0B0E0482B592B6A2B1C
:100EA0007B2BD80155964D935D936D937C9358970A
:100EB0008385887159F4848D958DA68DB78DF80141
:100EC000818B928BA38BB48B81E010C0803139F57C
:100ED00098012F5E3F4FD80159968D919C915A975A
:100EE0000E94EA958823D9F084E0F8018383872D56
:100EF0008F70D80111968C931197F8011482158286
:100F00001682178218961D921D921D921C921B9795
:100F100074FEDAC0C801C5DE8111D6C0E3C0D801B5
:100F200013961C92DEC0872D8274823409F0D9C0DA
:100F3000EE20E1F0D8015096FC9050971C966D91F0
:100F40007D918D919C911F9741E00E94C8918823CB
:100F500009F4C7C0F8018089F0E28F9FC001112415
:100F6000865B9B4F009709F08FC0BBC0D5011396DD
:100F70008C911397823009F4B4C051968D919D9154
:100F80000D90BC91A02D803E9F4FAF41B10508F060
:100F9000A8C0C5010E946BC4882309F4A2C00E94A6
:100FA0008A91882309F49DC0D5015996ED91FC9151
:100FB0005A971496CD90DD90ED90FC901797B2E083
:100FC000CB1AD108E108F108058404C0CC0CDD1C63
:100FD000EE1CFF1C0A94D2F786859785A089B189FB
:100FE000C80ED91EEA1EFB1E81E080938B0EC092B4
:100FF0008C0ED0928D0EE0928E0EF0928F0E80E0CD
:1010000092E0EAE4F4E0DF019C011D9221503040BF
:10101000E1F766246394D5015996ED91FC915A97B6
:101020008481681698F42AE434E0B701A601460DDD
:10103000511D611D711D8091890E90918A0E0E9433
:101040001E91882309F44DC06394E5CF40E052E03F
:1010500060E070E0058404C0440F551F661F771FD1
:101060000A94D2F751968D919D910D90BC91A02D2F
:10107000840F951FA61FB71FF501818B928BA38B41
:10108000B48B8AE494E0F12C20E2DC011D922A95D5
:10109000E9F72BE0F401DC0101900D922A95E1F7CC
:1010A00021E238E2FC01318B208B40E058E0578789
:1010B0004687338B228B318F208F578B468B0E9434
:1010C0008A918111C1CE0DC075FE09C0F801418918
:1010D000528963897489C8010E94519503C081E0D7
:1010E00001C080E00F90DF91CF911F910F91FF9091
:1010F000EF90DF90CF90BF90AF909F908F907F90B8
:101100006F9008952F923F924F925F926F927F92CD
:101110008F929F92AF92BF92CF92DF92EF92FF9207
:101120000F931F93CF93DF9300D01F921F92CDB7E1
:10113000DEB78C015B014D83252EDC0113968C916B
:1011400013978130C9F411968C9181FF15C082FFED
:1011500019C0F80141895289638974898085918514
:10116000A285B38584179507A607B70759F0C8016C
:101170000E945195811106C081E0F80180838FEFB4
:101180009FEF2DC1ED80F22C7FC0D8015996ED91D3
:10119000FC915A9734803A94DB01CA0139E0B69544
:1011A000A795979587953A95D1F738224A01B1E0EE
:1011B0009B22332009F474C080E092E088199909D9
:1011C00067018E159F0508F46C01D8015996ED91C1
:1011D000FC915A9714964D905D906D907C90179766
:1011E000B2E04B1A510861087108058404C0440C30
:1011F000551C661C771C0A94D2F786859785A089B2
:10120000B189480E591E6A1E7B1E430C511C611C7D
:10121000711CC114E2E0DE0609F08BC080918C0ED7
:1012200090918D0EA0918E0EB0918F0E8415950524
:10123000A605B70569F410928B0E8FEF9FEFDC01C6
:1012400080938C0E90938D0EA0938E0EB0938F0E84
:101250009501B301A2018091890E90918A0EEED77B
:10126000882309F489CFF80180859185A285B3850B
:101270008C0D9D1DA11DB11D80879187A287B3870D
:10128000AC0CBD1CEC18FD08D80118964D915D9171
:101290006D917C911B97E114F10409F076CF7EC02B
:1012A0008114910409F088CFD80114964D915D9175
:1012B0006D917C911797411551056105710559F4A0
:1012C00055968D919D910D90BC91A02D0097A105F3
:1012D000B10549F522C09E012F5F3F4FCF010E940B
:1012E0005893882309F448CF89819A81AB81BC81C6
:1012F000F801218D328DF9012789203139F4883F99
:10130000FFEF9F07A105B10540F40DC0883F2FEF07
:101310009207A2072FE0B20730F0C8010E946BC409
:1013200081114ACF29CFF80184839583A683B7839F
:1013300043CF8114910411F5D80118964D915D9118
:101340006D917C911B9751968D919D910D90BC91C3
:10135000A02D481759076A077B0780F0DBD7882341
:1013600009F40ACF81E080938B0E40928C0E50924C
:101370008D0E60928E0E70928F0E08C041E0C301F8
:10138000B2010E94C891882309F4F6CEA601B501E6
:10139000C401865B9B4F0F946C0865CF51968D916D
:1013A0009D910D90BC91A02D84179507A607B707B6
:1013B00040F4F801418B528B638B748B8181806880
:1013C0008183D80111968C9183FD03C08D81922D6C
:1013D00006C0C8010E942DC48111F8CFCDCE0F9058
:1013E0000F900F900F900F90DF91CF911F910F9161
:1013F000FF90EF90DF90CF90BF90AF909F908F9035
:101400007F906F905F904F903F902F900895CF9373
:10141000DF931F92CDB7DEB7698341E050E0BE0194
:101420006F5F7F4F04966EDE0F90DF91CF9108952E
:10143000CF93DF93EC010E942DC41B82DF91CF91EB
:1014400008951092911280918614882319F083E8F0
:1014500094E1EECF0895CF92DF92EF92FF921F9327
:10146000CF93DF93109292128091EC12882319F09F
:1014700089EE92E1DDDF1092601410925D1485E335
:1014800080935C140E94C950EB01A89580915C1474
:101490009ED48CE594E10E94C5502398229A219A0B
:1014A000209A289A85E080935E1482E58CBD1DBC4D
:1014B0001AE08FEF0E94744B1150D9F720E030E012
:1014C000A90160E08CE594E10E948B51182F809374
:1014D0005F14813049F00E94C9506C1B7D0B613D47
:1014E000774060F381E054C02AEA31E040E050E008
:1014F00068E08CE594E10E948B5182FF03C0109359
:1015000060140EC014E00E94794B80935F14115058
:10151000D1F78A3A11F082E03BC082E080936014F8
:1015200080916014823031F4C12CD12CE12C40E444
:10153000F42E03C0C12CD12C760120E030E0A901AB
:1015400067E38CE594E10E948B51A701960169E263
:101550008CE594E10E948B5180935F14882349F0BD
:101560000E94C9506C1B7D0B613D774030F38AE0CF
:101570000FC080916014823011F520E030E0A901A5
:101580006AE38CE594E10E948B51882351F088E056
:1015900080935D148CE594E10E94C550EBE4FAE37E
:1015A00019C00E94794B807C803C19F483E08093C1
:1015B00060140E94794B0E94794B0E94794B8CE514
:1015C00094E10E94C55010925E1481E018D78111F9
:1015D00031C015C08491EF012196882321F00E942B
:1015E000804BFE01F7CFE1EAFDE28491EF01219605
:1015F000882309F456C00E94804BFE01F6CF80E09C
:10160000FED6811117C0E4E1FAE38491EF0121963F
:10161000882321F00E94804BFE01F7CFEDE8FDE228
:101620008491EF012196882309F43BC00E94804BEE
:10163000FE01F6CF61E674E189EE92E10E945096D8
:10164000811116C0E4E1FAE38491EF012196882329
:1016500021F00E94804BFE01F7CFECE7FDE2849180
:10166000EF0121968823E9F00E94804BFE01F7CF1D
:1016700081E080939212EBE4FAE38491EF012196EA
:10168000882321F00E94804BFE01F7CFE0E7FDE2C6
:101690008491EF012196882321F00E94804BFE0166
:1016A000F7CF8BE1E9EEF2E1AAE0B3E101900D9210
:1016B0008A95E1F78091E7129091E81290930913CF
:1016C0008093081385EE92E19093051380930413A1
:1016D000DF91CF911F91FF90EF90DF90CF90089511
:1016E000FC0123812111A4CE08952F923F924F92A5
:1016F0005F926F927F928F929F92AF92BF92CF92A2
:10170000DF92EF92FF920F931F93CF93DF93CDB7AA
:10171000DEB7C454D1090FB6F894DEBF0FBECDBFFB
:101720004C015B017A01322E1C8E1F8E19821C82A5
:101730006115710511F410E0ACC0FC0183818111C9
:10174000FACFFA0180818F3261F4CA017C010196DF
:10175000F70120812F32D1F3F5018381825082304D
:1017600010F465010BC0618D728DCE0101960E944F
:101770005096882301F3CE0101966C018E01045E20
:101780001F4F280157E3652E712C6C0E7D1E9BE0C8
:10179000690E711CFE0131962496FFAFEEAF2497BF
:1017A00025960FAF2597212E35C080E28193E6154F
:1017B000F705D9F7D70120E097E04A2F3B2F8D910D
:1017C00081112BC08FA9803209F4B5CF842F932FBC
:1017D0007C01FC01208101962F32D1F3222309F4F0
:1017E00050C021E0AE01495C5F4FB601C8019ADAF2
:1017F000882309F4A0CFCA14DB0411F0C60118DE57
:1018000004151505B9F125969FAD2597822D680120
:10181000092F182FFE01F796C8CF8F3299F28E321A
:1018200019F0EFEAFDE20AC09A3009F484CF28E00B
:101830009AE0C3CF3196381709F47DCF3491311136
:10184000F9CF921708F477CF813208F474CF8F372D
:1018500009F471CF31E0320FE7E3F0E0EC0FFD1F48
:10186000E20FF11D2FE9280F2A3108F480528083FE
:10187000232FA3CF23969FAD239724968FAD249734
:10188000C6CF232DAE01495C5F4FB601C4014ADAD1
:10189000182FCE01019624DFCE014C9621DF812F37
:1018A000CC5BDF4F0FB6F894DEBF0FBECDBFDF912C
:1018B000CF911F910F91FF90EF90DF90CF90BF904D
:1018C000AF909F908F907F906F905F904F903F90E0
:1018D0002F90089527E033E0FC01318320830496A4
:1018E000FFCE2F923F924F925F926F927F928F9294
:1018F0009F92AF92BF92CF92DF92EF92FF920F939F
:101900001F93CF93DF93CDB7DEB7C057D1090FB682
:10191000F894DEBF0FBECDBF7C016B014A012DB72D
:101920003EB7AF963FAF2EAFAF97AD961FAEAD9718
:1019300034E0C30ED11C8E01015A1F4F77E0672E91
:1019400073E0772EE0E42E2E312C2C0E3D1E84E029
:10195000280E311C41EA52E1BE016F5F7F4FC60184
:101960000E94CB9418160CF057C12C85922F9871B9
:10197000903109F0CDC080913D158150823008F43E
:10198000C7C04DB65EB6BE016F5F7F4FC8010E94F3
:101990009C4481E0F70190819111B2C0E1E0F0E058
:1019A000D8010D900020E9F7E01BF10BEA0FFB1FB7
:1019B00031962DB73EB72E1B3F0B0FB6F8943EBFA6
:1019C0000FBE2DBFEDB7FEB731965F01882319F02A
:1019D00066E973E001C0B701C5010F949E08B80124
:1019E000C5010F94880866E973E0C5010F94880863
:1019F00025961FAE259728961FAE289724961FAED2
:101A00001EAE249722967FAE6EAE229721E0A801EB
:101A1000B601C1016ADE81114DC080913D15811171
:101A200049C0EBE4FAE384919F012F5F3F4F882385
:101A300081F0E0962FAFE097E1963FAFE1970E94EB
:101A4000804BE0962FADE097E1963FADE197F9012D
:101A5000EACFEFEBFDE284919F012F5F3F4F8111B1
:101A600002C0980110C0E0962FAFE097E1963FAF1B
:101A7000E1970E94804BE0962FADE097E1963FAD55
:101A8000E197F901E8CFF90181919F01882379F06D
:101A9000E0962FAFE097E1963FAFE1970E94804B31
:101AA000E1963FADE197E0962FADE097ECCF8AE06D
:101AB0000E94804B8BE1FE01EC5BFF4FDE019596AF
:101AC00001900D928A95E1F724968EAD9FAD2497F3
:101AD0009CA38BA37AA269A240E050E0BE016F5D97
:101AE0007F4FC501FEDECE018196F4DECE01805C23
:101AF0009F4FF0DE0FB6F8945EBE0FBE4DBE2ACFEC
:101B000080E001900020E9F73197EE19FF0948CFF6
:101B10008981882309F480C0853E09F41BCF8E3269
:101B200009F418CF8091A1128E3209F413CF2A70D4
:101B300009F010CF81E0903109F080E0809393129A
:101B4000811108C08985873409F004CF8A858E37D2
:101B500009F400CF80913D15813021F068F082308A
:101B6000A9F1F8CE80913E1590913F150196909382
:101B70003F1580933E15EECEBE016F5F7F4F84E927
:101B800092E10E949C445701F50181915F018823F5
:101B900019F00E94804BF8CF64E9A62E62E1B62EC0
:101BA000F50181915F01882319F00E94804BF8CFE5
:101BB00080E20E94804B6D8D7E8D8F8D98A14AE0D2
:101BC0000E94916F8AE00E94804BC4CEBE016F5F7D
:101BD0007F4F84E992E10E949C448114910441F07A
:101BE00064E972E1C4010F947508892B69F414C08B
:101BF000AD96FFADAD972F2F30E080913E159091BF
:101C00003F152817390741F0AD963FADAD973F5FBF
